:020000040800F2
:100000000000012055880308A1880308CDD200080C
:10001000A1880308A1880308A18803080000000044
:10002000000000000000000000000000A18803089C
:10003000A188030800000000A188030869D1000816
:10004000A1880308A1880308A1880308A1880308E0
:10005000A1880308A18803081D910108499201089D
:100060000D920108D1910108959101085DB1000838
:100070004DB100083DB100082DB100081DB10008C8
:1000800009B10008F5B00008A1880308A188030899
:10009000A1880308A1880308A188030859910108D1
:1000A000A1880308A1880308A1880308A188030880
:1000B000A188030865A40008A1880308A188030893
:1000C000A1880308A1880308A1880308A188030860
:1000D000A1880308C99A0008BD9A0008B19A0008CF
:1000E000E1900108A1880308A1880308A1880308FA
:1000F00051A40008A188030841A40008E1B0000849
:10010000A1880308A188030855A40008A188030852
:10011000A59A0008999A0008A18803089D7A030807
:10012000CDB00008B9B00008A5B0000891B0000833
:100130007DB000080000000000000000000000008A
:100140000000000000000000000000000D40020858
:1001500069B0000855B0000841B00008A188030844
:10016000A1880308A1880308A1880308A1880308BF
:10017000A1880308A1880308000000000000000017
:10018000A1880308A1880308A1880308A18803089F
:10019000A1880308A188030800000000A1880308C3
:1001A000000000000000000000000000A18803081B
:1001B000A1880308A18803080000000000000000D7
:1001C000000000000000000000000000000000002F
:1001D000000000000000000000000000A1880308EB
:1001E0000C02010038250120342501200000000008
:1001F0002C06000816000800442501204C2501208B
:10020000000000002E060008270004002C29012011
:10021000342A0120000000003606000803123300D3
:10022000B72C0120842C0120000000003C060008AF
:1002300025005A00D02B01202A2C012000000000AC
:1002400000000000F6110C00C42B0120B82B012087
:10025000000000007006000801200800002D0120A9
:100260004C2D0120000000007C06000829005000F1
:100270001C2F012048330120000000000000000076
:1002800014000200182F0120983301200000000004
:100290008406000810000300A82E01209C330120D2
:1002A000000000008606000828000C009C2E01209B
:1002B000A0330120000000008A060008230010007F
:1002C0008C2E0120AC33012000000000C5890208FB
:1002D00019000500842E0120BC330120000000001D
:1002E00096060008F8110100802E0120C433012079
:1002F000000000009C060008000104007C2E012084
:10030000C8330120000000009E0600082F001100E5
:10031000682E0120CC33012000000000A206000856
:10032000050006001636012090360120000000006E
:10033000B40600080C002400DE35012098360120A8
:1003400000000000792A02080E20EA00D6340120BD
:10035000BC360120000000001DCA02081300040082
:1003600048360120A837012000000000BC06000824
:1003700012100B00B6340120AC3701200000000041
:10038000C006000802010300B1340120B837012083
:1003900000000000A12A0208F5116200F6330120D6
:1003A000BC370120000000000180000801020500A8
:1003B000403A0120DC4D0120000000005D120208DF
:1003C0000002050020380120E44D0120000000005B
:1003D000000000001E0004008C3E0120EC4D0120B6
:1003E00000000000CC06000801010400304E01208E
:1003F000BC6E0120000000000000000008020C009C
:10040000326B0120C06E01200000000079890108D4
:1004100002000C00A06E0120CC6E01200000000044
:1004200000000000F70106002C6B0120D86E0120AF
:1004300000000000D00600081F000E00FC73012021
:10044000D875012000000000D60600080502010052
:10045000E4730120E875012000000000E4060008B4
:10046000F9010400E07F0120E47F0120000000008A
:10047000DDB50008FD011E00C07F0120E87F0120DE
:100480000000000069B5000818102C00707F0120E2
:100490000880012000000000599E0208FB010100B5
:1004A000387F0120348001200000000025B50008BD
:1004B000FC010900047E01203880012000000000BA
:1004C000F1B400080A101200EC75012044800120EC
:1004D00000000000E60600081B00F4003482012042
:1004E0002883012000000000E949030826000E00CF
:1004F0002C8401201C84012000000000317B0208B4
:100500000B201000CC8001203C8401200000000062
:10051000F80600082C00100064890120548901208D
:10052000000000001D9302082B0024009889012080
:100530007489012000000000ED920208030106000A
:10054000F4890120088A0120000000000807000843
:100550001A000800049101201C91012000000000F5
:100560000E07000815007000088B0120249101205F
:10057000000000000000000003000100048B0120C7
:100580009491012000000000000000002A0060009B
:10059000148A01209891012000000000A9C90208D6
:1005A0000600160030940120609C0120000000002D
:1005B0003DCA0208340010006C920120789C012092
:1005C00000000000D1C902080A020A00509D012063
:1005D000609D0120000000001607000822000C00AA
:1005E000489F0120CC9F0120000000002007000848
:1005F0000D003400DCA3012010A401200000000045
:10060000E9F9020802020300D0A3012044A401205A
:1006100000000000000000000400800058BB012022
:0C062000A4BD012000000000000000004C
:10062C000100C40900001901282820030000000063
:10063C0000000000000000000000000000000000AE
:10064C00000000000000000000000000000000009E
:10065C00000000000000000000000000000000008E
:10066C00000001000000000000000000000000007D
:10067C00E8036400040A0001030000010500000007
:10068C000001000000000000000000002801000034
:10069C0004009001000000000000000000000000B9
:1006AC00000000000000000020000300010000001A
:1006BC0018200000000000010041574637000000E0
:1006CC00000001001201000000000000000000000A
:1006DC000100000000050000000000300100005A7D
:1006EC000000000090012C01C80064002B21231E87
:1006FC0064000200000001000A012900040101004D
:10070C0000007E05EA05B405320000004A01B40081
:10071C00D6010000C800141E010064002C01280042
:10072C000000803F0000803F0000803F010000007F
:10073C0001010000BCE703085C2104080000000074
:10074C0000000000CCE70308D4E703080000000019
:10075C0001200000D8E70308E0E7030800000000D0
:10076C0001400000E4E703087CFC030800000000E3
:10077C0001200000F0E70308FCE70308000000007C
:10078C000400000000E80308E41604080000000060
:10079C00040000000CE803084010040800000000EE
:1007AC0001000000020100000000803F0000803FBB
:1007BC00FF0100000000803F00600240106002401A
:1007CC0000000000000B00000000200000000000F2
:1007DC0000000000006002402860024000000000A1
:1007EC00060C0000000020000000000000000000CB
:1007FC00006002404060024000000000100D00004C
:10080C00000020000000000000000000006002401A
:10081C005860024000000000160E0000000020008E
:10082C000000000000000000006002407060024008
:10083C0000000000200F000000002000000000005D
:10084C0000000000006002408860024000000000D0
:10085C002610000000002000000000000000000036
:10086C0000600240A0600240000000003011000057
:10087C0000002000000000000000000000600240AA
:10088C00B860024000000000362F0000000020007D
:10089C0000000000000000000064024010640240F0
:1008AC0000000000003800000000400000000000C4
:1008BC0000000000006402402864024000000000B8
:1008CC00063900000000400000000000000000009D
:1008DC00006402404064024000000000103A000036
:1008EC000000400000000000000000000064024016
:1008FC005864024000000000163B0000000040005D
:10090C00000000000000000000640240706402401F
:10091C0000000000203C000000004000000000002F
:10092C0000000000006402408864024000000000E7
:10093C002644000000004000000000000000000001
:10094C0000640240A064024000000000304500003A
:10095C0000004000000000000000000000640240A5
:10096C00B864024000000000364600000000400061
:10097C000000000000000000FFFFFFFF30303030AF
:10098C002D30312D30315430303A30303A30300057
:10099C0000010101010000000101010040200408D8
:1009AC000F00000091FB0108000000000000000097
:1009BC00FC030120142004080000000000000000CB
:1009CC0000000000000000005C2104080000000092
:1009DC0000000000B004012004000000941F040873
:1009EC000D00000005030208F01C012000000000AF
:1009FC00501904080D000000D5020208E41C012067
:100A0C0000000000341A0408080000000000000078
:100A1C00D81C012004000000B01904080D000000CF
:100A2C00ED010208CC1C012000000000441A04084F
:100A3C00030000008D660308B41C012000000000B8
:100A4C0024200408030000008D6603089C1C012070
:100A5C00000000000817040801000000000000005E
:100A6C000000000000000000000000000E0000006C
:100A7C00000000000000000000000000142004082A
:100A8C00000000000000000000000000000000005A
:100A9C005C2104080000000000000000B0040120EC
:100AAC0004000000401F0408030000003D01020880
:100ABC00841C012008000000B01904080D0000007F
:100ACC00ED010208CC1C012000000000441A0408AF
:100ADC00030000008D660308B41C01200000000018
:100AEC0024200408030000008D6603089C1C0120D0
:100AFC0000000000081704080100000000000000BE
:100B0C000000000000000000000000000E000000CB
:100B1C000000000000000000000000002C20040871
:100B2C0000000000000000000000000000000000B9
:100B3C005C2104080000000000000000B00401204B
:100B4C0004000000481F0408030000008D66030821
:100B5C00FC1C012000000000081704080100000024
:100B6C000000000000000000000000000000000079
:100B7C000E0000000000000000000000000000005B
:100B8C0020700020702D7200082004080F00000057
:100B9C0000000000000000000000000034180120DC
:100BAC00FFFFFFFFFA000000010000000100000041
:100BBC002D202D2D202D2D2D2D202D2D2D2D0000DA
:100BCC000000000000000000000000000000000019
:100BDC002D202D2D202D2D2D2D202D2D2D000000E7
:100BEC0000000000000000000000000000000000F9
:100BFC00CC160408D41604080017040800000000E2
:100C0C000000000000000000000000009D16040819
:100C1C0004000000CD0002080000000000000000ED
:100C2C00081704080100000000000000000000008C
:100C3C0000000000000000000E000000000000009A
:100C4C0000000000000000006A9E01200100C409A1
:100C5C0000000000689E01200100C4090000000093
:100C6C00669E01200100C40900000000649E012062
:100C7C000100C40900000000609E01200100C409AD
:100C8C0000000000629E01200100C4090000000069
:100C9C005E9E01200100C409000000005C9E012042
:100CAC000100C40900000000623401200100C800EA
:100CBC000100000060340120320030753200000069
:100CCC005E340120055A05005934012000FF010053
:100CDC005D34012001000000D00401205B340120B0
:100CEC0002000000D0D403085834012000FF01009A
:100CFC005C34012001000000D00401205A34012092
:100D0C0002000000D0D403083C1704080F000000B8
:100D1C00000000000000000000000000D8040120CA
:100D2C00F08901209CFF2C01000000007A020120B8
:100D3C000A000000DCD40308E0330120E0150C1796
:100D4C00000000007902012008000000ACD4030868
:100D5C007802012005000000C0D50308E233012011
:100D6C0002000000F4D403081C3601200100FF7FB0
:100D7C0001000000143601200200000000D5030819
:100D8C00C53401200300000010D50308C434012031
:100D9C000300000010D50308C83501200000F40141
:100DAC0001000000C63501200000F4010100000024
:100DBC00C43501200000F40101000000C2350120FF
:100DCC000000F40101000000C035012000FF01000B
:100DDC00DC350120E803D0070A000000DA350120D9
:100DEC00006401000A000000DB35012000640100F2
:100DFC000A000000D4350120006401000A00000044
:100E0C00D9350120006401000A000000D83501200A
:100E1C00006401000A000000D735012000640100C5
:100E2C000A000000D335012000FF01000A00000079
:100E3C00D235012000FF01000A000000D23401204D
:100E4C000000F40101000000D03401200000F40186
:100E5C0001000000CE3401200000F401010000006C
:100E6C00CC3401200000F40101000000CF3501203A
:100E7C0000C80100CE35012000C80100CD3501208D
:100E8C0000C80100CC350120006401000A000000FC
:100E9C00CB35012000FF01000A0000000B360120B9
:100EAC0000C801000A36012000C8010009360120E3
:100EBC0000C801000836012000C8010007360120D7
:100ECC0000C801000636012000C8010005360120CB
:100EDC0000C801000436012000C8010003360120BF
:100EEC0000C80100441704080000000000000000C6
:100EFC000000000000000000541704080900000066
:100F0C00000000007C050120040000005C170408B0
:100F1C000900000000000000700501200400000022
:100F2C00F81C040809000000000000006405012002
:100F3C000400000000E703080900000000000000A6
:100F4C005805012004000000641704080900000083
:100F5C00000000004C050120040000006C17040880
:100F6C000900000000000000400501200400000002
:100F7C00741704080900000000000000340501206B
:100F8C00040000007C1704080900000000000000A9
:100F9C0028050120040000000817040801000000C7
:100FAC000000000000000000000000000000000035
:100FBC000E00000000000000000000000000000017
:100FCC00541804080000000000000000000000009D
:100FDC0000000000F4E90308070000000000000016
:100FEC00A00501200000000064180408080000009F
:100FFC000000000094050120000000007018040897
:10100C00080000000000000088050120000000001E
:10101C000817040801000000000000000000000098
:10102C0000000000000000000E00000000000000A6
:10103C000000000000000000781804080000000008
:10104C0000000000000000000000000088180408E8
:10105C000D00000000000000DC0501200000000075
:10106C00901804080D00000000000000D0050120BD
:10107C0000000000981804080700000000000000A1
:10108C00C805012000000000A01804080D00000095
:10109C0000000000BC05012000000000A818040896
:1010AC000D00000000000000B00501200000000051
:1010BC00B01804080700000000000000A80501207B
:1010CC0000000000081704080100000000000000E8
:1010DC000000000000000000000000000E000000F6
:1010EC00000000000000000000000000B818040818
:1010FC0000000000000000000000000000000000E4
:10110C00F4E903080C000000000000006434012026
:10111C0000000000CC1804080C00000000000000C7
:10112C006634012000000000DC1804080C000000EC
:10113C00000000009C34012000000000EC180408A2
:10114C000C000000000000009034012000000000A2
:10115C00001904080C000000000000006834012095
:10116C00000000000C1904080C0000000000000036
:10117C006A34012000000000141904080C0000005F
:10118C00000000006C340120000000002819040845
:10119C000C000000000000006E3401200000000074
:1011AC00301904080C00000000000000703401200D
:1011BC0000000000381904080C00000000000000BA
:1011CC007234012000000000441904080C000000D7
:1011DC00000000007434012000000000C006040868
:1011EC000C0000000000000076340120000000001C
:1011FC004C1904080C000000000000007834012099
:10120C0000000000581904080C0000000000000049
:10121C007A3401200000000008EA03080C000000EA
:10122C00000000007C340120000000006419040858
:10123C000C000000000000007E34012000000000C3
:10124C00701904080C00000000000000803401201C
:10125C00000000007C1904080C00000000000000D5
:10126C009434012000000000841904080C000000D4
:10127C000000000092340120000000008C190408CA
:10128C000C00000000000000A03401200000000051
:10129C00981904080C00000000000000A234012082
:1012AC0000000000A41904080C000000000000005D
:1012BC00A83401200000000024EA03080C00000000
:1012CC00000000008234012000000000B019040866
:1012DC000C000000000000008A3401200000000017
:1012EC00B81904080C000000000000008434012030
:1012FC0000000000C41904080C00000000000000ED
:10130C008634012000000000D01904080C000000F5
:10131C00000000008834012000000000D8190408E7
:10132C000C000000000000008C34012000000000C4
:10133C00940704080C000000000000009634012003
:10134C0000000000E41904080C000000000000007C
:10135C008E3401200000000078E703080C00000028
:10136C00000000009E34012000000000F019040869
:10137C000C00000000000000983401200000000068
:10138C00F81904080C000000000000009A34012039
:10139C0000000000001A04080C000000000000000F
:1013AC00A434012000000000081A04080C000000FE
:1013BC0000000000A63401200000000008170408FB
:1013CC000100000000000000000000000000000010
:1013DC00000000000E0000000000000000000000F3
:1013EC0000000000101A04080000000000000000BB
:1013FC000000000000000000201A04080500000096
:10140C0000000000C334012000000000081704088D
:10141C0001000000000000000000000000000000BF
:10142C00000000000E0000000000000000000000A2
:10143C0000000000281A0408000000000000000052
:10144C0000000000000000005C2104080000000007
:10145C00000000009004012004000000FCE60308DA
:10146C000D000000150102083C06012000000000E0
:10147C00941F04080D0000003DFB010830060120FC
:10148C0000000000501904080D00000009FB0108C1
:10149C002406012000000000341A04080800000093
:1014AC00000000001806012004000000B019040818
:1014BC000D000000F5FA01080C06012000000000E8
:1014CC003C1A04080900000000000000000601207E
:1014DC0004000000441A0408030000008D66030891
:1014EC00E8050120000000000817040801000000B6
:1014FC0000000000000000000000000000000000E0
:10150C000E000000000000000000000000000000C1
:10151C00481A040800000000000000000000000051
:10152C0000000000581A04080D0000000000000024
:10153C005406012000000000601A04080A00000094
:10154C00000000002D360120000000006C1A040879
:10155C000A000000000000003536012000000000E9
:10156C00741A04080A000000000000003D36012037
:10157C00000000007C1A04080800000000000000B5
:10158C0048060120000000000817040801000000B4
:10159C00000000000000000000000000000000003F
:1015AC000E00000000000000000000000000000021
:1015BC00841A040800000000000000000000000075
:1015CC0000000000981A04080D0000000000000044
:1015DC006C06012000000000A81A0408040000009A
:1015EC00FD0302080000000000000000B01A04080F
:1015FC000D0000000000000060060120000000004B
:10160C00C41A040804000000DD03020800000000F6
:10161C000000000008170408010000000000000092
:10162C000000000000000000000000000E000000A0
:10163C00000000000000000000000000CC1A0408AC
:10164C00000000000000000000000000000000008E
:10165C00E01A04080700000000000000A8060120A2
:10166C0000000000EC1A0408080000000000000054
:10167C009C06012000000000F81A04080800000075
:10168C00000000009006012000000000041B04086C
:10169C00080000000000000084060120000000008B
:1016AC00101B040808000000000000007806012050
:1016BC0000000000081704080100000000000000F2
:1016CC000000000000000000000000000E00000000
:1016DC000000000000000000000000001C1B0408BB
:1016EC000000000000000000630401200000000066
:1016FC00281B04080B00000000000000100701204C
:10170C0000000000301B04080B000000000000006B
:10171C0004070120000000003C1B04080B00000023
:10172C0000000000F806012000000000481B04081F
:10173C000B00000000000000EC060120000000007F
:10174C00541B04080B00000000000000E006012000
:10175C0000000000601B04080B00000000000000EB
:10176C00D406012000000000681B04080B000000D8
:10177C0000000000C806012000000000741B0408D3
:10178C000B00000000000000BC060120000000005F
:10179C00801B04080800000000000000B0060120B7
:1017AC000000000008170408010000000000000001
:1017BC000000000000000000000000000E0000000F
:1017CC000000000000000000000000008C1B04085A
:1017DC0000000000000000000000000000000000FD
:1017EC00A01B0408080000000000000040070120B6
:1017FC0000000000AC1B0408080000000000000002
:10180C003407012000000000B81B04080800000089
:10181C00000000002807012000000000C41B040881
:10182C0008000000000000001C0701200000000060
:10183C000817040801000000000000000000000070
:10184C0000000000000000000E000000000000007E
:10185C000000000000000000CC1B04080000000089
:10186C00000000006004012000000000DC1B0408E4
:10187C000B000000000000007007012000000000B9
:10188C00E81B04080B0000000000000064070120A6
:10189C0000000000F41B040807000000000000001A
:1018AC005C07012000000000001C04080700000079
:1018BC000000000054070120000000000C1C04086C
:1018CC0007000000000000004C0701200000000091
:1018DC0008170408010000000000000000000000D0
:1018EC0000000000000000000E00000000000000DE
:1018FC000000000000000000181C0408000000009C
:10190C00000000006004012000000000241C0408FA
:10191C000700000000000000BC07012000000000D0
:10192C002C1C04080700000000000000B407012074
:10193C0000000000341C0408070000000000000038
:10194C00AC070120000000003C1C0408070000004C
:10195C0000000000A407012000000000441C040843
:10196C0007000000000000009C07012000000000A0
:10197C004C1C040807000000000000009407012024
:10198C0000000000541C04080700000000000000C8
:10199C008C070120000000005C1C040807000000FC
:1019AC00000000008407012000000000641C0408F3
:1019BC0007000000000000007C0701200000000070
:1019CC0008170408010000000000000000000000DF
:1019DC0000000000000000000E00000000000000ED
:1019EC0000000000000000006C1C04080F00000048
:1019FC000000000011FE010800000000C4070120D7
:101A0C00C13401201700000020D50308B534012093
:101A1C000A320100B434012001FA0100B034012073
:101A2C0000C80100AE340120E803D007010000001B
:101A3C00414C49454E57484F4F5046370000000027
:101A4C00F433012000030100F333012000030100F3
:101A5C00741C04080F0000003DFD010819FD01086D
:101A6C0000000000A0080120801C04080F000000EA
:101A7C00D9FC010891FC01080000000018090120A4
:101A8C008C1C04080F00000079FD010861FD0108A1
:101A9C0000000000CC090120981C04080F00000075
:101AAC0027FE010800000000AD030208C40C012051
:101ABC00A01C04080F00000055FA010800000000EB
:101ACC0000000000140D0120A81C04080F000000E9
:101ADC007D0102087D00020879000208F00D01204A
:101AEC00B01C04080F0000004DFE010800000000AF
:101AFC0000000000900E0120B81C04080F0000002C
:101B0C00EDFE0108BDFE0108000000001C0F0120C5
:101B1C00C01C04080F00000069FF0108B1FF010898
:101B2C0000000000BC0F0120D03501200103010092
:101B3C00CC1C04080F00000089FE010861FE01089E
:101B4C0000000000AC100120D41C04080F000000A1
:101B5C001DFF01081D0402080000000038110120BF
:101B6C00E01C04080F000000DDFF010865040208FA
:101B7C0000000000D8110120CA350120010301002A
:101B8C00E81C040800000000000000000000000039
:101B9C0000000000F41C0408080000000000000015
:101BAC000413012000000000FC1C040807000000C6
:101BBC0000000000FC120120000000000C1D0408B5
:101BCC000700000000000000F412012000000000DB
:101BDC00181D04080700000000000000EC12012092
:101BEC0000000000241D04080D000000000000008F
:101BFC00E012012000000000301D0408030000006A
:101C0C008D660308C81201200000000008170408A4
:101C1C0001000000000000000000000000000000B7
:101C2C00000000000E00000000000000000000009A
:101C3C0000000000381D0408000000000000000037
:101C4C000000000000000000481D04080A0000000D
:101C5C000000000018E8030800000000501D0408F4
:101C6C000A000000000000009CE7030800000000D0
:101C7C00581D04080A000000000000000C3601206A
:101C8C0000000000601D04080A00000000000000B5
:101C9C0010130120000000000817040801000000C8
:101CAC000000000000000000000000000000000028
:101CBC000E0000000000000000000000000000000A
:101CCC00681D040800000000000000000000000077
:101CDC0000000000741D0408030000008D6603085A
:101CEC006013012000000000841C040803000000A5
:101CFC008D6603084813012000000000781C0408BE
:101D0C00030000008D660308301301200000000062
:101D1C00801D04080500000000000000F2330120C3
:101D2C0000000000881D04080700000000000000EF
:101D3C002813012000000000941D04080700000077
:101D4C000000000020130120000000000817040808
:101D5C000100000000000000000000000000000076
:101D6C00000000000E000000000000000000000059
:101D7C0000000000A01D040800000000000000008E
:101D8C00000000000000000038EA03080300000017
:101D9C008D660308A813012000000000B41D040880
:101DAC00030000008D6603087C0201200000000087
:101DBC00BC1D0408030000008D660308901301206D
:101DCC0000000000C41D0408030000008D66030819
:101DDC00781301200000000008170408010000001F
:101DEC0000000000000000000000000000000000E7
:101DFC000E000000000000000000000000000000C9
:101E0C00D01D0408000000000000000000000000CD
:101E1C0000000000DC1D040807000000B1040208EB
:101E2C005814012000000000D4190408030000001D
:101E3C008D6603084014012000000000E81D040812
:101E4C00030000008D660308281401200000000028
:101E5C00F01D0408030000008D6603081014012017
:101E6C0000000000F81D040807000000950402089B
:101E7C000814012000000000B01F0408030000003B
:101E8C008D660308F013012000000000041E0408F6
:101E9C00030000008D660308D81301200000000029
:101EAC00101E0408030000008D660308C0130120F7
:101EBC0000000000081704080100000000000000EA
:101ECC000000000000000000000000000E000000F8
:101EDC000000000000000000000000001C1E0408B0
:101EEC000F000000D1FD010891FD01080000000069
:101EFC0060140120241E04080F0000004D0002088D
:101F0C00000000000000000014150120301E040821
:101F1C000F00000075FC010859FC010800000000CE
:101F2C00A0150120381E04080F000000000000005E
:101F3C00000000000000000054160120481E040898
:101F4C000F00000025000208CD040208000000006C
:101F5C00E0160120501E04080000000000000000E4
:101F6C0000000000000000005C1E040803000000DC
:101F7C008D6603081C180120000000003C1E04089C
:101F8C00030000008D660308041801200000000007
:101F9C00341E0408030000008D660308EC170120B2
:101FAC0000000000641E0408030000008D66030896
:101FBC00D417012000000000701E0408030000006C
:101FCC008D660308BC17012000000000781E040871
:101FDC0002000000E90402080000000000000000FC
:101FEC00801E040802000000E90402080100000041
:101FFC00000000008C1E040802000000E904020826
:10200C000200000000000000000000000E000000B4
:10201C00000000000000000000000000EE33012072
:10202C0088130C1701000000F033012088130C17E3
:10203C0000000000981E04080000000000000000D2
:10204C000000000000000000A81E040808000000AA
:10205C00000000000819012004000000B41E040850
:10206C000800000000000000FC1801200000000027
:10207C00441A040804000000D1010208000000000A
:10208C000000000008170408010000000000000018
:10209C000000000000000000000000000E00000026
:1020AC00000000000000000000000000EC330120E4
:1020BC0088130C1701000000EA33012088130C1759
:1020CC0000000000F01E04080F000000E9FB0108EE
:1020DC000000000000000000141901204636012009
:1020EC000100000080D50308E93301200100000045
:1020FC008CD50308E07301200200000094D503087E
:10210C000EBC012000000000000000000CBC0120EF
:10211C0000000000000000000ABC012000000000CC
:10212C000000000008BC01200000000000000000BE
:10213C0006BC0120000000000000000004BC0120CF
:10214C000000000000000000981D012000000000AD
:10215C0000000000E833012002000000A0D50308B5
:10216C00F81E040800000000000000000000000041
:10217C0000000000A81E0408080000000000000079
:10218C009819012004000000B41E04080800000087
:10219C00000000008C19012000000000441A040803
:1021AC0004000000C9FB0108000000000000000052
:1021BC0008170408010000000000000000000000E7
:1021CC0000000000000000000E00000000000000F5
:1021DC000000000000000000081F040800000000C0
:1021EC00000000000000000000000000181F0408A0
:1021FC000D00000075020208D41901200400000033
:10220C00241F04080D0000000DFC0108C819012052
:10221C0004000000301F04080D0000003502020805
:10222C00BC190120000000003C1F04080300000042
:10223C005D010208A419012008000000481F0408D1
:10224C00030000008D660308FC1C01200000000048
:10225C000817040801000000000000000000000046
:10226C0000000000000000000E0000000000000054
:10227C00000000000000000000170408000000002F
:10228C000000000000000000000000009D16040883
:10229C0004000000350302080000000000000000EC
:1022AC0008170408010000000000000000000000F6
:1022BC0000000000000000000E0000000000000004
:1022CC0000000000000000009C1F0408000000003B
:1022DC00000000000000000000000000340A0408A8
:1022EC000D00000000000000341A01200400000062
:1022FC00AC1F04080800000000000000281A012090
:10230C0004000000B81F04080800000000000000D2
:10231C001C1A012004000000C01F04080800000063
:10232C0000000000101A012004000000C81F04085F
:10233C000800000000000000041A01200400000046
:10234C00D01F04080800000000000000F81901204C
:10235C0004000000D81F0408080000000000000062
:10236C00EC19012004000000E01F04080800000024
:10237C0000000000E0190120040000000817040808
:10238C000100000000000000000000000000000040
:10239C00000000000E000000000000000000000023
:1023AC0000000000E81F04080F000000D9FB010822
:1023BC000000000000000000401A0120F01F04087B
:1023CC000F000000000000000000000000000000F2
:1023DC00B81A0120F81F04080F00000000000000CC
:1023EC000000000000000000581B012045360120B1
:1023FC0004000000ACD50308E4330120E0150C17F1
:10240C0000000000E733012008000000ACD40308F2
:10241C00E633012005000000C0D5030800200408A5
:10242C000F00000000000000000000000000000091
:10243C00A81B0120E0010800A8D803080508040027
:10244C0000000000C0D50308ACD4030894D80308DE
:10245C0000000000D4D8030805080A0000000000A2
:10246C00C0D50308ACD40308DCD40308000000007A
:10247C001A03000000000000000000000000000033
:10248C0000000000000000000000000000FFFF0042
:10249C0000000000AA5503009FAA5505010000AAE0
:1024AC00550701000001AA550B010000AA550902AD
:1024BC000000000001000000C0120100C007040869
:1024CC000000000000000000B52A0208A0860100F0
:1024DC0004000000000000000000000000000000EC
:1024EC0000000000000000000000000000000000E0
:1024FC00D41904081407040800000000511701083F
:10250C007D0000000600000000000000000000003C
:10251C0000000000000000000000000000000000AF
:10252C0000000000C82104080000000000000000AA
:10253C004D370308E8030000030000000000000012
:10254C00000000000000000000000000000000007F
:10255C000000000000000000D02104080000000072
:10256C0000000000A1AC01081027000003000000CF
:10257C00000000000000000000000000000000004F
:10258C0000000000000000000000000044180408D7
:10259C0000000000759102080D670108204E000034
:1025AC00050000000000000000000000000000001A
:1025BC00000000000000000000000000000000000F
:1025CC00340904080000000000000000E531030895
:1025DC0010270000010000000000000000000000B7
:1025EC0000000000000000000000000000000000DF
:1025FC0000000000DC2104080000000000000000C6
:10260C00BDB40008E8030000050000000000000055
:10261C0000000000000000000000000000000000AE
:10262C000000000000000000E82104080000000089
:10263C0000000000B12C0208204E00000300000036
:10264C00000000000000000000000000000000007E
:10265C00000000000000000000000000F821040849
:10266C000000000000000000E52A0208204E0000D7
:10267C00030000000000000000000000000000004B
:10268C00000000000000000000000000000000003E
:10269C000822040800000000000000006D2F030851
:1026AC00400D0300030000000000000000000000CB
:1026BC00000000000000000000000000000000000E
:1026CC000000000074080408000000000000000076
:1026DC00B1060308102700000100000000000000F4
:1026EC0000000000000000000000000000000000DE
:1026FC00000000000000000030070408000000008B
:10270C0000000000051F0208102700000300000055
:10271C0000000000000000000000000000000000AD
:10272C000000000000000000000000001822040857
:10273C0000000000000000007D7C0308A086010062
:10274C00010000000000000000000000000000007C
:10275C00000000000000000000000000000000006D
:10276C003C09040800000000000000001DD3000814
:10277C00A00F00000100000000000000000000009D
:10278C00000000000000000000000000000000003D
:10279C0000000000202204080000000000000000DF
:1027AC00B9430308102700000100000000000000DE
:1027BC00000000000000000000000000000000000D
:1027CC000000000000000000341E0408000000009F
:1027DC0000000000899F01081A4100000100000060
:1027EC0000000000000000000000000000000000DD
:1027FC00000000000000000000000000A009040818
:10280C000000000000000000D94F02081027000053
:10281C0001000000000000000000000000000000AB
:10282C00000000000000000000000000000000009C
:10283C000C07040800000000000000004506020818
:10284C001A41000001000000000000000000000020
:10285C00000000000000000000000000000000006C
:10286C00000000002C220408000000000000000002
:10287C00C5F90208400D0300000000000000000034
:10288C00000000000000000000000000000000003C
:10289C0000000000000000003422040800000000CA
:1028AC000000000081F90208400D03000000000048
:1028BC00000000000000000000000000000000000C
:1028CC000000000000000000000000003C22040892
:1028DC000000000000000000992E0208A0860100F4
:1028EC0003000000000000000000000000000000D9
:1028FC0000000000000000000000000000000000CC
:10290C0001010000698F02080000000000000000B7
:10291C000403090412010002020000408304405722
:10292C0000020102030100000A0600020000004040
:10293C000100000009074300020104C03209040031
:10294C000001020201000524001001052401000110
:10295C00042402020524060001070582030800FF77
:10296C0009040100020A00000007050102400000F2
:10297C00070581024000000009024300020100C06B
:10298C0032090400000102020100052400100105B7
:10299C00240100010424020205240600010705821B
:1029AC000308001009040100020A000000070501D9
:1029BC000200020007058102000200000902430028
:1029CC00020100C0320904000001020201000524CA
:1029DC000010010524010001042402020524060054
:1029EC00010705820308001009040100020A000017
:1029FC0000070501024000000705810240000001AC
:102A0C0059B702084DB70208D53F0208E93F020842
:102A1C00653F0208C13F0208AD3F020805C9020824
:102A2C00DDB802087DC802080000000095B7020856
:102A3C00F1B70208BDB7020800000000000000005A
:102A4C00000000007DB7020889B7020871B70208C0
:102A5C0065B702087D730308F5710308A9710308B3
:102A6C009971030800000101FFFF00000000803F86
:102A7C0000E6DF0C00C2010000000800430000006B
:102A8C00000000000000000000000000000000003A
:102A9C0000000000000000000000000043000000E7
:102AAC00000000000000000000000000000000001A
:102ABC0000000000000000000000000043000000C7
:102ACC0000000000000000000000000000000000FA
:102ADC0000000000000000000000000043000000A7
:102AEC0000000000000000000000000000000000DA
:102AFC000000000000000000000000004300000087
:102B0C0000000000000000000000000000000000B9
:102B1C000000000000000000000000004300000066
:102B2C000000000000000000000000000000000099
:102B3C000000000000000000000000004300000046
:102B4C000000000000000000000000000000000079
:102B5C000000000000000000000000004990030885
:102B6C00898E030800000000C32504089816040889
:102B7C004D2304084D2304084D2304084D23040859
:102B8C004D2304084D2304084D2304084D23040849
:102B9C004D230408FFFFFFFFFFFFFFFFFFFFFFFFB9
:102BAC00FFFF0000010041534349490000000000B1
:102BBC000000000000000000000000000000000009
:102BCC000000000000004153434949000000000090
:102BDC0000000000000000000000000000000000E9
:102BEC000000000000000000CC24012000000000C8
:102BFC0000000000000000000000000000000000C9
:102C0C0000000000000000000000000000000000B8
:102C1C0000000000000000000000000000000000A8
:102C2C000000000000000000000000000000000098
:102C3C000000000000000000000000000000000088
:102C4C000000000000000000000000000100000077
:108000002DE9F04140F6280340F62C0240F63601F7
:1080100040F66A1440F6210740F64D1640F6E10599
:108020000380428040F6791340F681124181048238
:1080300040F6611140F6F7048781C68140F6DA0701
:1080400040F633064582838240F6A71540F6C713F3
:10805000C282018340F6E71240F64111C48340F624
:108060004C044783868340F6591740F64916058429
:10807000438440F6010540F601138284C18440F632
:10808000211240F64101848540F60A140785468591
:1080900040F62F1740F62E164586838640F6881543
:1080A00040F6C803C286018640F6520240F68A01B5
:1080B000A0F8444040F65304C787868740F6371837
:1080C000058740F6171C83804FF0013EC3804FF0B8
:1080D000011703814FF00126C28514230125418732
:1080E000A0F846202821A0F848400C4A0C4CA0F8E3
:1080F0004080A0F842C0C0F84AE0C0F84E70C0F816
:10810000526080F85B50C465C0F8562080F861105A
:1081100080F85A3080F86030BDE8F081980864003B
:10812000000A010A4FF40063038370474FF40063B1
:1081300003837047012250F8043CA0F1100180F83D
:1081400049200BB108461847704700BFD0F8F0200F
:10815000034630B46AB1C168D0F808214469881A6E
:10816000013A205C08BF0A46C0B2C3F8082130BCFF
:108170007047006A5D69411CDC68285CA14228BF29
:108180001146C0B2196230BC704700BFD0F8F4305D
:1081900013B190F888017047836A406A181AB0FAE0
:1081A00080F04009704700BF416A836A99420ED34C
:1081B000CB1AD0F8F410026981B1D0F87411501EB6
:1081C0000A685268134483420BD2C01A704702698E
:1081D0001144CB1AD0F8F4100029EED1501EC01A69
:1081E00070470020704700BFD0F8F0306BB1D0F876
:1081F0007831D0F808211B685B68934201D3981A44
:108200007047C068801A18447047C269036A9A426E
:1082100003D2C0681044C01A7047D01A704700BF1C
:10822000BFF34F8F0549064BCA6802F4E06213435F
:10823000CB60BFF34F8F00BFFDE700BF00ED00E054
:108240000400FA05704700BF70B582B00446056EA1
:1082500006236A4643211430A847C0B19DF8003078
:1082600001209DF801109DF8026041EA03219DF86C
:1082700003209DF804509DF8053042EA0622A4F838
:10828000401043EA0523A4F84220A4F8443002B089
:1082900070BD00BF70B582B00446856A06236A4689
:1082A0003B210830A847A8B19DF8003001209DF877
:1082B00001109DF8026041EA03219DF803209DF81A
:1082C00004509DF8053042EA0622618343EA052303
:1082D000A283E38302B070BD08B504F0FFFD044B38
:1082E0005B68C01AC0F5FA5020EAE07008BD00BF14
:1082F000B0A3012000B5002183B00A202DF0D0FBEF
:108300000F210A202DF0CCFB01AA032110202DF013
:10831000EFFB9DF90430F7EE007A9FED265A06EE4A
:10832000103A9DF90530DFED245A002106EE903A0F
:108330009DF90630B8EEC66A0A2007EE103AF8EE4C
:10834000E66A1E4BB8EEC77A76EEC56A36EE456A27
:1083500037EE457AB0EE675AA6EE255AB0EE456A7A
:10836000B0EE675AE7EE257AA6EEA55AF3EE0E5A5E
:1083700026EE256A67EEA57A25EE257A83ED006A5A
:10838000C3ED027A83ED017A2DF08AFB0DF1030231
:10839000012102202DF0ACFB0DF103020121092087
:1083A0002DF0A6FB01210A202DF07AFB012003B05D
:1083B0005DF804FB000000430000803B000001204A
:1083C00038B5044690F85D0000285AD104F1140530
:1083D000636E80226B2128469847642004F026FEB5
:1083E000636E0722682128469847642004F01EFE29
:1083F000636E00226B2128469847642004F016FE25
:10840000636E01226B21284698470F2004F00EFE70
:1084100094F85720636E1B21032A28468CBF1A222A
:10842000182298470F2004F001FE636E18221C21C9
:10843000284698470F2004F0F9FD636E94F8562003
:108440001A21284698470F2004F0F0FD636E94F837
:108450005820192128469847642004F0E7FD636EF0
:1084600010223721284698470F2004F0DFFD2846C8
:10847000636E0122382198470F20BDE8384004F090
:10848000D5BD10F048FD38B10268838812691340E9
:108490009CD12022C3718271034B214641F8103FC9
:1084A0002CF0A6FF92E700BF35810008F8B590F8E0
:1084B0007D3190F87E21134303F02103212B0FD04F
:1084C000436A846AA3420CD802690023121B92B249
:1084D00090F87D1100258362202980F8885103D00F
:1084E000F8BD1A1B92B2F3E78369E34203EB040180
:1084F000F6D0B2FA82F46409002CF1D190F87C3104
:10850000012BEDD005460127A0F866211346A0F8FF
:1085100064214FF0210ED0F87461C0F86011C0F8EA
:108520008041304685F87C710C4A0D4F85F87DE11D
:10853000F76332640B4FD5F8142134652832F764A1
:1085400023F01AFDD5F8143140221A6285F87C41D7
:108550009A6842F080029A60C2E700BF7DB80208C4
:10856000B9B8020815B80208426A10B48469A15467
:10857000426A04690132D0F8F410A24228BF0022F6
:10858000426241B10B68DB0702D55DF8044B7047CE
:108590005DF8044B8AE7D0F814215DF8044B1368AA
:1085A00043F08003136070474069903023F010BCA3
:1085B000F8B5D0F814310446DA69910614D5586A32
:1085C000E36AC0B2002B00F0A7809847D4F81431BA
:1085D0001A6822F480721A609A6822F001029A6086
:1085E0009A6942F008029A61DA69D20701D501223C
:1085F0001A62DA69970701D502221A62DA69560708
:1086000001D504221A62DA69150701D508221A6217
:10861000D4F8F420002A00F08B80D969490600D4F0
:10862000F8BDD96904F58A701E680F079D6819D1D5
:108630008F0602D5B50600F1FC800F0602D535067F
:1086400000F1D980480602D5710600F1AD80002AFC
:10865000E6D0626AA36A9A4240F08380012384F8DC
:108660008831F8BD15F001057FD116F4907FE4D074
:1086700011F0010700F0DB8016F4807779D13D46D8
:1086800005EA91073FB104271F62D4F8807147F0D3
:108690000207C4F880710F070AD5B70640F195802C
:1086A00008251D62D4F8805145F00805C4F88051B2
:1086B000D4F88051002DCAD08F0605D5B50603D554
:1086C00023F034FAD4F81431D4F88021110773D58B
:1086D0001A68202122F490721A609A6822F001022E
:1086E0009A6084F87E119A6852066BD59968D4F81E
:1086F000782121F040019960002A63D092F835304A
:108700005A49022B116564D080231046536523F02B
:1087100079F8D4F8F4209AE7E3696269D054E36900
:10872000E1680133B3FBF1F201FB1233E3614DE782
:10873000D96908067FF571AF94F87D1121293FF4BE
:108740006CAFA16A606A81424ED0A069405C013181
:10875000C0B298622569B1FBF5F005FB1011A1626A
:108760005BE72046BDE8F840A0E6CF0709D5F7054E
:1087700007D501271F62D4F8807147F00107C4F8BC
:108780008071EDB215EA51073FF47AAF4FF0020E57
:108790003D46C1F38007C3F820E0D4F880E14EF0F5
:1087A000040EC4F880E16DE71968202021F0400133
:1087B000196084F87D014AE79A6812F0400287D177
:1087C000C4F88021D4F8F42041E7002D3FF470AFC5
:1087D00066E71168052382F835300B68D4F8F42079
:1087E00023F001030B6032E7A4F86621196821F039
:1087F0008001196011E794F87D1121297FF427AFDA
:10880000B4F8661189B2C9B1D4F81C11B1F5805F12
:108810001DD0D4F86011481CC4F860010978996231
:10882000B4F86631013B9BB2A4F866310FE73D46D0
:1088300031E723F07BF9D4F8F42008E7196821F038
:1088400080011960196841F040011960FFE6D4F811
:1088500024110029DDD1D4F8601131F8020BC0F3E6
:1088600008009862C4F86011DAE700BF05B8020892
:108870002DE9F0470569C3681D4028D00F4606461C
:108880004FF000484FF00009B5FA85F328FA03F2DB
:108890001B3BD24332611540042B16D8DFE803F0AE
:1088A0003129211903007B6A002B32D003F1FF3AF2
:1088B000C7F824901FFA8AFA3C6A34B1236820462C
:1088C000514698476468002CF8D1002DDCD1BDE8F2
:1088D000F0873868716B036889B29847002DD3D14F
:1088E000F5E77868B16B036889B29847002DCBD162
:1088F000EDE7B868F16B036889B29847002DC3D1E2
:10890000E5E7F868316C036889B29847002DBBD160
:10891000DDE7F36A1FFA83FACEE700BF4269C2EBD4
:10892000421270B5D4000D4D2E19738903EB42032A
:108930001E3355F8230023F04BFA736804F15800F6
:10894000DA7959792844530703D4BDE8704022F0FE
:108950004BBABDE8704023F027BD00BF58940120FA
:10896000436910B508330D4C54F8230023F030FA56
:108970000B4B1B7843B90B4B2046198822F034FA75
:10898000094B00221A7010BD064B2046198823F0AF
:108990000BFD054B00221A7010BD00BF344D0120A5
:1089A000314D0120744D0120349E01202DE9F0410C
:1089B000174E044608461746356888462FF06CFA6D
:1089C000023029684346A8722246EC7228464D6957
:1089D0000221A84733684FF0150E22461D68142166
:1089E00083F80AE01846DC720A4B6D69A8473568BF
:1089F00038462FF051FA29681630EC7222463B4671
:108A0000A87228464C691621A446BDE8F04160478B
:108A1000302B012040E60308AA4B33F81020110543
:108A200013D501212DE9F0430446A74891B066090A
:108A300004F01F0550F82600A940014206D0A349C2
:108A4000097819B111B0BDE8F083704702F01F0733
:108A5000C2F34415242CF5D8DFE814F04300550088
:108A60009000A2005401A101A101B5036E0391037E
:108A70008302B502CF02DA02ED02F80209031903FC
:108A8000D501CA049C04AA04E5012002200249027F
:108A90005D025D02D403370445045704690451059F
:108AA0001205420525008A4B1A680AB1B2F908205E
:108AB00008AE8849DFF84882304610F0FCFF3046A7
:108AC000D8F800402FF0E8F938442A46E572A07241
:108AD00033462068394645692046A84711B0BDE8AD
:108AE000F0837D49642308AE01220C8830467B491F
:108AF00003FB04F3DFF808829B12632BA8BF6323F8
:108B000010F0D9FFDBE7764B764A1B781488022BEE
:108B100000F03785744904EB840374484A785B009D
:108B2000007802EB8202097893FBF0F3520001EB2C
:108B300081019B1AC2EB4102C3EBC30393FBF2F327
:108B4000062BA8BF062323EAE373C3F19603DBB227
:108B5000674A06268DF820300DF12100A2FB04E2C1
:108B60006449009608AED208DFF8948102EB8203D4
:108B7000A4EB43039BB210F09EFFA0E7DFF88081D7
:108B800010AE0D27D8F8000003681B6998475A4BB0
:108B9000B0F5F07F46F8203D0CBF072506258EE78F
:108BA00093F8612093F8606002EB8202534906EB70
:108BB00086065300B1F9002076005F42BA4203DB1B
:108BC0009342A8BF13461F46B1F902307542AB422B
:108BD00003DBB342A8BF33461D46DFF8248105EB13
:108BE0008505D8F8000005EB850503681B699847E3
:108BF000B0F5F07F95FBF6F618BF0224BB00A6F196
:108C0000290648BF3F33C6EBA313512B40F27585AD
:108C100007EB4705002D2B46B8BF05F13F03C6EB18
:108C2000A313512B40F24B85ED1B002D2B46B8BFF3
:108C300005F13F03C6EBA313512B40F22285ED1B38
:108C4000002D2B46B8BF05F13F03C6EBA313512BF4
:108C500040F2F984ED1B002D2B46B8BF05F13F0310
:108C6000C6EBA313512B40F2E585ED1B002D2B46DF
:108C7000B8BF05F13F03C6EBA313512B40F2BC85EF
:108C8000ED1B002D2B46B8BF05F13F03C6EBA31328
:108C9000512B40F26C85ED1B002D2B46B8BF05F122
:108CA0003F03C6EBA313512B40F24385ED1B48BF96
:108CB0003F35C6EBA516512E40F294840420FFF7F1
:108CC000ABFEBFE6F6330120303A012091000120CF
:108CD000402B012094E60308069E012064E6030869
:108CE000099E0120F4730120CC8001200A74012028
:108CF000CDCCCCCC6CE60308267E2700C4800120B6
:108D0000302B0120DFF82C840827D8F800000368F6
:108D10001B699847B0F5F07F0DBF4FF007094FF082
:108D200006090324042409F10406D8F80050224659
:108D300013230721D5F800E02846EC72AF72DEF865
:108D40001850A847D8F8001022464FF0160ECC72E3
:108D500001340D680846E4B281F80AE013231521B6
:108D6000AD69A847A642E0D1D8F8001009254A46C7
:108D700003230C68084681F80B908D720821A469C2
:108D80001525A047D8F800104A4602230C6808466B
:108D900081F80B908D721421A469A04752E603EB71
:108DA0004403B3F8524014F00F0300F00584022B83
:108DB000C4F303148CBF20229C22012B8DF82020A9
:108DC00000F0F985C0F0FD83022B00F0F085002350
:108DD0001A461846012C40F0E583B54C4FF0640E5E
:108DE000B44EA4FB0010B449DFF84883440B0DF1E6
:108DF0002100A6FB04C676090EFB164408AE0094BB
:108E000010F059FE5BE6AD4B08AEAD4A196830462E
:108E1000DFF820830C7A8B790194CC79A9490094EE
:108E200010F049FE4BE6A84BA84A1B88A84903EB63
:108E30008303127809785B00022A93FBF1F300F0B8
:108E4000A383A44A5178127801EB810102EB8200DE
:108E500049005A1AC1EB4001C2EBC20292FBF1F287
:108E6000062AA8BF062222EAE272C2F19602D2B214
:108E70009049D8178DF82020062681FB0312642420
:108E8000009608AEC0EB621293490DF12100DFF8A5
:108E9000A48204FB123310F00EFE10E68F4A182C49
:108EA0008F4B08AE116818BF6020546804BF64205F
:108EB0000C468C498DF8200003A883FB0423E2179D
:108EC000DFF87082C2EBA35210F0F5FD224685490F
:108ED00005A810F0F0FD03A82EF0DEFF05AB03AAF5
:108EE000814903440DF1210010F0E5FDE7E57F48DD
:108EF00008AE7F49B0F906E0B0F90440B0F902309D
:108F0000B0F900203046CDF804E0009410F0D3FD15
:108F1000DFF82082D3E51A2C764B774C08AE0CBFD5
:108F2000B3F90200B3F90000744984FB0024C317AD
:108F30000028DFF80082C3EBA40EACBF20222D2254
:108F40000EEB8E048EEAEE73A3EBEE73A0EB440EF1
:108F500030468EEAEE74A4EBEE74009410F0ABFD94
:108F6000ADE5674E002433688DF80B408DF80C405A
:108F7000002B00F042851A68D269002A00F01F8594
:108F800003A90DF10B00904733688DF81440002BB6
:108F900000F038851B681A6A1AB105A890479DF839
:108FA00014209DF80C1008AE564B574C304653F821
:108FB00021309DF80B100092625C5449DFF87481F7
:108FC00010F079FD7BE5524B9A213A4A64241B68E4
:108FD00008AE009183EAE37E3046DFF85881AEEBBD
:108FE000E37E82FB0E314FEAEE72C2EB6112494919
:108FF00004FB12E310F05FFD61E5454A08AE07236C
:1090000045499268304610F056FDDFF8288156E554
:10901000324B08AE414ADB893046414903EBC3037A
:10902000DFF810819B0082FB0342DB17C3EBA21227
:1090300010F041FD43E5294B08AE1F2239491B7D45
:10904000304610F038FDDFF8EC8038E593F85B200F
:10905000002308AE34499A421A463046DFF8D480DD
:109060000CBF0F240C24009410F025FD27E5134BB2
:1090700008AE2E4A19683046DFF8B8808C780B7835
:1090800001944C780F49009410F015FD17E50B4B37
:1090900008AE274A19683046DFF898804C79CB78BB
:1090A00001940C790749009410F005FD07E500BF15
:1090B0005917B7D11F85EB51C0E60308C83401200A
:1090C00000E70308ECE60308F4730120099E012081
:1090D0000A740120CC8001204CE70308E8800120BD
:1090E0006BCA5F6B94E6030898E603082C730120B3
:1090F00058E70308C4800120676666666CE70308CA
:1091000078400120ACD40308A4D40308DCE60308AB
:109110006080012078E6030884E60308D34D6210DE
:109120008CE6030864E60308A8E60308E8E60308FB
:10913000FCE60308302B0120B84B1A78002A00F017
:10914000D98303F1FF3903F10F080DF11F0699F8D8
:1091500001402FF08BFE20442246437803F00303A6
:10916000022B19F8013F08BFA4F1200206F8012FD5
:109170000BB1C845EBD108AEDFF8C0829FE4A84B25
:109180000424A84A0521B3F906300DF122008DF818
:10919000204008AEB3F5FA6F8DF82110A249A8BFA0
:1091A0004FF4FA63DFF89482B3F57A7FB8BF4FF4D7
:1091B0007A73A3F57A7382FB0342DB17C3EBA20237
:1091C00010F079FC7BE4994B1B68DE0040F1DE81F6
:1091D0000322974B974909884C0500F19C81C807E9
:1091E00000F1E2838E0701D50322934B9348BE180A
:1091F00039462A46046827682046A672E5727C69CB
:10920000A0471FE48E4A8F4B10899B688E49C31A72
:10921000A1FB001283424FEAD202A8BF034607EE29
:10922000902A23EAE373B8EEE77A07EE903AF8EE75
:10923000E77AC7EE876A16EE900A2EF099FF41ECA6
:10924000100B2FF011FF51EC100B2FF07FFA8A2337
:10925000C0B28DF82030002840F08A818D238DF82F
:1092600021308D238DF82230022800F257818D2382
:109270008DF823308D238DF824308D238DF8253003
:109280008D238DF826308D238DF827308D238DF892
:1092900028308D238DF829308D238DF82A308D23A9
:1092A0008DF82B30431E8F22092B8DF82C2004D8EB
:1092B00010AB18448E2300F81F3C002308AEDFF8E3
:1092C0007C818DF82D30FFF7FABB604B1B78DB07F4
:1092D0003FF5B8AB08AE5E49DFF86081304610F06C
:1092E000EAFBFFF7ECBB5B4B1B7803F00303032B9C
:1092F00000F027832D238DF82030002308AEDFF8FF
:109300003C818DF82130FFF7DABB524A127802F027
:109310000302032A00F0FB822D22002308AEDFF8AF
:109320001C818DF820208DF82130FFF7C8BB4A4BF7
:1093300016213C484FF4347EB3F9043008AE474A56
:1093400080FB0340DB17DFF8F480C3EBA0031BB204
:1093500001EB430182FB0140CC170844C4EB6024BD
:1093600030460EFB14143E4982FB042EE21774446F
:10937000C2EB6412D2B2C2F11802544202F00F02E0
:1093800004F00F0458BF62426032D2B210F093FB77
:10939000FFF795BB334A08AE33495378304612780D
:1093A0000133DFF89880013210F085FBFFF787BBAF
:1093B00000211E4810F0DBFD002840F05982234BAD
:1093C0001B7813F0020F294B1B7802D1002B00F001
:1093D0000083012B00F02E81022B40F01D8108AE8E
:1093E0002349DFF85880304610F065FBFFF767BB74
:1093F000204A08AE134B118830461B681E4A03FBF7
:1094000001F31E49DFF8348082FB0342DB17C3EB14
:10941000A21210F050FBFFF752BB00BF682E0120D4
:109420005C9E01206766666694E6030838A6012004
:1094300044E60308849E012060E60308302B0120E7
:10944000CC80012060800120A38B2EBAD08901201E
:1094500078E70308E4800120C4800120B7600BB6E0
:1094600084E70308B63401200CE70308099E0120B5
:1094700034E70308F4730120D34D621004E70308B6
:10948000CA4B0226CA4A1624B3F904304FF4347E7C
:10949000C84882FB0312DB17C749C3EBA203DFF8FE
:1094A000548313FB064308AE80FB0324DA171C44E5
:1094B000C2EB642234460EFB12324FF0000E80FBEA
:1094C0000230D3170244C3EB621351FA83F31868D6
:1094D00059681B7A03C423708DF829E0FFF7EFBAAF
:1094E000B64B1A680AB192F9012008AE0E23B449AE
:1094F0003046DFF8008310F0DEFAFFF7E0BA08AE7E
:1095000000236822AF4930460093DFF8E88210F06C
:10951000D2FAFFF7D4BA0422AB4B67E68B230328B9
:109520008DF823307FF6A6AE04288DF824307FF620
:10953000A4AE05288DF825307FF6A2AE06288DF85A
:1095400026307FF6A0AE07288DF827307FF69EAE36
:1095500008288DF828307FF69CAE09288DF8293030
:109560007FF69AAE0A288DF82A303FF699AE96E635
:109570008B2301288DF821303FF473AE8DF8223013
:1095800072E69723FFF7E4BA972271E48F4A904975
:109590001268904B02F48002002A0ABF0B46032295
:1095A000042217E68C490DF1210010F084FA08AE70
:1095B000DFF84082FFF783BA9B23C4F303148DF8CE
:1095C000203003F08BFC854BA3FB0013844A9B0CDB
:1095D00082FB03121A445211C2EB0211A3EB810366
:1095E000FFF7F8BB7F4AF317D8F80050132082FB2F
:1095F000061212212F68C3EB6203A872284603EB00
:10960000C3022344B61ADAB2A6F18003EA72BC6937
:10961000DBB2A047FFF752BB734B1B78002B3FF424
:1096200011AA08AE7149DFF8CC81304610F043FA38
:10963000FFF745BA08AE6E49DFF8B881304610F042
:109640003AFAFFF73CBA6749DA17D8F800C00E209B
:1096500081FB031E0D218CF80A006046C2EB6E02EE
:10966000DCF800E002EBC2092244A3EB0903D2B20A
:10967000803B8CF80B20DEF81890DBB2C847FFF770
:10968000E9BA5849DA17D8F800C00D2081FB031E4B
:109690000C218CF80A006046C2EB6E02DCF800E098
:1096A00002EBC2092244A3EB0903D2B2803B8CF83F
:1096B0000B20DEF81890DBB2C847FFF7C0BA494963
:1096C000DA17D8F800C00C2081FB031E0B218CF8A0
:1096D0000A006046C2EB6E02DCF800E002EBC20951
:1096E0002244A3EB0903D2B2803B8CF80B20DEF8B6
:1096F0001890DBB2C847FFF797BA3A49DA17D8F89B
:1097000000500B2081FB031E0A21A8722846C2EBE1
:109710006E02D5F800E002EBC20C2244A3EB0C036E
:10972000D2B2803BEA72DEF81850DBB2A847FFF7EE
:109730006FBA2C49DA17D8F800C0122081FB031E3B
:1097400011218CF80A006046C2EB6E02DCF800E0E2
:1097500002EBC2092244A3EB0903D2B2803B8CF88E
:109760000B20DEF81890DBB2C847FFF79FBA1D49FF
:10977000DA17D8F800C0112081FB031E10218CF8E5
:109780000A006046C2EB6E02DCF800E002EBC209A0
:109790002244A3EB0903D2B2803B8CF80B20DEF805
:1097A0001890DBB2C847FFF776BA00BFC48001202B
:1097B00067666666B7600BB66CB70308402B01207E
:1097C000A0E603088CE7030850E60308FC7D0120AF
:1097D00048E6030844E60308B4E6030883DE1B43B7
:1097E00089888888398EE338142B012040E70308E4
:1097F00028E70308302B01209249DA17D8F800C077
:10980000102081FB031E0F218CF80A006046C2EB7A
:109810006E02DCF800E002EBC2092244A3EB09036C
:10982000D2B2803B8CF80B20DEF81890DBB2C84730
:10983000FFF726BA8349DA17D8F800C00F2081FB5A
:10984000031E0E218CF80A006046C2EB6E02DCF8A3
:1098500000E002EBC2092244A3EB0903D2B2803B31
:109860008CF80B20DEF81890DBB2C847FFF7FDB983
:10987000754B1B88002B3FF4A2ADDC0700F1C580BF
:10988000C3F3400252BB580700F1D980190700F119
:10989000D480DA0600F1CF809E0600F1CA805C0613
:1098A00000F1C580180600F1C080D90500F1BB8029
:1098B0009A0500F1B6805E0500F1B1801C0500F14B
:1098C000AC80D80400F1A780990400F1A2805A046A
:1098D00000F19D80DB0B3FF44EAC0F225B4B08AEDA
:1098E0005B4953F82220304610F0E5F8DFF8A481F8
:1098F000FFF7E5B8574A08AEDFF89881334607CA44
:1099000003C3110C23F8022B1970FFF7D8B8524A81
:1099100093F85B301288002B55D14FF4A4714F4857
:109920000F2301FB02F280FB0201D217C2EB61128E
:1099300008AE4B49DFF85C81304610F0BCF8FFF709
:10994000BEB8454B1B88002B3FD0464B4FF43470BC
:109950004549B3F90430454C81FB0321DA17B4F9CA
:109960000030C2EBA102424912B29B1A5B001633CF
:1099700081FB0324DA171C44C2EB642200FB123281
:1099800081FB0231D3170A44C3EB6213DBB2C3F18C
:1099900018035A4203F00F0302F00F0258BF53425C
:1099A00060338DF82030A8E40422324B1EE4324AA2
:1099B000324BD06808E6324A304B106804E68DF826
:1099C0001420FFF7E7BA0C23B2E705238DF8203007
:1099D00093E42C4A2C4B11781B882C4A93FBF1F30F
:1099E000927B9A427FF618AE08AE2949DFF8A48030
:1099F000304610F060F8FFF762B88DF814301A4660
:109A0000FFF7CFBA1A46FFF7CCBA002266E70E225C
:109A100064E70D2262E70C2260E70B225EE70A2270
:109A20005CE709225AE7082258E7072256E7062290
:109A300054E7052252E7042250E703224EE70222B0
:109A40004CE700BF398EE338309E012044C1030843
:109A500014E70308D0E60308F89E01201F85EB51A8
:109A6000A0E60308C480012067666666FA9E0120AE
:109A7000B7600BB658E60308202B012083DE1B439A
:109A8000342B01200A740120F4730120CC800120C2
:109A900018E70308302B0120014B1869FEF788BD39
:109AA0000C6B0120014BD868FEF782BD0C6B0120C6
:109AB000014B9868FEF77CBD0C6B0120014B586888
:109AC000FEF776BD0C6B0120014B1868FEF770BDE8
:109AD0000C6B0120F8B510F58A75044614D0D0F847
:109AE00014212421002380F87D11116821F0010147
:109AF0001160136053609360C0F8803180F87C314E
:109B000080F87D3180F87E31A279A36812F00401DB
:109B1000C4F8183100F0F8804FF48053C4F81C31B9
:109B200012F0020300F029814FF400534FF48061DA
:109B3000C4F8203163790020C4F8241113F0010126
:109B4000C4F82C01C4F83401C4F8280102D0042060
:109B5000C4F8280113F0020605D0D4F8280140F01B
:109B60000800C4F82801D0070DD549B1D4F8380150
:109B70004FF4803740F00200C4F84071C4F8380157
:109B8000002E40F0E88012072AD5002D58D094F816
:109B90007D3103F0FF02002B00F0E880D4F814219F
:109BA0002423284684F87D31136823F001031360D1
:109BB00022F088FC012840D0D4F83831002B40F046
:109BC000D880D4F8143128465A6822F490425A605A
:109BD0009A6822F022029A609A6842F0080225E010
:109BE00075B394F87D3103F0FF020BB984F87C2142
:109BF000D4F814212423284684F87D31136823F0F7
:109C00000103136022F05EFC012816D0D4F838312D
:109C100013B1284621F032FFD4F8143128465A688F
:109C200022F490425A609A6822F02A029A601A68D6
:109C300042F001021A6021F0EBFE637903F00101AA
:109C400000292ED0D4F8F020002A75D00023D4F8B3
:109C5000F8004FF4806E4FF4803104F130074FF478
:109C60008076A363E3636364A3646365A36523668B
:109C7000E365226360633846C4F840E02165E6642A
:109C800022F0BEF9384622F0F9F994F87E31C4F892
:109C90007871202BA5667AD0226B63795268C4F85C
:109CA00008219B072FD5D4F8F420002A3DD00023AB
:109CB00040204FF48031C4F8902004F19006D4F88D
:109CC000FC204FF48067C4F89800C4F89420304614
:109CD000C4F89C30C4F8A430C4F8A830C4F8AC3040
:109CE000C4F8B430C4F8B830C4F8C030C4F8BC30DC
:109CF000C4F8A070C4F8B01022F082F9304622F007
:109D0000BDF950B1FEE7F8BD12F00203C4F81C1112
:109D100038D1C4F8203119460CE7D4F89030C4F893
:109D20007461C4F8C8505860F8BDD4F88421136831
:109D300043F080031360F8BDD4F88421116841F426
:109D400080711160916841F001019160116841F0EA
:109D500020011160A5E7D4F838014FF4003640F037
:109D60000100C4F83C61C4F838010CE784F87C2198
:109D700014E7284621F082FE23E7C4F820314FF48F
:109D80008061D7E64FF40053C4F82031D2E6E3688F
:109D9000626999B2002A3FF47FAFB1FA81F6760981
:109DA000002E7FF479AF94F87C0101283FF474AF62
:109DB0000B46A4F86C1138461449154F4FF0010CAE
:109DC0004FF0220E2167E766D4F81411114FC4F842
:109DD00080612431C4F86821C4F8806084F87CC1B3
:109DE00084F87EE1E76722F0C7F8D4F8143184F8EC
:109DF0007C611A6842F480721A609A6842F001022B
:109E00009A609A6842F040029A6045E781B8020879
:109E100085B8020815B8020841715BE6816059E611
:109E2000B0B5BB4BB8B0BB491A6C00AFBA4842F0F2
:109E30008052BA4C1A641A6C02F08052C7F8D820CB
:109E4000D7F8D8201A6B42F480221A631A6B02F4F6
:109E50008022C7F8D420D7F8D4200A6842F4807250
:109E60000A600268A24200F04882AD4C4FF6FF053E
:109E7000AC4AE168AC4829400A43E2605A6F02608C
:109E80001A6B42F480221A631A6B02F48022C7F81C
:109E9000DC20D7F8DC201A6B42F480121A631A6BAC
:109EA00002F48012C7F8D020D7F8D0201A6B42F401
:109EB00080021A631A6B02F48002C7F8CC20D7F82C
:109EC000CC201A6B42F000521A631A6B02F0005257
:109ED000C7F8C820D7F8C8201A6B42F080421A632E
:109EE0001A6B02F08042C7F8C420D7F8C4201A6B5E
:109EF00042F001021A631A6B02F00102C7F8C02097
:109F0000D7F8C0201A6B42F002021A631A6B02F0F3
:109F10000202C7F8BC20D7F8BC201A6B42F004023A
:109F20001A631A6B02F00402C7F8B820D7F8B820F9
:109F30001A6B42F008021A631A6B02F00802C7F8A3
:109F4000B420D7F8B4201A6B42F010021A631A6BCF
:109F500002F01002C7F8B020D7F8B0201A6B42F018
:109F600020021A631A6B02F02002C7F8AC20D7F85F
:109F7000AC201A6B42F040021A631A6B02F04002E6
:109F8000C7F8A820D7F8A8201A6B42F080021A63FD
:109F90001A6B02F08002C7F8A420D7F8A4201A6B2D
:109FA00042F480721A631A6B02F48072C7F8A02020
:109FB000D7F8A0201A6C42F001021A641A6C02F061
:109FC0000102C7F89C20D7F89C201A6C42F00202CC
:109FD0001A641A6C02F00202C7F89820D7F8982089
:109FE0001A6C42F004021A641A6C02F00402C7F8F8
:109FF0009420D7F894201A6C42F008021A641A6C64
:10A0000002F00802C7F89020D7F890201A6C42F0AE
:10A0100010021A641A6C02F01002C7F88C20D7F8EC
:10A020008C201A6C42F020021A641A6C02F0200292
:10A03000C7F88820D7F888201A6C42F040021A64CA
:10A040001A6C02F04002C7F88420D7F884201A6CFA
:10A0500042F080021A641A6C02F08002C7F8802075
:10A06000D7F880201A6C42F480721A641A6C02F4D9
:10A070008072FA67FA6F1A6C42F400721A641A6CF2
:10A0800002F40072BA67BA6F1A6C42F480421A6422
:10A090001A6C02F480427A677A6F1A6C42F40042BA
:10A0A0001A641A6C02F400423A673A6F1A6C42F46E
:10A0B00000321A641A6C02F40032FA66FA6E1A6CF4
:10A0C00042F480221A641A6C02F48022BA66BA6ED4
:10A0D0001A6C42F400221A641A6C02F400227A66A6
:10A0E0007A6E1A6C42F480121A641A6C02F48012AE
:10A0F0003A663A6E1A6C42F400121A641A6C02F450
:10A100000012FA65FA6D1A6C42F480020EE000BF8C
:10A11000003802400070004004400240EFBEADDE57
:10A1200000ED00E00005FA05BC7F01201A641A6CFE
:10A1300002F48002BA65BA6D1A6C42F400021A6425
:10A140001A6C02F400027A657A6D1A6C42F00072A1
:10A150001A641A6C02F000723A653A6D1A6C42F099
:10A1600000521A641A6C02F00052FA64FA6C1A6C0B
:10A1700042F080421A641A6C02F08042BA64BA6CEF
:10A180001A6C42F000421A641A6C02F000427A64BF
:10A190007A6C5A6C42F001025A645A6C02F0010265
:10A1A0003A643A6C5A6C42F002025A645A6C02F0F9
:10A1B0000202FA63FA6B5A6C42F010025A645A6C4B
:10A1C00002F01002BA63BA6B5A6C42F020025A6471
:10A1D0005A6C02F020027A637A6B5A6C42F48072F5
:10A1E0005A645A6C02F480723A633A6B5A6C42F4C5
:10A1F00000725A645A6C02F40072FA62FA6A5A6C7B
:10A2000042F480625A645A6C02F48062BA62BA6A9A
:10A210005A6C42F400625A645A6C02F400627A6228
:10A220007A6A5A6C42F480525A645A6C02F4805230
:10A230003A623A6A5A6C42F400525A645A6C02F416
:10A240000052FA61FA695A6C42F480325A645A6CCC
:10A2500002F48032BA61BA695A6C42F400325A642C
:10A260005A6C02F400327A617A695A6C42F48022A4
:10A270005A645A6C02F480223A613A695A6C42F488
:10A2800080125A645A6C02F48012FA60FA685A6CAE
:10A2900042F480025A645A6C02F48002BA60BA68CE
:10A2A0005A6C42F400025A645B6C03F400037B6056
:10A2B0007B6822F0CBF81D4B02461D491B681D48E8
:10A2C000A1FB03131C49A0FB02029B09920C013B5A
:10A2D0000A60B3F1807F08D2184AF02500200721D8
:10A2E000536084F8235090601160144AE03713687B
:10A2F00043F004031360BD46B0BD114A01F5484167
:10A3000002605A6C0F4842F480425A645B6C03F45A
:10A310008043C7F8DC30D7F8DC300A6803680A608D
:10A3200083F30888084B1B689847FEE750230120F9
:10A33000D34D621083DE1B43A8A2012010E000E091
:10A34000EDFEFECA0000F01F0400F01F08B5054B2B
:10A350001B6803B19847044B044A1A6072B6FDF7B4
:10A360005FFF00BF7C2F012004400240EFBEADDE46
:10A3700008B5034B1B6803B1984772B6FDF750FF51
:10A380007C2F012030B439240C4D0022A0422B46F2
:10A3900006D001321833052A0CD01C79A042F8D11E
:10A3A0009C79214201D10029F3D102EB420205EB55
:10A3B000C20000E0002030BC704700BF64DC03082E
:10A3C00030B5A02285B000211A4831F04EF81A4A63
:10A3D0001A4C0423116C04F1780541F00201116458
:10A3E000116C01F0020101910199116C41F0080119
:10A3F0001164116C01F0080102910299516C41F055
:10A4000002015164526C02F002020392039A2BB9CA
:10A410001834AC420CD0A379002BF9D02079183431
:10A420000EF079FD14F8101C2BF0C6FAAC42F2D1F4
:10A4300005B030BD8C9C01200038024064DC03086C
:10A4400001490248FEF714BADC9C012000040140D7
:10A45000FFF7F6BF01490248FEF70ABAB49C012093
:10A46000000C004001490248FEF702BA8C9C012012
:10A470000004004003682DE9F0439B0A464CA342C8
:10A480007ED03E34A34258D0403CA34201D0BDE828
:10A49000F08300244079414F8608002953D04FEAC9
:10A4A000841E02254FEA840C57F80E8005FA06F048
:10A4B0000CEB040ED8F80C9006EB4E05DFF8E0E04C
:10A4C00040EA09002E1D4EF825104EF82620C8F847
:10A4D0000C00314A934257D03E32934252D0403A18
:10A4E0009342D4D100260CEB0403DB0003F12000DF
:10A4F0007044EFF31185502282F31288103300224A
:10A5000073441968013211B1016018680430042ADB
:10A5100003F10403F5D10023EDB2036085F3118844
:10A520006444B6010EEBC404BA59236A73B3D3680A
:10A5300043F00103D360BDE8F08340790224174F54
:10A5400086080029ABD1A5014FF0020E4FEA840C1A
:10A5500057F8058020FA0EF00CEB04050EFA00FE09
:10A56000D8F80C0006EB450520EA0E00DFF830E0D5
:10A570002E1DC8F80C004EF825104EF82620A8E72E
:10A58000012487E70226AEE70126ACE7D36823F073
:10A590000103D360BDE8F08303001000ACA20120EA
:10A5A0008C9C0120F0B5830A4F4C85B0A34200F08B
:10A5B00095803E34A34200F08F80403CA34201D0FE
:10A5C00005B0F0BD0025AD01484E74597319A04285
:10A5D000F6D00446464801394FF0000E0768184689
:10A5E00089B2C3F810E0C3F808E0D960C3F814E0FA
:10A5F0007451B7FBF2F2013A5A6020F051FC3D4928
:10A60000B4F1804F18BF8C420CBF0121002111D042
:10A61000394B9C420ED003F580639C420AD0374AE6
:10A6200003F57C439C4218BF944203D003F570535A
:10A630009C42C5D1721900234FF4805792F83C0018
:10A6400001930128029303930097B9D07059022710
:10A65000DFF8B0E04FF0010C82F83D70876807EA40
:10A660000E0E274FC0F808E0D0F808E00EEA070702
:10A67000876082F83C3082F83DC0B9B91E4B9C42DD
:10A6800014D003F580639C4210D003F580639C4294
:10A6900003D003F578439C4292D17219002392F8BB
:10A6A0003C200093012A0193029389D073591148E9
:10A6B0005A688342996813D000F5806083420FD0B6
:10A6C00022F0700221F08001354400205A60996028
:10A6D00085F83C0005B0F0BD022574E7012572E75E
:10A6E00022F47002ECE700BF03001000ACA20120CE
:10A6F000502301200000014000040040000C0040F5
:10A70000F8FFFEFF8800FEFF2DE9F041284EC0EB68
:10A71000401506EBC5056B6883B3DB6873B32B7B11
:10A72000C0EB40100027234A43EA41011268C400ED
:10A730008BB22F732846191281EA1311594001F088
:10A740000F0141EA031189B290476A6895F8953084
:10A75000D179490710D4022B10D095F89530517952
:10A76000012B1CD004F11002583483B2324430194A
:10A77000BDE8F04120F0BABA022B01D1BDE8F0816A
:10A7800095F895305179012B0DD004F11002583411
:10A7900083B232443019BDE8F04121F093BD022369
:10A7A00085F89530DEE7022385F89530EDE700BFA8
:10A7B000589401204C940120114B98421ED003F56F
:10A7C000806398421AD0036823F04003036059B1B4
:10A7D00041F48071002991FAA1F3B3FA83F108BF23
:10A7E0004FF0FF310139C900036823F038031943E2
:10A7F0000160036843F04003036070474908E2E7E3
:10A800000038004030B44468012B24F48054446084
:10A810001CDD40F2E93401E0013C35D08568AD072C
:10A82000FAD500293DD031F8024B848140F2E93459
:10A8300001E0013C28D08568ED07FAD5C468A4B2D0
:10A840000AB122F8024B023B012BE2DC446844F4DB
:10A850008054446013B340F2E93301E0013B37D048
:10A860008468A407FAD5002936D00B78037340F228
:10A87000E93301E0013B2BD08168C907FAD5C368F1
:10A88000DBB25AB1137009E0144B98420CD0144B50
:10A89000984219D003F58063984217D0012030BC4C
:10A8A00070474FF6FF74C0E723460E4AD82101FBDC
:10A8B00003239A89013292B29A81988980B200303A
:10A8C00030BC18BF012070470123EEE70223ECE7FC
:10A8D000024A9042DBD1E8E7FF23C7E7003001409E
:10A8E00000380040406B012070B5044682B0006A19
:10A8F0000EF0E1FB6A4607231049A069FFF782FFCB
:10A90000206A0EF0DEFB9DF801309DF80210012058
:10A910009DF8036041EA03219DF804209DF805504D
:10A920009DF8063042EA0622A4F8401043EA0523C7
:10A93000A4F84220A4F8443002B070BD84B70308E4
:10A9400040F2E93300E09BB18268013B12F0020F54
:10A950009BB2F8D0017340F2E93300E043B1826862
:10A96000013B12F0010F9BB2F8D0C068C0B2704733
:10A970000C4A904209D00C4B984211D003F58063E9
:10A98000984201D0FF2070470223084AD82101FBDA
:10A9900003239A89013292B29A819889C0B2704792
:10A9A0000123F2E70030014000380040406B0120F5
:10A9B0002DE9F84F0123DFF8D4B010212F488BF890
:10A9C0000030FFF7F9FE2E4BDFF8C4A018680EF038
:10A9D00072FB05212948FFF7B3FF00212748FFF745
:10A9E000AFFF06212548FFF7ABFF00212348FFF703
:10A9F000A7FF9AF800400421204844F00104214FA9
:10AA0000FFF79EFF1D482146FFF79AFF3B88B3B131
:10AA100000241D4EDFF87C80184D16F804900721A5
:10AA20002846FFF78DFF49462846FFF789FF315D2D
:10AA3000621C3B8808F8041094B2A342EDD80721A9
:10AA40000E48FFF77DFFFF210C48FFF779FF9AF8CA
:10AA5000004004210948FFF773FF21460748FFF72C
:10AA60006FFF074B18680EF02CFB04210348FFF71B
:10AA7000A3FE00238BF80030BDE8F88F00380040BB
:10AA8000C8A30120141D0120283801203D3A0120CF
:10AA9000453A0120543A01202DE9F843544F102142
:10AAA0005448FFF789FE38680EF005FB524B1B78BF
:10AAB000012B00F08E8072D3022B0CD1DFF8549161
:10AAC000082389F800300D264FF4C373DFF848815E
:10AAD000A8F8003011E0DFF83C91DFF83C8199F8EC
:10AAE000003003F04003002B15BF4FF4F0734FF418
:10AAF000C37310260D26A8F8003000243D4D04F144
:10AB0000100128460134C9B2FFF71AFF0121284677
:10AB1000FFF716FFA3B2B342F1D399F8004000212A
:10AB20003448FFF70DFF21463248FFF709FF334B4A
:10AB3000022130481C78FFF703FF2E482146304D94
:10AB4000FFF7FEFE2F4B03212A481C78FFF7F8FE83
:10AB500028482146FFF7F4FE2B4B042125481C789A
:10AB60000C43FFF7EDFE23482146FFF7E9FE386866
:10AB70000EF0A7FA04211F48FFF71EFEB8F80020C8
:10AB80000021224830F071FC2B7B33B1204B1B7825
:10AB900043B300232B73BDE8F883BDE8F883A021FD
:10ABA0001448FFF7CDFE00211248FFF7C9FE00F060
:10ABB0000603DFF86090022B07D000F005000128A3
:10ABC00003D1482389F8003008E0082389F80030D1
:10ABD00079E7DFF84090482389F8003010264FF4D9
:10ABE000F07373E7FFF7E4FE00232B73BDE8F883EF
:10ABF000C8A3012000380040CCA30120D3A301202A
:10AC000000000120D4A30120453A0120543A01203C
:10AC10003D3A0120161D0120141D0120F8B50446FF
:10AC20000F4615461E46C0680EF045FA47F08001F3
:10AC30006068FFF785FE33462A4600216068FFF70B
:10AC4000E1FDE0680EF03DFA0120F8BD70B50B4C57
:10AC50000646237853B90A490025324663780868C6
:10AC600049212570FFF7DAFF012070BDFDF734FBA5
:10AC70000028F0D002F080F9EDE700BFB0A301207A
:10AC8000ACA30120F0B54A4C83B02578012D13D038
:10AC900028D3022D0DD1474B06461B78002B77D1C8
:10ACA0006846FFF7D3FF20B19DF8063013F0030785
:10ACB00022D0002003B0F0BD3E4E3378002B62D18D
:10ACC0006846FFF7C3FF9DF8003008B1DB0764D486
:10ACD0000023237033784BB100230133002023700D
:10ACE00003B0F0BD334E3378002BF5D101210220A3
:10ACF0002AF02CFF2378F0E79DF8012001219DF830
:10AD000000500A209DF8033045EA02259DF80220F4
:10AD10009DF805E042EA03229DF804302DB2277029
:10AD200043EA0E23244C12B26D421BB294ED005A3A
:10AD3000524206EE905A5B42D4ED015A07EE102AB9
:10AD4000F8EEE66A07EE903A94ED026AB8EEC77A3A
:10AD5000F8EEE77A66EE856A27EE257A67EE867A60
:10AD6000FDEEE66ABDEEC77AFDEEE77A16EE904A92
:10AD700017EE102A17EE903A34807280B3802AF0D2
:10AD80008FFE03B0F0BDFDF7A7FA002898D090E73A
:10AD9000FDF7A2FA00288CD182E7337823B9072186
:10ADA00003202AF0D3FE257801350020257081E7A5
:10ADB00030250120B0A301200000012070B5044619
:10ADC0000E461546C0680EF076F931466068FFF70A
:10ADD000B7FD29466068FFF7B3FDE0680EF071F932
:10ADE000012070BD10B54FF4807104468069FFF7F3
:10ADF000E3FC012002F0C0F82046FDF7E1FA102242
:10AE00006A2104F11400FFF7D9FF642002F00EF963
:10AE1000A0690421FFF7D0FC0120BDE8104002F03A
:10AE2000ABB800BFF8B55B4DD823044603FB005315
:10AE3000661C18790EF06FF80746F6B210B11223AF
:10AE4000C6718371D82303FB045358790EF063F85D
:10AE500010B11323C6718371D82303FB045398796F
:10AE60000EF059F810B11423C6718371D82303FB77
:10AE700004539A7B002A5CD0DA7938464E210EF0D2
:10AE800013F9D82606FB04F6AF1978790EF043F8CB
:10AE90003A7A2E210EF008F9B8790EF03CF87A7A59
:10AEA0000E210EF001F9AB593B491A688B4222F092
:10AEB00040021A604ED0394A934255D0384A9342E4
:10AEC0005DD0384A93423AD0374A934209D102F5CD
:10AED0006842516A41F480115162516A21F4801133
:10AEE0005162D822596802FB045441F48051A27B7C
:10AEF0005960002A196814BF0024022449060FD49F
:10AF00001D6882F00102294829492840024342F481
:10AF1000457222431A605A68114041F4E061596059
:10AF2000DA6922F40062DA611A6842F040021A60BB
:10AF3000F8BDDA7938462E210EF0B6F8A1E702F511
:10AF40008232516A41F400515162516A21F4005138
:10AF50005162C6E7174A516A41F480515162516A01
:10AF600021F480515162BCE702F50032116A41F4CC
:10AF700080411162116A21F480411162B1E702F54A
:10AF8000FE32116A41F400411162116A21F400415C
:10AF90001162A6E7406B01200030014000380040FC
:10AFA000003C004000340140005001404000FFFFE1
:10AFB000FBF0FFFF0038024070B5C0EBC000104C42
:10AFC000104E82B004EB8004306B25692843306357
:10AFD000366B94F90D003540A160636191090195CC
:10AFE000019B2AF0A9F994F90D300122064903F0DA
:10AFF0001F005B09824041F8232002B070BD00BFF2
:10B00000980001200038024000E100E00A4BC0EB4C
:10B01000C00030B403EB8000084C82B0256B03699C
:10B020001D432563246B0176234042760193019BE7
:10B0300002B030BC704700BF9800012000380240C9
:10B040000348D0F8AC3113B100F5D27018477047FF
:10B05000980001200348D0F8903113B100F5C47076
:10B0600018477047980001200348D0F8743113B195
:10B0700000F5B67018477047980001200348D0F8D3
:10B08000583113B100F5A870184770479800012097
:10B090000348D0F83C3113B100F59A701847704757
:10B0A000980001200348D0F8203113B100F58C70CE
:10B0B00018477047980001200348D0F804310BB1BD
:10B0C000FC301847704700BF980001200348D0F8B3
:10B0D000E8300BB1E0301847704700BF98000120FE
:10B0E0000348D0F8CC300BB1C4301847704700BFCC
:10B0F000980001200348D0F8B0300BB1A8301847B1
:10B10000704700BF980001200348D0F894300BB17D
:10B110008C301847704700BF980001200248836FA9
:10B120000BB1703018477047980001200248C36D7A
:10B130000BB1543018477047980001200248036C47
:10B140000BB1383018477047980001200248436A15
:10B150000BB11C30184770479800012002488368E3
:10B1600003B11847704700BF98000120A54A00218D
:10B17000A54BA64870B5D2F888404FF00065A44EA4
:10B18000A4B044F47004C2F888401C6844F0010480
:10B190001C6099601C68204018605E60186820F48C
:10B1A00080201860D9609560BFF34F8FBFF36F8F19
:10B1B000C2F85012516941F400315161BFF34F8F11
:10B1C000BFF36F8F196C934A41F080511964196C69
:10B1D00001F0805102910299116841F440411160DF
:10B1E000126802F440420192019A9A6802F00C023D
:10B1F000042A52D09A6802F00C02082A4AD0824BE4
:10B20000854C1A68194642F480321A60226803E0BD
:10B2100023689B1A642B3CD80B689803F8D57A4BAB
:10B220009A6802F00C02082A33D01A68184622F0F5
:10B2300080721A60226803E023689B1A022B28D8C8
:10B2400003689B01F8D447F6C07393FAA3F34FF455
:10B250004031B3FA83F291FAA1F14FF0706191FAA3
:10B26000A1F10926B1FA81F14FF4D8736B4D8E40EC
:10B270006549934033431D434560036843F0807341
:10B28000036022680B689E010BD423689B1A022B73
:10B29000F8D9FEE75B685C02B1D55B4B5E4C1B687E
:10B2A000BDE7086C5B4A40F0805013460864096CA7
:10B2B00001F0805103910399116841F480311160CC
:10B2C00021685A68D50305D42268521AB2F57A7FEC
:10B2D000F7D9FEE71A684F4942F400321A60226833
:10B2E00004E023689B1AB3F57A7FF2D84B68980381
:10B2F000F7D54FF400164FF000654FF4C0710722E8
:10B30000032304A804962195089109920A932DF02D
:10B31000CFFA00B1FEE7424A136803F00F03062B91
:10B320001BD9394B9A6822F0F0029A601A68920190
:10B3300067D59A68184641F2883122F0030242F03C
:10B3400002029A602268836803F00C03082B10D075
:10B3500023689B1A8B42F6D90AE0136823F00F0387
:10B3600043F007031360136803F00F03072BD8D0D3
:10B37000FEE72B4A136803F00F03072B35D8224C46
:10B38000A36823F4E05343F4A053A360A36823F419
:10B39000604343F40043A36021F058F8A368F0220F
:10B3A00092FAA2F2B2FA82F203F0F0031D4ED340F9
:10B3B0001D4D334493F8203020FA03F32B6029F01D
:10B3C000EFFF0023194A04A80492139314931593D2
:10B3D00016931793189319931A931B931C931D9309
:10B3E0001E932DF065FA18B3FEE7136823F00F03E0
:10B3F00043F007031360136803F00F03072BB7D163
:10B40000BDE7B5E700ED00E000380240FFFFF6FEC3
:10B410001030002400700040B87F01200800402058
:10B42000003C02406CB7030850230120C0FF03001A
:10B43000D4F88C3023F08073C4F88C30D4F88C307E
:10B4400043F08073C4F88C30A36803F00C03042B22
:10B4500027D0082B0DD0154B154A16499268C2F318
:10B460000312164496F82020D3408B422B601AD04A
:10B47000FEE7616862684B02616802F03F024CBF00
:10B480000D4B0A4BB3FBF2F3C1F3881203FB02F33B
:10B49000074A5268C2F3014201325200B3FBF2F391
:10B4A000DAE7054BD8E724B070BD00BF0024F400F4
:10B4B0000038024000E6DF0C00127A0038B50B4C71
:10B4C00023688BB15A680546821A002A04DA0CE018
:10B4D0005A68AA1A002A07DB9A6818461B68226075
:10B4E00098472368002BF3D138BD38BD0887012069
:10B4F00000210B4B10B40A460424017202E0072914
:10B500000BDC9C79A40702F1010202D51C7944549A
:10B510000131042A03F11803F1DD5DF8044B704793
:10B5200064DC030810B404230E4C0022214613F0FF
:10B53000010301F1180107D10132052A0DD08B79E1
:10B54000183113F00103F7D002EB420204EBC20200
:10B550005DF8044B13790370704703705DF8044B7A
:10B56000704700BF64DC03080B4B30B503F11404D3
:10B5700093F90020043313F8035C072AC8BF143A78
:10B5800081188D7213F8025C855413F8012CA342C4
:10B590000A75EDD130BD00BF9CB7030803682DE9E3
:10B5A000F041DF691FB13B46BDE8F0411847002A72
:10B5B000164611DD04460D460E4400E023689B68E4
:10B5C000204698470028F9D02368204615F8011B2B
:10B5D0001B689847AE42F1D1BDE8F08100233C21C1
:10B5E0004222017042708370C370704708B522F028
:10B5F000A9FBFEF7BDFE00BFA0F10A032DE9F04F45
:10B600000C462DED028B89B0E72B00F24F87DFE867
:10B6100013F01C014D074D074D074D074D074D0712
:10B620004D074D074D074D074D074D074D074D077A
:10B630004D074D074D074D074D074D074D074D076A
:10B640004D0780014D074D074D0771014D074D070F
:10B650004D0764014D0781024D073E024D0733023D
:10B660004D072B024D07FF014D07EC014D074D071C
:10B670004D07E601DF014D07AA034D074D07A30360
:10B680004D077B034D074D074D076F034D074D07D2
:10B690004D074D0717034D07FC004D0759033603AF
:10B6A0004D074D074D074D074D074D074D07150534
:10B6B0004D07E6044D07B2044D075E044D074A04EA
:10B6C0004D074D074D074D07F303B903B203C502FC
:10B6D000E80030061C06550611064D07D805B905C9
:10B6E0004D074D074D074D079A054D074D07780546
:10B6F0004D074D074D073D07FF06B2066D064D0786
:10B700004D074D07DF06C706EF0657054D074D07E6
:10B710004D074D074D074D074D074D074D074D0789
:10B720004D074D074D074D074D07F3034D074D07D7
:10B730004D074D074D074D074D074D074D074D0769
:10B740004D074D074D072D014D074D074D074D077F
:10B750004D074D074D074D074D074D074D074D0749
:10B760004D074D074D074D074D074D074D074D0739
:10B770004D074D074D074D074D074D074D074D0729
:10B780004D074D074D074D074D074D074D074D0719
:10B790004D074D074D074D074D074D074D074D0709
:10B7A0004D074D074D074D074D074D074D074D07F9
:10B7B0004D074D074D074D074D074D074D074D07E9
:10B7C0004D074D074D074D074D074D074D074D07D9
:10B7D0004D074D074D074D074D074D074D07A2017A
:10B7E000AD01B74E337853B1B64F002537F8021F7D
:10B7F00020460EF07DF801353378AB42F6DC0120AF
:10B8000009B0BDEC028BBDE8F08FAD4E3378002B54
:10B81000F5D0AD4F0025B8462368204617F815200F
:10B820000135591C08F1020821601A7018F8011C32
:10B8300001EB810101EB810101F2EE2189B20EF0F1
:10B8400057F83378AB42E7DCD9E7A04D28462CF017
:10B8500023FB0028D3DD2B460544226813F8011B87
:10B86000501C9D4220601170F7D1C8E70B68DFF8CB
:10B87000A0C2591C9CF8002021601A709CF800306E
:10B88000002BBCD0924E0023924D934893492268DE
:10B89000013316F8017F02F1010EC4F800E01770C1
:10B8A000226815F8017F02F1010EC4F800E017705C
:10B8B000226810F8017F02F1010EC4F800E0177051
:10B8C000226811F8017F02F1010EC4F800E0177040
:10B8D0009CF800209A42DADC91E70B680120804A4C
:10B8E0001D18117825601970236852781918216085
:10B8F0001A7085E77B4D084629880DF0F9FFA98865
:10B9000020460DF0F5FF204629890DF0F1FF0120BA
:10B9100076E7754D05F150062878043528F00EFAC3
:10B920002368027A591C21601A70236815F8032CC9
:10B93000591C21601A70236815F8022C591C2160CB
:10B940001A7015F8012CAE42236803F10101216041
:10B950001A70E1D153E7654D0846E9890DF0C8FF3B
:10B960002046A9890DF0C4FF012049E7604B03F18F
:10B9700070052268073313F8071C501C20601170F3
:10B98000226813F8061C501C20601170226813F8FE
:10B99000051C501C20601170226813F8041C501CF8
:10B9A00020601170226813F8031C501C2060117075
:10B9B000226813F8021C501C2060117013F8011C3F
:10B9C0009D42226802F1010020601170D1D116E77A
:10B9D0000B6801229918104621601A7010E708467A
:10B9E00000210DF06FFF01200AE7424D424E05F1A4
:10B9F000300795F90210414B93F9062008338A422B
:10BA000000F057859E42F7D10835BD42F1D1F6E6E8
:10BA10003B4B03F15A052268063313F8011C501CF6
:10BA200020601170226813F8061C501C20601170F1
:10BA3000226813F8051C501C20601170226813F84E
:10BA4000041C501C20601170226813F8031C501C49
:10BA50002060117013F8021C9D42226802F101005F
:10BA600020601170D7D1CAE60B680120254A191849
:10BA7000527D21601A70C3E6234D05F1800655F80A
:10BA8000041F20460DF01EFFAE42F8D1B7E61F4D51
:10BA900005F14006B5F8801020460DF029FF236817
:10BAA00095F882200435591C21601A7095F87F2082
:10BAB000B542236803F1010121601A70EAD19EE6C4
:10BAC000348601205A9E012098890120682E012089
:10BAD000A73E0120B73E0120D73E0120C73E0120EE
:10BAE000182F0120A06E01201C2F01208C2E012078
:10BAF000088B0120DCA301206C7F01203C7F01200A
:10BB0000D02B0120707F012030820120348201205F
:10BB1000A53E0120C04D08460B682A7A591C2160B9
:10BB20001A70A98B0DF0E4FE298B20460DF0E0FE83
:10BB3000698B20460DF0DCFE2368EA7C2046591C08
:10BB400021601A70A98C0DF0D3FEE98C20460DF00F
:10BB5000CFFE2368AA7F2046591C21601A702368F3
:10BB600095F82020591C21601A70698C0DF0C0FED8
:10BB70002368EA7A2046591C21601A70E9680DF0A2
:10BB8000A1FE236801202A7C191821601A702368FD
:10BB900095F82120191821601A7031E69F4DA04EAA
:10BBA00005F12007DFF8BC82DFF8BC929FED9D8A8B
:10BBB000DFF8B8B2DFED9C8ADFF8B4A20DE0FCEE4E
:10BBC000E77ACDED017ABDF80410043520460DF07A
:10BBD0008FFE1836AF423FF412AE717C0029F4D0CC
:10BBE00098F80030D5ED007A012BE8D1D9F8003073
:10BBF000DB0440F11985F5EE407AF1EE10FA00F021
:10BC00002B85F4EEC87AF1EE10FA00F12585F4EEFA
:10BC1000E87AFDEEE77AF1EE10FA17EE903A00F2CC
:10BC200039856FF4F972303B02FB03F38AFB031290
:10BC3000D9171344C1EB632101F2DB5189B2C4E788
:10BC40000B680846794D591C2A7921601A702368BF
:10BC50006A79591C21601A7029880DF049FE236801
:10BC6000AA792046591C21601A7069880DF040FE9F
:10BC700023680120EA79191821601A70C0E50B6861
:10BC800001256B4E5A190A601D700B68B27859195C
:10BC900021601A702AF0E6FE2368664A5F19664939
:10BCA00027601870B1F90010B2F900000DF0A6FF7E
:10BCB00023685A1922601870204631880DF018FE4A
:10BCC00028469DE50B68002508465A1C2946226037
:10BCD0001D7023685A1C22601D7023685A1C226044
:10BCE0001D700DF0EFFD294620460DF0EBFD86E5B9
:10BCF0000B68002508465A1C294622601D700DF06D
:10BD0000E1FD29462046ECE70B6808464B4A5E1CDD
:10BD10004B4D11784B4A2660197011680DF0D2FD19
:10BD200023683D4A2046591C127A21601A702988DE
:10BD30000DF0DEFDA98820460DF0DAFD29892046A8
:10BD40000DF0D6FD002120460DF0D2FD2046002149
:10BD50000DF0CEFD012053E5084608222E490DF0D6
:10BD600084FD01204CE50B680120374A1D189178AD
:10BD700025601970B8E50846102234490DF075FDAC
:10BD800001203DE5324B1B8BB3F5006F00F261845F
:10BD9000B3F5806F00F27B84B3F5007F34BF0127D9
:10BDA00002272C4D05F10C0655F8041B204691FB8B
:10BDB000F7F189B20DF09CFDB542F5D1264D274F24
:10BDC00005F10C06B5EC010AD7ED097A80EE270AD9
:10BDD0002DF030FA81B220460DF08AFDB542F1D146
:10BDE0001F4D05F10C0655F8041B204689B20DF0D5
:10BDF0007FFDAE42F7D102E500238146DFF8748073
:10BE000001211D464FF6FF7ADFF86CB004930693CC
:10BE10000593079338E000BF707F0120F02E0120CA
:10BE2000709301200000404200E08244002D012078
:10BE300016360120B8A40120BAA40120182F012031
:10BE4000A06E012048360120A82E0120E02E0120FE
:10BE500070800120AC800120F07D0120007601205F
:10BE6000D02E012054940120FC7D0120DB9B9141C8
:10BE700021053483E0B70308849E012001350B2D92
:10BE800000F0358318F9011F4F1C4AFA05F3F5D06D
:10BE9000DE07F3D5BBF800302B41D807EED506A856
:10BEA0000EF056F8EAE70B680120AD4A1E18AD49BE
:10BEB000D57826601D70236849791D18AA4A256027
:10BEC00019702368D278191821601A7098E400213B
:10BED00020460DF00DFD00212046A44D0E460DF02C
:10BEE00007FD204631460DF003FD236820465A1C0D
:10BEF00022601E7023682A68591C92F82C20216049
:10BF00001A7023682A68591C92F8362021601A702A
:10BF100023682A68591C92F8372021601A70236818
:10BF20005A1C22601E7023685A1C22601E702368EF
:10BF30005A1C22601E702B68598F0DF0D9FC2B689B
:10BF40002046198F0DF0D4FC23682A682046591C1E
:10BF500092F82E2021601A7023685A1C22601E70ED
:10BF60002B68598E0DF0C4FC2B682046998E0DF07D
:10BF7000BFFC012044E47E4E08460B6872797B4D7D
:10BF8000591C21601A702B68198C0DF0B1FC2B68BC
:10BF90002046D98B0DF0ACFC718920460DF0A8FC31
:10BFA000B18920460DF0A4FC2B682046598C0DF079
:10BFB0009FFC2B682046998C0DF09AFCF189204655
:10BFC0000DF096FC318A20460DF092FC2A68236819
:10BFD000012092F82620191821601A7010E4644E8E
:10BFE000F378002B00F029830B68012208219818B0
:10BFF000206019702368991821601A702368204600
:10C000005C4D591C2A7921601A702368AA78591C42
:10C0100021601A7029880DF06BFCE98920460DF02B
:10C0200067FC23680120F279191821601A702368CF
:10C03000EA78191821601A70FFF7E2BB16F0A8FA27
:10C04000FF28064600F00C8308A900250DF10D001D
:10C0500001F8125D8DF80D5016F07AFA08A800F874
:10C06000115D16F069FA08A800F8105D16F058FA8C
:10C0700008A820F8085D16F047FA236820465A1CE5
:10C0800022601E7023689DF80D20591C21601A70D3
:10C0900023689DF80E20591C21601A7023689DF8B2
:10C0A0000F20591C21601A7023689DF81020591C1C
:10C0B00021601A70BDF818100DF01AFCFFF79FBB35
:10C0C0000B682D4F591C3A7821601A703B78002B71
:10C0D0003FF495AB0025EEB20135304619F08AFCED
:10C0E000236842783046591C21601A7019F082FC8E
:10C0F000018920460DF0FCFB3B78AB42EBDCFFF7FF
:10C100007EBB1E4D05F16006A98820460DF0F0FBB0
:10C11000E98820460DF0ECFB298920460DF0E8FB6C
:10C120002368AA7A2046591C21601A702368EA7A8B
:10C13000591C21601A7055F80C1B0DF0C3FBAE4260
:10C14000E2D1FFF75CBB52230D492268501C2060EE
:10C15000137011F8013F002BF7D1FFF750BB00BF60
:10C160008C2E01202C8401209C2E0120C83401201B
:10C17000EC75012030940120D8BB0120148A0120E5
:10C18000B0B703080023AE48226803EB43010568FB
:10C190000133561C6D5C0A2B2660157002682568F9
:10C1A0000A4405F10106527826602A700268256863
:10C1B0000A4405F10101927821602A70E4D1FFF769
:10C1C0001EBBA04D00230A682968501C0978206016
:10C1D0001170296822688978501C206011702A68C3
:10C1E00021681A440133481C5279032B20600A70DD
:10C1F000F5D1236820462A68591C127A21601A70EA
:10C2000023682A68591CD27821601A7023682A682A
:10C21000591C127921601A702B6859890DF068FB3E
:10C220002A6823680120527A191821601A702A6836
:10C23000FFF75ABB002120460DF044FB20460021A9
:10C240000DF056FB0120FFF7DBBA7F4B084619883B
:10C250000DF04EFB7D4B204619880DF049FB7C4BC1
:10C26000226801201B781118034021601370FFF72A
:10C27000C7BA784B08460A681B78511C764D03F004
:10C2800002032160137023682A7D591C21601A70F3
:10C2900029680DF017FB696820460DF013FB29890A
:10C2A00020460DF025FBE98920460DF021FB2046B4
:10C2B000298A0DF01DFB0120FFF7A2BA674D084641
:10C2C00029880DF015FB698820460DF011FBB5F9A2
:10C2D0000430634A2046D91782FB0323C1EBA30134
:10C2E00089B20DF005FB0120FFF78ABADFF898E16B
:10C2F0000027FEB2714600232268501C2060167091
:10C300002268501C206013700133226811F8010F5D
:10C31000062B02F1010525601070EDD101370EF1F9
:10C32000060E062FE5D14F4900232268501C2060DD
:10C3300017702268501C206013700133226811F8B6
:10C34000010F0B2B02F1010525601070EDD1236860
:10C350000725012000215E1C434A26601D702368CA
:10C360001D1825601970236892F8F02019182160B3
:10C370001A70FFF745BA0B6801203C4A1E183C4969
:10C38000157826601D70236889781D18394A256044
:10C39000197023689278191821601A70FFF730BA63
:10C3A0000A680120344B151819782560117022682D
:10C3B000597815182560117022689978151825602C
:10C3C00011702268DB78111821601370FFF718BA1A
:10C3D0002A4D0846298A0DF08BFA698A20460DF00D
:10C3E00087FA2046A98A0DF083FA0120FFF708BAE0
:10C3F000204B08461A49B3F9003081FB0321DB17B3
:10C40000C3EBA10189B20DF073FA0120FFF7F8B96F
:10C410000A6808461A4B561C1A491D782660157082
:10C4200022685D78561C2660157022689B78551C22
:10C4300025601370C9880DF05BFA0120FFF7E0B9A1
:10C44000C8340120F8910120F89E0120FA9E0120B5
:10C45000AC9E0120E4800120E8800120C4800120FE
:10C46000676666661783012034820120EC7501201F
:10C470008C2E01209C2E01208C3E01203094012026
:10C48000842E012004910120F3820120934D08465F
:10C4900029880DF02DFA698820460DF029FA2046EA
:10C4A000A9880DF025FA0120FFF7AAB90020FFF7AF
:10C4B000A7B9236820465A1C2260197029880DF0FC
:10C4C00017FA2368EA78591C21601A7023682A79C0
:10C4D000591C21601A702368AA79591C21601A70AE
:10C4E00023686A79591C21601A70FFF78DBA0025FC
:10C4F000DFF80CA24FF008080135C5F12002A5F1C4
:10C500002003252D2AFA05F608FA02F228FA03F389
:10C5100010D016431E43002306F001021343EBD054
:10C52000E8B222F0B1FE0028E6D0294606A80DF0B8
:10C530000FFDE1E76A4B1B78DA0700F198800025D0
:10C54000684E2F4602E00135252D0DD02946304694
:10C550000DF00DFD0028F6D0294606A80DF007FDC8
:10C5600000285CD10137EEE75F4B20465F4DB3F802
:10C5700050100DF0BDF9002120460DF0B9F95C4BCB
:10C58000204619684A01C1F34003C1F3800EC1F38C
:10C59000C00602F020021343C1F3401201F0100163
:10C5A00043EA4E0343EA860343EAC20319430DF00C
:10C5B0009FF904A9042220460DF057F92368297831
:10C5C00020465E1C4B4A2660197011886429A8BF5A
:10C5D00064210DF08DF9B9F1960F4DD00021204660
:10C5E0000DF086F9B7F11903256805A9204648BF63
:10C5F000A7F112036E1CA3F3C40326601A462B7026
:10C600000DF033F9236810213B4A5D1C204625605C
:10C61000197011880DF056F90120FFF7F1B839466D
:10C6200004A80DF095FC9DE7F4EEC87AF1EE10FA3F
:10C6300041DA4FF47A71FFF7C8BA0B68B178581C29
:10C640002E4A2060197023681278591C21601A70D4
:10C65000D4E40827FFF7A5BB40F2DC51FFF7B5BAD9
:10C66000236801201A1822601E70FFF7C9B8069BC4
:10C6700043F00103069362E723680322591C2160FB
:10C680001A7023686A78591C21601A70AAE7042777
:10C69000FFF787BB40F2F312A3F5836302FB03F3BA
:10C6A0008AFB0312D9171344C1EB632101F2DD5158
:10C6B00089B2FFF78ABAFDEEE77A40F2E73217EE69
:10C6C000903A303B02FB03F38BFB0312D917C1EB0B
:10C6D000622101F2E93189B2FFF777BA04910120B2
:10C6E000D0890120E49D01209C1D0120B634012049
:10C6F000E0800120FE2C0120309E0120802E0120B0
:10C7000090E33FF40228094B094928BF022000EBBF
:10C710008002C0EBC20230B4064D441C03EB42035E
:10C720002870E0B20B6030BC24F0A2B8D6340120EF
:10C73000C8340120B634012008B51DF0DBFD0CF033
:10C7400065FEBDE808401DF0BDBD00BF434B9989A3
:10C750005A89914210B501D300225A81198ADA8987
:10C76000914201D30022DA81DA78072A18BF002A21
:10C770003B4A3CD092F85B2001213A4C00200A2A27
:10C7800099702170D8715FD00C2A5BD1364CDFEDE7
:10C79000377AA278062A3DD92179DFED356A00295A
:10C7A00040D19B782F4A07EE103A1178B8EEC77A3D
:10C7B00027EE277A07EE901AF8EEE77A67EE877A87
:10C7C000F4EEE76AF1EE10FA3BDDC6EE877AFDEE95
:10C7D000E77A17EE903A102BA8BF1023012BB8BFB1
:10C7E0000123DBB28B4238BF0B46137010BD92F8A9
:10C7F0005B200A2A2BD00C2ADA792CD1DFED1D7AA6
:10C80000002A9FED1B7A18BFF0EE477A164CA278EB
:10C81000062AC1D8184901EB8201D1ED146A2179A9
:10C820000029BED0013A032A0BD8B7EE000A80EEE9
:10C83000260A2CF0FFFC2388984228BF1846208047
:10C8400010BD10BD0A2AA1D1DFED0C7ADEE7DA793E
:10C85000DFED0B7AD4E7DFED0B7AD1E7EC75012041
:10C8600000760120802E0120309401206F12833A3F
:10C870006F1203380AD7A3399CB703080F506E3ADA
:10C880005304E9386F1203392DE9F047B44F1DF016
:10C8900031FDB44EBE421ED2DFF85483DFF854930C
:10C8A0004446258862197DB14A450DD2052D0BD924
:10C8B00033886188C3F30B03994200F0F780144674
:10C8C00025886219002DEFD17168304614360CF0BE
:10C8D00028FDBE42E4D3A44A1378A3F1170102292C
:10C8E00014D9A24911F83300002800F03481D8008F
:10C8F0000C186468002C00F030810144497829B19B
:10C900009B4911F833300BB918231370994C637895
:10C91000022B01D9002363702378022B00F2E780F9
:10C92000954B9A78042A00F0E98022B91A88B2F56A
:10C93000F07F00F20C81914D914A2B681A40002A39
:10C9400000F05A81D80700F1E680590400F1EA802E
:10C950001A0700F1EE809B0400F1F280894D2B68EC
:10C96000998C5A8C914201D300225A84FFF7EEFE33
:10C970001AF04CFA002800F0CA8040200CF008FDA4
:10C980004FF400700CF004FD4FF400300CF000FD8B
:10C990004FF400100CF0FCFC4FF000700CF0F8FCB1
:10C9A0004FF080600CF0F4FC6378022B06D803EBA8
:10C9B0004303754A754902EB83030B602378022B0E
:10C9C00007D803EB8301724AC3EBC10302EB4303B5
:10C9D0002B6022F0D1FC002130226E482EF045FD64
:10C9E000286820F061FE6C4B2D6803F1500102E0D5
:10C9F0000433994279D01A78002AF9D19C78D878F2
:10CA00008442F5D265492846654B0A701D6015F0D1
:10CA100013FD644AC8236448642115790022634CDD
:10CA200011FB0531624F634B30F8066C624DA46B0D
:10CA3000596038602E809A60DA601A615A619A6192
:10CA4000DA6183F8202083F821200CB112F076FE01
:10CA50005A4B9FED5B5A1B885A4A06EE903A9FED5F
:10CA60005A6A1388F8EEE66A557907EE103A538849
:10CA70001479C5EE265A07EE903A544B5449554A5C
:10CA80005548B8EEC77A1D72F8EEE77A5C7210600E
:10CA900027EE067A67EE867ABDE8F04783ED017AE5
:10CAA000C3ED007AC1ED005A1DF00CBC63799B0701
:10CAB0007FF405AF7168304694F804A00CF031FCA7
:10CAC0003388BAEB133F04D01436BE42FFF4E8AE0D
:10CAD00001E77388AA1FA11D7068C3F30B039A4274
:10CAE000A8BF1A462CF0E2F9EEE701228AE70023FC
:10CAF0002370214B9A78042A7FF417AF9A8AB2F5F3
:10CB00007A7FBFF418AF4FF47A729A8213E73348F2
:10CB100022F06AFF31E732480CF03AFC2B685904E6
:10CB20007FF516AF2F480CF033FC2B681A077FF502
:10CB300012AF2D480CF02CFC2B689B047FF50EAF38
:10CB40002A480CF025FC40200CF022FC06E74FF4AC
:10CB5000F0721A80EFE6D800CFE617241470CCE606
:10CB60002C060008E0010008182F012018E0030837
:10CB700070DA0308B63401203094012048360120D1
:10CB800009600002C8340120DE350120F89101203F
:10CB9000D6340120D02A01201C2F0120DF220120C1
:10CBA000042B0120002D0120922E012070800120F5
:10CBB000BC9D01200C9E0120D83201202C2901208F
:10CBC000C0C9FB484425012017B7D138782B012074
:10CBD000302901209C2B01203661023DDCA301207D
:10CBE0000860000209200002016000020940000202
:10CBF000024000080080000843F400532B60A1E6C7
:10CC000008B51DF077FB0CF001FC1DF05BFBFFF796
:10CC10003BFE0120BDE8084023F02ABE38B50D4C8C
:10CC20000D4DAC4206D26168204614340CF079FBFD
:10CC3000AC42F8D30DF0B6FE084C094B0022094D6A
:10CC400009490A481A705A7025600860BDE83840E2
:10CC500027F016BFE00100082C060008C8340120A8
:10CC6000B6340120D6340120F8910120DE350120B0
:10CC700008B5FFF7D3FF1DF03DFB0CF0C7FBBDE887
:10CC800008401DF01FBB00BF01302DE9F04FC3B2BB
:10CC900085B08D4C03930B4602918C4E002B00F017
:10CCA000998019F065FA8A4D4FF4FA7A894FDFF8C6
:10CCB00028924FF0100C4FF47A70D9F80430C3F377
:10CCC0000803002B40F0DE80EFF31183002B40F0CF
:10CCD000D9802968A26800BF2B689942F9D1D7F89A
:10CCE00000E000FB0EF39B1AB3FBFEF300FB0131E7
:10CCF0004FF0010E0191D9F80430C3F30803002B63
:10CD000040F08780EFF31183002B40F082802B6886
:10CD1000A16800BF2A689342F9D1D7F800B000FBA0
:10CD20000BF2521AB2FBFBF200FB0323019A9B1A8F
:10CD3000B3F57A7FDFD3BAF1010ABED1039B002B92
:10CD400040F0BD804FF47A7ADFF88C914FF0100CF0
:10CD50005046D9F80430C3F30803002B75D1EFF324
:10CD60001183002B71D12968A26800BF2B689942FA
:10CD7000F9D1D7F800E000FB0EF39B1AB3FBFEF3EA
:10CD800000FB01314FF0010E0191D9F80430C3F3DB
:10CD9000080313BBEFF31183FBB92B68A16800BF35
:10CDA0002A689342F9D1D7F800B000FB0BF2521A6F
:10CDB000B2FBFBF200FB0323019A9B1AB3F57A7FC7
:10CDC000E3D3BAF1010AC4D1029B013B0293002BC9
:10CDD0007FF467AF05B0BDE8F08FEFF311888CF3F7
:10CDE0001288A1682368DB0302D5C6F800E0A168B9
:10CDF0002B685FFA88F8326888F31188D7F80080CA
:10CE00001A4400FB08F35B1AB3FBF8F300FB023390
:10CE1000D2E7EFF311888CF31288A1682368DB0353
:10CE200002D5C6F800E0A1682B685FFA88F832687E
:10CE300088F31188D7F800801A4400FB08F35B1AC6
:10CE4000B3FBF8F300FB023370E7EFF311828CF3CE
:10CE50001288D4F808E02368D90303D5012333608E
:10CE6000D4F808E02B68D2B2316882F311883A68AE
:10CE7000194400FB02F3A3EB0E03B3FBF2F300FB38
:10CE800001317FE7EFF311828CF31288D4F808E0C8
:10CE90002368D90303D501233360D4F808E02B6855
:10CEA000D2B2316882F311883A68194400FB02F368
:10CEB000A3EB0E03B3FBF2F300FB013118E71846B6
:10CEC00023F088FF3EE700BF10E000E0A0A20120B1
:10CED000A4A20120A8A2012000ED00E0214B5B6884
:10CEE000C3F3080310B4C3B9EFF31183ABB91E4BFE
:10CEF0001E4C1868A16800BF1A689042F9D11C4BFB
:10CF00004FF47A721C6802FB04F3591AB1FBF4F176
:10CF10005DF8044B02FB00107047EFF31182102301
:10CF200083F3128811498C680B6813F4803F114B0E
:10CF300002D0012018608C680B49D2B209681868C9
:10CF400082F311880A4B4FF47A720844196802FB85
:10CF500001F31B1B5DF8044BB3FBF1F302FB003044
:10CF6000704700BF00ED00E0A4A2012010E000E047
:10CF7000A8A20120A0A201202DE9F84F8046102789
:10CF8000FFF7ACFF244E844624494FF47A74DFF84F
:10CF900098E00120224A234DDEF80430C3F3080351
:10CFA000D3B9EFF31183BBB90B68D2F808A000BF67
:10CFB000D1F800904B45F7D1D6F800B004FB0BF93F
:10CFC000A9EB0A09B9FBFBF904FB0393A3EB0C03E0
:10CFD0004345E1D3BDE8F88FEFF3118A87F3128858
:10CFE000D2F808B01368DB0302D52860D2F808B085
:10CFF0000B685FFA8AFAD5F800908AF31188D6F8A0
:10D0000000A0994404FB0AF3A3EB0B03B3FBFAF370
:10D0100004FB0933DAE700BFA8A20120A4A2012083
:10D0200010E000E0A0A2012000ED00E02DE9F04FAB
:10D03000DFF830C180461027464A4749474E484DE1
:10D0400018F1FF38C0F08480DCF80430C3F3080323
:10D05000002B5CD1EFF31183002B58D10B6894683F
:10D0600000BF08688342F9D1D6F800904FF47A7077
:10D0700000FB09FEAEEB040EBEFBF9FE00FB03EE67
:10D08000DCF804304FF47A740120C3F30803FBB9D1
:10D09000EFF31183E3B90B68D2F808A000BFD1F811
:10D0A00000904B45F7D1D6F800B004FB0BF9A9EB83
:10D0B0000A09B9FBFBF904FB0393A3EB0E03B3F5D9
:10D0C0007A7FBDD2DCF80430C3F30803002BDFD035
:10D0D000EFF3118A87F31288D2F808B01368DB03E4
:10D0E00002D52860D2F808B00B685FFA8AFAD5F842
:10D0F00000908AF31188D6F800A0994404FB0AF343
:10D10000A3EB0B03B3FBFAF304FB0933D5E7EFF30F
:10D11000118487F31288D2F808901368D80303D5D6
:10D1200001232B60D2F808900B68E4B2286884F3DE
:10D1300011884FF47A74D6F800A000EB030E04FBBC
:10D140000AF3A3EB0903B3FBFAF304FB0E3E97E7E4
:10D15000BDE8F08F10E000E0A4A20120A8A2012009
:10D16000A0A2012000ED00E030B4EFF31183102203
:10D1700082F3128808490025084CDBB20A68084887
:10D1800001320A602560026883F31188054A13683A
:10D19000013330BC13607047A4A20120A0A201207B
:10D1A00010E000E0B87F0120104B01461B8843B916
:10D1B0000F4B104A1B7810680BB981F001010BF07E
:10D1C00085BF0D4B5A6982B118B91A68106058743E
:10D1D00070470A4801210A4A10B40488186892FB73
:10D1E000F4F25DF8044B0260597470474C930120CF
:10D1F0004E93012050930120549301206C93012001
:10D2000020A1070003682DE9F041DF691FB13B460B
:10D21000BDE8F0411847002A164611DD04460D46C8
:10D220000E4400E023689B68204698470028F9D008
:10D230002368204615F8011B1B689847AE42F1D1C0
:10D24000BDE8F08103689B69184700BF03685B690C
:10D25000184700BF03681B69184700BF0368DB68F5
:10D26000184700BF03685B68184700BF03681B6866
:10D27000184700BF38B50C46097849B10546013456
:10D280002B6828461B68984714F8011B0029F7D122
:10D2900038BD00BF01230B4A10B483400A4C1278FA
:10D2A00054F82000134031B9B3FA83F15DF8044B10
:10D2B00049090BF00BBF191C5DF8044B18BF012185
:10D2C0000BF004BF3C9301204093012008B50121DD
:10D2D0000220FFF7DFFF094B1B7803F00503052B46
:10D2E00008D000210120FFF7D5FF00210846FFF7F5
:10D2F000D1FFFEE720F0B8FDF3E700BF086B012087
:10D30000054B53F8203033B11A689B8851690B42A2
:10D3100018BF1B0493617047409301202DE9F04F23
:10D320002DED028B93B083461AF082FF8C4B1D7853
:10D3300025B113B0BDEC028BBDE8F08F894B1B68A3
:10D340005C05F6D5884BDFF87C821B686BB1874A99
:10D35000D8F800101368CB1A7C2B06D984481160CA
:10D360000378013303701AF019FC824B1B78002BF1
:10D370006DD0814C814AD4F81031ABEB030393425A
:10D3800001F2E68294F81891B9F1000F32D17C4F86
:10D390003868FFF767FFC0B201280FD9022841F0B3
:10D3A000AC87784E3378002B42F0E580D4F81C31FE
:10D3B000ABEB0303B3F57A6F82F0A982D4F8203186
:10D3C000002B44D094F81831BBB96F4B01210022D7
:10D3D0001B6884F818119B7884F82C211E3B8B4223
:10D3E00042F24F8238680221043018F076FE94F839
:10D3F000243110E0D4F820314BB3D4F8283140F672
:10D40000B732ABEB0303934221D994F82431002BBC
:10D4100001F074865A4F013BDBB284F82431002BB3
:10D4200001F0BC83D4F8206194F82C2116F8011B7C
:10D4300094F82D310A4438680133C4F8206184F827
:10D440002C2184F82D31FFF711FFC4F828B14F4B80
:10D45000D8F800601B7843B14D4F386828B14D4B68
:10D460001B78013B012B41F2A8834B4B1B7863B126
:10D470004A4F3B684BB1404CD8F80090D4F8443147
:10D48000A9EB0303632B00F2E780454F3B78022BA7
:10D4900001F014863B4E96F87430032B01F069833B
:10D4A000404B1B7873B1404D2B685BB1324CFFF79A
:10D4B00015FD44F61F620290D4F85031C31A93420E
:10D4C00000F2A681394B1B78002B7DD1384B1B789D
:10D4D0003BB1294C374BD4F8A02213449B4581F033
:10D4E000E281354B1B78002B3FF423AF224E334CA7
:10D4F00006F2C127324D2068FFF7B4FE00283FF442
:10D5000018AF2068FFF7AAFE2B7880465A1E33B169
:10D5100020682A70FFF7A6FE0028F2D109E703224F
:10D520003946781E2DF087FF96F8C0124FF6FF732C
:10D5300096F8C12286F8C3821FFA88F84B409B1ADE
:10D540009BB2B8EB132FD6D1DBB296F8C2229A4227
:10D55000D1D1781E18F0CEFA2B7818442870CAE77B
:10D560003C3A0120FC7D012058800120C080012030
:10D57000BC80012092810120542501203F0D030031
:10D58000D075012010000120D47501209481012064
:10D59000AC7301209C810120A4810120C875012069
:10D5A000CE870120AC810120B08101201C820120A6
:10D5B0002D820120A0860100B6810120BC810120BE
:10D5C000C0810120A4A201207D4C2278A2B17D4B14
:10D5D0009B7A53B1FFF782FC7B4B1B68C31AA3F500
:10D5E0007A73B3F5FA6F07D82278784B78491868C0
:10D5F000FFF708FE00232370764C774BD4F898226F
:10D6000013449B45FFF462AF744DC4F898B22B7875
:10D61000002B41F0AD86724D2B78002B41F0068631
:10D62000704994F89C228D5CE80701F1E987A9070D
:10D6300001F1A7876A0701F16B872A0701F11C87AF
:10D6400094F89C32684A0133117893FBF1F201FBA4
:10D65000123384F89C3239E7644E412018F0EAFC1A
:10D66000634AB6F90230029282FB0310DB17DFF83F
:10D670009CA1C3EBA00080B218F0C0FCB6F900304A
:10D68000029A82FB0310DB17C3EBA00080B218F0F4
:10D69000B5FCB6F90430029A82FB0320DB17C3EB1A
:10D6A000A00080B218F0AAFC9AF800103868FFF7C2
:10D6B000DDFD94F8482112F0010601F042854D4B42
:10D6C0001B689B066CD54C4B1B78980742F1E18098
:10D6D0004A4E337D042B8CBF032302230293472041
:10D6E00018F0A8FC306818F051FC706818F04EFC77
:10D6F000F389434A3868A2FB0323C3F3471319464F
:10D700000393FFF7B3FD9AF80010039B642032895E
:10D710004B4000FB02F08AF8003018F037FC029B07
:10D72000367D386843EA8606F6B23146FFF79EFD3D
:10D730009AF8003038685E4031468AF80060FFF79A
:10D7400095FD94F848215ABB2E4E4F20029218F0B6
:10D7500071FC306818F01AFC706818F017FC029A17
:10D76000104618F013FC01213868FFF77FFD224AAC
:10D770009AF80030167883F00103386806F0010645
:10D780008AF800303146FFF771FD9AF800303868AA
:10D790005E4031468AF80060FFF768FD94F8482142
:10D7A000531C194AC4F84491DBB2A2FB0312D208FD
:10D7B00002EB8202A3EB420384F8483165E600BF26
:10D7C00084810120707F0120408701202082012078
:10D7D0004481012054250120A086010024820120DB
:10D7E00025820120288201202C820120C480012072
:10D7F00067666666E0800120E4800120E880012001
:10D800001F85EB51F09E0120CDCCCCCCCC750120F6
:10D8100094F85631002B41F08F84D74A4AF60B47D3
:10D8200048F603404BF60F43126849F6074602F0EC
:10D83000080100294FF0190104BF3B46064612F0CB
:10D84000040F84F8561118BF1E46910603D546F4FE
:10D85000804646F02006C94AC6F3090351790029DB
:10D8600042F081809279002A42F08F8191466420B3
:10D870004FF0FF3A00220C930121FE230AAF0A96D3
:10D880000B964FF01F0EADF83690ADF838A08DF81E
:10D890004600ADF83420CDF83A20CDF83E20CDF842
:10D8A00042206271E171A370B54E84F803E00FCF9E
:10D8B0000FC697E80F0007C61A0C26F8023BC823CC
:10D8C0003146701CA37101F81E2994F8662182F07C
:10D8D000F103561C227183EA031384F86661DAB2FD
:10D8E000130983F0E70343EA022383EAC2031BB26E
:10D8F00083EA0312C3F30723D2B283EA121343EA83
:10D90000022383EAC2031BB283F0C802C3F30723D6
:10D9100082EA0212D2B283EA121343EA022383EAB2
:10D92000C2031BB283F00106C3F3072286EA061383
:10D93000DBB282EA131242EA032282EAC3021646EB
:10D94000228011F8013B7340814283EA0313DBB26A
:10D950004FEA131282EA162242EA032282EAC30342
:10D960001BB29EB22680ECD183F07C03854F04F17C
:10D97000220A83EA031307F5C77CDBB24FEA131EC2
:10D980008EEA162E8EEA032E8EEAC30E0FFA8EFE54
:10D990001FFA8EF35FFA8EFE4FEA1329238084F874
:10D9A00027E084F828903868103757F80C1C664632
:10D9B00057F8082C0CF1100C57F8043C57450FC6CB
:10D9C000F1D13868704ECCF800003B7906F127079A
:10D9D0008CF8043084F8B5E184F8B69116F8011F8C
:10D9E0002868FFF743FCB742F8D194F85711002993
:10D9F00041F01784654B0A22D8F800001B78039089
:10DA000084F85721002B01F02785614A012BB2F8D9
:10DA100000C042F2C680022B568801F0C087908871
:10DA2000032B059002F0D480042BB2F806E002F03C
:10DA3000CA80052BB2F8089002F0C180062BB2F81C
:10DA40000AA002F0B980072B908900D0D18994F800
:10DA5000663100274F4A069383F030036CF30F07BB
:10DA6000128883EA031366F31F47039EDBB2C2EBFF
:10DA700002220A960493049B474E0B971F0986FBCC
:10DA8000026C0023059E87F07A07CDF81CC066F370
:10DA90000F03079EDDF818C06EF31F4316444FF0C6
:10DAA000000ED2170393049BC2EB6622764669F3FD
:10DAB0000F0E47EA03278DF83D2060F30F066AF347
:10DAC0001F4E87EAC303624661F31F46CDF834E078
:10DAD0001BB24FF0C80E01324FF0230A83EA031144
:10DAE000C3F30729039B0020C9B284F866210C9375
:10DAF0000AAF89EA111384F804C04FF0160C84F8B9
:10DB000006E043EA01230E9684F803C04FF0FE09B5
:10DB100083EAC1038DF83C0060711BB2184E84F893
:10DB200007A083EA0E02C3F3072384F8029082EA77
:10DB30000211C9B283EA111242EA012282EAC10249
:10DB400012B282EA0A03C2F3072E83EA031C5FFAC9
:10DB50008CFC0FCF8EEA1C1E0FC64EEA0C2397E8F2
:10DB6000030083EACC0346F8040BB01C26F8141912
:10DB70001946238012E000BFE0800120CC80012004
:10DB80005C25012056250120E32601203486012052
:10DB90005C9E0120069E01200308208016F8012BC0
:10DBA0004A40864282EA0212D2B24FEA121383EA54
:10DBB000112343EA022383EAC20212B291B2218006
:10DBC000ECD182F0F402DFF8EC9304F28F1604F249
:10DBD000AD1782EA0212D9F8000009F5C77CD2B26B
:10DBE0004FEA121E8EEA112E8EEA022E8EEAC20E25
:10DBF0000FFA8EFE1FFA8EF35FFA8EFE4FEA132A9B
:10DC0000238084F81EE084F81FA0D9F80410D9F806
:10DC10000820D9F80C30ACE80F00D9F81000D9F87A
:10DC20001410D9F81820ACE8070084F8ADA184F8E6
:10DC3000ACE116F8011F2868FFF718FBB742F8D1CE
:10DC400094F85A31002B41F0DC82D64B19221B6824
:10DC500084F85A219A0640F1FB82D34B1B789B072C
:10DC600041F17C86D14E337D042B8CBF4FF0030AEB
:10DC70004FF0020AFFF732F9338A32894FF47A7192
:10DC800003EB83030A900AAF01FB02F230685B00EA
:10DC90000E92BE46ADF842304FF000090C904FF0A6
:10DCA000FF31F3894FF0C80C327D70688DF844A0C5
:10DCB0004FF0180A0D90ADF840308DF84520CDF8A2
:10DCC0002C900F910397BA4FBEE80F000FC79EE844
:10DCD0000F0007C73A461E20B91CFE2722F81C3940
:10DCE00094F866E1E0708EF07803A77084F804E0A1
:10DCF0000EF1010E83EA031384F807A084F805905F
:10DD0000D8B284F866E184F806C0030983F0F6030C
:10DD100043EA002383EAC0031BB283EA0310C3F380
:10DD20000723C0B283EA101343EA002383EAC00347
:10DD30001BB283EA0C00C3F3072380EA0017FFB28B
:10DD400083EA171040EA072080EAC70000B280EAA1
:10DD50000A07C0F3072387EA0710C0B283EA10134B
:10DD600043EA002383EAC0031F46238012F8010B15
:10DD700078408A4280EA0010C0B24FEA101383EA6A
:10DD8000172343EA002383EAC00000B287B227804A
:10DD9000ECD180F01800874A04F1220980EA0010D3
:10DDA0000592964602F5C77CC0B24FEA101A8AEA7D
:10DDB000172383EA002A8AEAC0000FFA80FA1FFAC2
:10DDC0008AF35FFA8AF2190A23800492069184F892
:10DDD000262084F82710DEF800000EF1100E5EF801
:10DDE0000C1C67465EF8082C0CF1100C5EF8043C25
:10DDF000CE450FC7EFD1DEF800006F4FCCF8000022
:10DE00009DF8103007F12609BA4684F8B4319DF820
:10DE1000183084F8B5311AF8011F2868FFF726FA80
:10DE2000D145F8D1FFF75AF8644BDFF898E14FF489
:10DE30007A7CB3F90430002132898EFB039E4FEACD
:10DE4000E37933680CFB02F276684FF01C0C0B93FD
:10DE5000C9EBAE030D92ADF8423021230E92FE22A3
:10DE6000DDF80CE00C960A90ADF83C10ADF83E10D1
:10DE7000ADF840106171E371A2704D4E84F803C09B
:10DE8000BEE80F000FC6C82206F10C03A271A3F171
:10DE90001C0C9EE8070086E8070094F8661181F0E4
:10DEA0006A02481C217182EA021284F86601D1B22A
:10DEB0000A0982F0D50242EA012282EAC10212B2C4
:10DEC00082EA0211C2F30722C9B282EA111242EABF
:10DED000012282EAC10212B282F0C801C2F3072213
:10DEE00081EA0111C9B282EA111242EA012282EAF0
:10DEF000C10212B282F02100C2F3072180EA0012AF
:10DF0000D2B281EA121141EA022181EAC201084635
:10DF100021801CF8012B42409C4582EA0212D2B2B9
:10DF20004FEA121181EA102141EA022181EAC2027C
:10DF300012B290B22080ECD182F068021D4E04F142
:10DF4000220982EA021206F5C77CD2B24FEA121AFF
:10DF50008AEA102181EA022A8AEAC2020FFA82FAC8
:10DF60001FFA8AF35FFA8AFA1A0A238084F824A037
:10DF7000049284F825203068103656F80C1CE646CA
:10DF800056F8082C0CF1100C56F8043C4E45AEE83F
:10DF90000F00F0D13388B946094EACF800309DF837
:10DFA000103011E0E0800120E4800120E8800120B1
:10DFB0005C25012056250120E3260120C480012094
:10DFC000072701206766666684F8B2A184F8B3313A
:10DFD00019F8011F2868FFF749F94E45F8D194F860
:10DFE00066110023DFF814E6312681F0EB020C9372
:10DFF0006371FE20DEF8043082EA021221710131E1
:10E00000D2B20B93DEF800304FF00C0E84F866119C
:10E01000C8210A931309E67183F0C503DFF8E09580
:10E02000A07043EA0223A17184F803E083EAC203EB
:10E030001BB283EA0312C3F30723D2B283EA12139B
:10E0400043EA022383EAC2031BB283EA0102C3F359
:10E05000072382EA0212D2B283EA121343EA0223AE
:10E0600083EAC203039A1BB25E40C3F3072386EA26
:10E070000616F6B283EA161343EA062307CA83EAB2
:10E08000C603A9F5C4761BB286E80700267A607A33
:10E090005E40C3F30723A17A86EA0616E27A94F873
:10E0A0000CE0F6B294F80DC094F80EA083EA1613B3
:10E0B00043EA062383EAC603E67B1BB25840C3F358
:10E0C000072380EA0010C0B283EA101343EA00235A
:10E0D00083EAC003207C1BB25940C3F3072381EAC3
:10E0E0000111C9B283EA111343EA012383EAC10390
:10E0F000617C1BB25A40C3F3072382EA0212D2B2F8
:10E1000083EA121343EA022383EAC203A27C1BB20E
:10E110008EEA030EC3F307238EEA0E1E5FFA8EFE0D
:10E1200083EA1E1343EA0E2383EACE0394F813E036
:10E130001BB28CEA030CC3F307238CEA0C1C5FFAB6
:10E140008CFC83EA1C1343EA0C2383EACC031BB246
:10E150008AEA030AC3F307238AEA0A1A5FFA8AFAE9
:10E1600083EA1A1343EA0A2383EACA031BB25E4016
:10E17000C3F3072386EA0616F6B283EA161343EAC8
:10E18000062383EAC6031BB25840C3F3072380EA81
:10E190000010C0B283EA101343EA002383EAC003ED
:10E1A0001BB25940C3F3072381EA0111C9B283EAC4
:10E1B000111343EA012383EAC1031BB25A40C3F39C
:10E1C000072382EA0212D2B283EA121343EA02233D
:10E1D00083EAC2031BB28EEA030EC3F307238EEA5F
:10E1E0000E1E5FFA8EFE83EA1E1343EA0E2383EAB5
:10E1F000CE031BB283F02706C3F3072386EA061279
:10E20000D2B283EA121646EA022686EAC20636B27D
:10E21000B3B25FFA86FA23804FEA132E059E84F884
:10E2200014A084F815E030687168B268F368B6F835
:10E2300010C0A9E80F0029F803CB84F8A3E184F803
:10E24000A2A117F8011F2868FFF710F8B945F8D107
:10E2500094F85E21002A40F0DF87DF4E052094F815
:10E2600066C10DF1280EB6F90270B6F900108CF0F7
:10E270006A0362711E2206EE901A794283EA031342
:10E28000E27107EE901AB6F90410FE22D8F8006089
:10E2900007EE101AD9B2A2701C220B090A96E2707E
:10E2A000C82283F0D503F8EEE66AA271F8EEE77AA9
:10E2B00043EA0123B8EEC77A9FEDC86A002783EAD4
:10E2C000C10384F85E0166EE866A0E971BB267EEA4
:10E2D000867A27EE067A0F9783EA0311C3F30723A2
:10E2E00010970CF10108C9B2CDED0B6ACDED0C7A97
:10E2F00083EA11138DED0D7AB94F43EA012383EAC6
:10E30000C1031BB25A40C3F3072382EA0212D2B2FE
:10E3100083EA121343EA022383EAC2031BB283F0A7
:10E320001E06C3F3072386EA06195FFA89F983EA12
:10E330001916BEE80F0046EA09260FC786EAC90685
:10E3400007F10C039EE80700A7F1100E87E807000D
:10E3500084F804C0268084F866811EF8012B724080
:10E360009E4582EA0212D2B24FEA121181EA1621C8
:10E3700041EA022181EAC20212B296B22680ECD1B1
:10E3800082F02702974F04F1220982EA021207F570
:10E39000C77CD2B24FEA121E8EEA162E8EEA022EE9
:10E3A0008EEAC20E0FFA8EFE1FFA8EF35FFA8EFE11
:10E3B0004FEA1328238084F824E084F82580386805
:10E3C000103757F80C1C664657F8082C0CF1100C47
:10E3D00057F8043C4F450FC6F1D1834E3B8806F1F8
:10E3E0002407ACF8003084F8B2E184F8B38116F861
:10E3F000011F2868FEF73AFFB742F8D194F85F9101
:10E40000B9F1000F40F00287784B05221B6884F8B1
:10E410005F219F0641F12A80754BDFED766ADA892C
:10E420001B8907EE902A07EE103AF8EEE77AB8EE6D
:10E43000477A67EEA67A94F866610AAB6E4A4FF0A7
:10E44000640E86F022011F46B2F9062081EA01110E
:10E450000393B2F5FA6F604BC9B2DFF8A8C1A8BF49
:10E460004FF4FA62B3F904000B092671B2F57A7F12
:10E4700006F1010683F05903CDED0B7AB8BF4FF4D6
:10E480007A7284F8666143EA01238DED0C7AA2F575
:10E490007A7283EAC1030EFB02F2DFF86CE11BB271
:10E4A0008CFB026CD2178EFB001E0021C2EBAC125B
:10E4B0004B4E83EA031CC3F30723ADF83A204A22EC
:10E4C0005FFA8CFC0A91E271FE2283EA1C130D9123
:10E4D000A270142243EA0C23C821E270002283EACE
:10E4E000CC03A1716271C0171BB2C0EBAE0083EA0E
:10E4F0000102C3F30723ADF8380082EA0212D2B258
:10E5000083EA121343EA022383EAC2031BB283F0B5
:10E510004A0EC3F307238EEA0E1C5FFA8CFC83EAD3
:10E520001C1E0FCF4EEA0C2E3F688EEACC0E0FC693
:10E53000A4F800E0321D46F8107916F8013B83EA92
:10E540000E03964283EA0313DBB24FEA131181EA0A
:10E550001E2141EA032181EAC3031BB21FFA83FE95
:10E56000A4F800E0E9D183F014031E4A04F2AB18CA
:10E5700083EA03131146059204F28F12DBB2086896
:10E58000164601F5C77C1A093746049682EA1E2E04
:10E590000E468EEA032E8EEAC30E0FFA8EFE1FFA87
:10E5A0008EF35FFA8EFE4FEA132A238084F81CE074
:10E5B00084F81DA0F3684968B268ACE80F003069C0
:10E5C0007169338B3E46ACE80300ACF8003084F848
:10E5D000ABA184F8AAE119E0C480012088C3E43A21
:10E5E0005C25012056250120E3260120E080012042
:10E5F000E88001200AD7233C5C9E0120F09E012088
:10E60000E4260120D34D62106766666617F8011F85
:10E610002868FEF72BFEB845F8D1C44BC44A1B78D6
:10E620001278013B049612F00101DBB214BF4FF0E7
:10E63000C00E4FF0400E172B03D8BE4A134493F878
:10E640003090BD4B1B889E0700F05F874EF0100E88
:10E65000002213F4027F18BF022213F0100F18BF1C
:10E66000062213F0200F18BF1022002941F0478125
:10E67000032794F8660103230A92002180F04602E2
:10E680008DF8303000F10108207182EA0212C820B2
:10E690008DF82F700927D2B28DF82C90E7704FF0CB
:10E6A000FE0C13098DF82EE08DF82D1083F09203E7
:10E6B000E171617143EA0223A071DFF890E283EA1D
:10E6C000C20384F8668184F802C01BB283EA031295
:10E6D000C3F30723D2B283EA121343EA022383EA85
:10E6E000C2031BB283EA0002C3F3072382EA0212C9
:10E6F000D2B283EA121343EA022383EAC203039AE3
:10E700001BB283EA0317C3F30723FFB283EA17138D
:10E7100043EA072307CA83EAC703AEE803001BB234
:10E72000207A617A0EF5C07C5840C3F3072394F831
:10E730000A800EF5C87780EA00108EF80020E27A91
:10E74000C0B294F80CE094F80DA083EA1013A67BF5
:10E7500094F8109043EA002383EAC003E07B1BB2E5
:10E760005940C3F3072381EA0111C9B283EA1113A7
:10E7700043EA012383EAC1031BB288EA0308C3F317
:10E78000072388EA08185FFA88F883EA181343EA2F
:10E79000082383EAC8031BB25A40C3F3072382EA63
:10E7A0000212D2B283EA121343EA022383EAC203BB
:10E7B0001BB28EEA030EC3F307238EEA0E1E5FFA26
:10E7C0008EFE83EA1E1343EA0E2383EACE031BB2B6
:10E7D0008AEA030AC3F307238AEA0A1A5FFA8AFA63
:10E7E00083EA1A1343EA0A2383EACA031BB286EABE
:10E7F0000302C3F3072382EA0212D2B283EA12139E
:10E8000043EA022383EAC2031BB25840C3F307233F
:10E8100080EA0010C0B283EA101343EA002383EABF
:10E82000C0031BB289EA0302C3F3072382EA021280
:10E83000D2B283EA121343EA022383EAC2031BB271
:10E8400083F03202C3F3072382EA0212D2B283EAD0
:10E85000121343EA022383EAC2031BB29AB2DBB269
:10E860004FEA122E2280637484F812E0059E30680D
:10E870007168B268B6F80C80049EACE807008CF8AA
:10E880000290ACF8008084F8A0E184F89F3116F87B
:10E89000011F2868FEF7EAFCB742F8D1029BC4F8D2
:10E8A0005031FEF70FBE94F8A432224AC4F8A0B249
:10E8B00002EB8302926C5AB312AD04F2AB2104F264
:10E8C000BD234FF0000E45F8201DA52680211B4FCB
:10E8D0000B9315232846A7F800E084F8AA3284F8A1
:10E8E000A86204F52A7684F8A91290472846398848
:10E8F0000AF0FEFF0A9D31461148AD1B152DA8BF39
:10E9000015252A462AF0D2FA0E4A94F8A432157038
:10E9100001330D4A82FB0312A2EBE37202EB4202C7
:10E920009B1A84F8A432FEF7DCBD00BF182F01202B
:10E93000D089012008B80308849E01205C80012052
:10E940001C85012031850120565555555C25012037
:10E95000C14A4FF47A71C14B0027D07AD8F80060D1
:10E9600001FB00F1D4F814011B88301ABC4A5FFA8D
:10E9700083FE88424FEA132382F81EE0D37782F8A1
:10E9800014E053759770177180F05A84B5494FF0B1
:10E99000F40EB54801270B684FF03009896880FBF9
:10E9A00003C6DB1780FB01C0C917C3EBA603AF4E3C
:10E9B000C1EBA001AE4813771B1200784FEA212A61
:10E9C00053774FF0750C82F820108007317DA94BEA
:10E9D00082F81AE04FF0780E82F821A09976D77667
:10E9E00082F8229082F823C082F824E040F1258446
:10E9F00072680529D6F800C011469F4F4FEAEC70A7
:10EA0000DFF8889287FB0CE2DFF884A287FB01E73E
:10EA10004FEAE17EC0EBA2500291CEEBA75E09FB6C
:10EA200000C700EB800009FB0E110EEB8E0E07EB0A
:10EA3000470701EB41014FEA47074FEA410100EB6D
:10EA400080000A468AFB07914FEAE77904904FEA73
:10EA5000A1410392F0898AFB02A20EEB8E0EB6F85A
:10EA600008A0A1EB090600EBC000CDF814E04FEAC6
:10EA7000A242DFF820E23146069076B203980EFB00
:10EA80001171049F0AF5FA7A4FEAE079069806EBCD
:10EA90008706A2EB09074FEA80001FFA86F9039E5A
:10EAA0003A464FEADC7C0EFB17671FFA8AF652B231
:10EAB00083F809C00396059EDFF8DCC102EB860EE1
:10EAC0006E4E6F4A1FFA8EFE83F80A9082FB00A2F8
:10EAD0004FEAE07086FB016A684E04924FEAE171EA
:10EAE00086FB07264FEAE777049AC1EB6A11C7EB6A
:10EAF0006616644FC0EBA210BCF80020B7F800A067
:10EB00004FEA1929029F83F80B904FEA1E294FEA1A
:10EB1000D77CC0F3072783F80FE04FEA262E029731
:10EB200083F80EC04FEA212C039F83F80DC038BF35
:10EB30004FF0320C83F8109028BF4FF0330C19734C
:10EB40004FEA1729110A5E7483F812E09DF80C60F1
:10EB5000D8719DF808005E7583F816901872DA7403
:10EB6000197583F81BC083F81CA0C4F810B1FEF718
:10EB700009BCDFF82891D9F80000FEF767FB0028F0
:10EB80003EF48EACD9F800000121FEF75BFB0222B7
:10EB9000002386F874203B70FEF782BC94F82C1199
:10EBA00094F82D314A1C3868013384F82C2184F8FC
:10EBB0002D31FEF75BFBFEF748BC334C4FF0000AEB
:10EBC000DFF8DC900AE01B2B00F08D820D2B00F0AB
:10EBD00071814FF0010389F801303868FEF742FB7C
:10EBE00000285FD03868FEF739FBD8F8003083B2D0
:10EBF0007E2B2AD099F801100029EED194F82E210D
:10EC0000002AE0D07D2B00F0548294F83CE1BEF164
:10EC1000000F04D080F0200384F83C11DBB2511CBB
:10EC20002244C9B282F83031092984F82E1100F04B
:10EC300034820829D1D8B4F83A21134403EB1323C2
:10EC400003F0FF03A4F83A31C7E784F82EA184F853
:10EC50002FA189F801A0C0E7FC730120F473012003
:10EC6000C48101206080012067666666E88001201B
:10EC7000E4800120F08101206BCA5F6B1F85EB519E
:10EC8000D34D6210FA9E012054250120806967FF50
:10EC900083DE1B4340420F00F89E01202C88012098
:10ECA0001000012094F83D3133B194F8313184F8EB
:10ECB0003D01302B00F0038694F82F21C74BC84943
:10ECC0009146DFF848A3DFF848E34A46002A3EF4BD
:10ECD000CCABD8F80020921B012A24D894F83E210E
:10ECE000002A40F01E8294F83FC133F81C00F8B9A6
:10ECF0004FF0010284F83F210A689706E5D59AF89B
:10ED000000209007E1D5B74E4FF4F363B6494FF4B6
:10ED10000360F28903FB02F381FB0321DB17C3EBE2
:10ED2000611117F0BFF9002384F82F31FEF79DBB66
:10ED30000CF1010CB0F5E06F5FFA8CFC84F83FC178
:10ED400000F097801AD8B0F5047F00F0878134D89E
:10ED5000B0F5887F00F07481B0F5007F00F05A8133
:10ED6000B0F5807FB1D10A685207AED5002117F007
:10ED700099F9002384F82F31FEF777BBB0F5026FC5
:10ED800000F015816AD8B0F5E46F00F08180B0F52D
:10ED9000006F00F09880B0F5E26F96D1934A64233B
:10EDA000166C118B03FB06F393FBF1F117F07AF964
:10EDB000002384F82F31FEF758BBB0F5826F00F0C6
:10EDC000D580B0F5C06F00F0C180B0F5806F7FF4E2
:10EDD0007CAF94F840310133DBB2032B00F29B810E
:10EDE00042F2107184F8403101FB03F1804B1B8823
:10EDF000002B40F08E8101317E4B1B78DB077E4B70
:10EE00001B8848BF0431DF0748BF0A31980748BF55
:10EE100014311A0648BF2831DF0548BF283158078A
:10EE200048BF64311A0748BFC8319F0548BF01F584
:10EE3000C87198064FF4806048BF01F57A71DA0610
:10EE400048BF01F5FA615F0648BF01F57A6117F026
:10EE500029F9002384F82F31FEF707BBB0F5046FC2
:10EE60001BD0B0F5116F57D0B0F5036F7FF42DAF05
:10EE700042E791465D4A6423D66B118B03FB06F390
:10EE800093FBF1F117F00EF984F82F91FEF7EDBA2C
:10EE90009146564A6423566CEFE7584B9146B3F9B6
:10EEA000041001EB8101490017F0FCF884F82F9160
:10EEB000FEF7DBBA4FF0010184F83031A4F83A21B3
:10EEC00084F82E1189E60A6897067FF5FEAE9AF857
:10EED000002090077FF5F9AE1CF0010F414E42492A
:10EEE00000F0DC84726882EAE273002AA3EBE2732A
:10EEF00003EB5303A1FB03314FEAD101ACBF41F057
:10EF0000004141F040414FF4006017F0CBF800237E
:10EF100084F82F31FEF7A9BA9EF80520002A3FF4A5
:10EF2000D4AE374A1278002A3FF4CFAE354B4FF4B7
:10EF300011601B8803EB8303590091FBF2F117F07A
:10EF4000B1F8002384F82F31FEF78FBA9EF806201F
:10EF5000002A3FF4BAAE2C4B4FF4C060996817F00A
:10EF6000A1F8002384F82F31FEF77FBA0A689006D3
:10EF700040F17681254B40F6B8321A4E4FF482604C
:10EF80001F78317D07F00203002B0ABF00234FF4E6
:10EF90007A734FF4FA6217F0010F18BF1346194441
:10EFA00017F080F8002384F82F31FEF75EBA0F685F
:10EFB000BF067FF58AAE9AF800C01CF0020F3FF43E
:10EFC00084AE084E64219146338901FB03F117F0AA
:10EFD00069F884F82F91FEF748BA00BF08B8030813
:10EFE000E0800120E88001201F85EB517080012026
:10EFF000309E0120D0890120849E0120C480012000
:10F000000A740120F473012060800120E480012053
:10F01000CC8001209EF80620002A3FF456AEBF4B5C
:10F020004FF40070BE491B6881FB0321DB17C3EB63
:10F03000A10117F037F8002384F82F31FEF715BA35
:10F040000A6852077FF541AE00214FF4887017F02F
:10F0500029F8002384F82F31FEF707BA9EF805201F
:10F06000002A3FF432AEAF4A107800283FF42DAEAC
:10F07000AD4B5B7B002B00F06A84AC4B1B8893FB91
:10F08000F0F000EB80014FF40470490017F00AF82B
:10F09000002384F82F31FEF7E8B9B4F83A21C2F121
:10F0A000FF0293427FF495AD4FF0010384F83D31A8
:10F0B0008FE54FF0010384F83C318EE5FDF70EFF3C
:10F0C0009B4A40F6B8331268801A984200F21C81BD
:10F0D000DFF898A29AF804303A2B00F0FF82002360
:10F0E0003B70FEF7DDB93868FEF7BCF800287FF406
:10F0F00070AD4FF0010384F82F316EE5C4F8203174
:10F1000084F8183117F01CF88A4F94F82431FEF770
:10F1100082B9023170E6012342F2107184F8403165
:10F1200064E68549062016F089FD002384F83E0137
:10F1300084F82F31FEF799B9013B84F85631FEF778
:10F1400054BC7E4B1B88D90513D4DA0600F1D58355
:10F15000980600F13784590600F13A841A0700F145
:10F160003A84D80700F1558413F0020F0CBF04262F
:10F170000C26734B734A1B78D27803F001030AB153
:10F1800043F0020353201E4316F054FF674B1B88C5
:10F1900003EB830303EB8303980080B216F02EFF8A
:10F1A000002016F02BFF684B684A1B883868C3EBB9
:10F1B000C3135B0082FB0312D9171344C1EB632313
:10F1C000DAB211460292FEF751F8029A9AF800302C
:10F1D0000021386853408AF80030FEF747F831467E
:10F1E0003868FEF743F89AF8003038687340DBB2AD
:10F1F00019468AF80030FEF739F894F84821FEF7EE
:10F20000A2BA013B84F85A31FFF722B809F1FF395D
:10F2100084F85F91FFF742BB013A84F85E21FFF763
:10F22000EDB8013984F85711FEF70ABD48493A2074
:10F2300016F004FD2870FEF749B92D22DA7694E421
:10F24000444BD8F800101B78C4F81411013B012B73
:10F250003FF69CAB1021022391701371FFF796BB10
:10F260003D4A1268120600F132832F4A127B002AAF
:10F270003FF42BAD94F84111032900F2C183DFE87C
:10F2800001F032281902354B1B6859799A7901F13E
:10F290004071DB7901EB022101EB0341002384F88B
:10F2A00041314FF4826016F0FDFE002384F82F31C7
:10F2B000FEF7DBB82A4B1A68137A50791B04927850
:10F2C00003EB002313444A1C03EB016184F8412142
:10F2D000E7E7234B1A68D37910791B04527803EBC4
:10F2E00000231344EFE71E4B1A689379D0781B0470
:10F2F000127803EB00231344E5E716F011FF194ED3
:10F3000001233370FEF75AB8174A0021B2F84A3188
:10F3100039700133A2F84A31FEF7C2B8608001208B
:10F32000676666660A740120FC730120F47301208D
:10F33000D4870120D07501209F600208849E01209F
:10F34000D08901200C9E0120069E01200308208008
:10F35000AD810208099E0120FC7D0120F891012069
:10F36000C83401201000012054250120BC87012051
:10F37000C84E0024C84B0AA8A6F13F01C74A009313
:10F380000891C74BC74906F8404C09960AF093FB11
:10F39000089E2920EA21C822731C08933470089B18
:10F3A0005F1C089718700AA8089B5F1C08971970C3
:10F3B000089B591C08911A7028F06EFD471C0AA979
:10F3C00008983A4629F072FDDDF820E00122FF217D
:10F3D0000EEB070312A8134408930EF80740089B8E
:10F3E0009F1808971C70089B9F1808971C70089B13
:10F3F0009F1808971C70089B9F1808971C70089B03
:10F400009F1808971C70089B9F1808971C70089BF2
:10F410009F1808971C70089B9F1808971C70089BE2
:10F420009F1808971C70089B9F1808971C70089BD2
:10F430009F1808971C70089B9F1808971970089BC5
:10F44000991808911A7050F8283D9B1B337018F0DA
:10F4500079FE2C70FEF73AB818469A4699469E46B1
:10F4600005931E469C461946FEF7F1BADFED8E7AEB
:10F47000B0EE677AFEF7DFBF864B12AD8B4E0020F1
:10F480002F46A3F13D05112103F8400C47F8205DFC
:10F49000022503F83F1C384603F83E5C31680B93A5
:10F4A00003970AF0ECF9384671680AF0E8F9F38935
:10F4B0007F49384603EBC3039B00053381FB0321DF
:10F4C000DB17C3EBA10189B20AF0EFF9338A3846A2
:10F4D00003EB8303590089B20AF0E7F9754B1B78F7
:10F4E0009B0740F13882318901F57A7189B2039D19
:10F4F00028460AF0DAF90A9B327D2846591C0A91FF
:10F500001A7018F01FFEFEF79BB80122FFF7A1B892
:10F51000694A00205F4B21211268A3F140070B9339
:10F5200003F8400CD300B97040F1408203266349D0
:10F53000634B1B88580500F12F82DA0700F14582E2
:10F54000980701D503265F49DFF88C813246404693
:10F5500029F0ACFC06EB0803A8F1020200210133FC
:10F5600012A806F808109A1A40F8203D7A7018F090
:10F57000E9FDFEF762B8C4F81CB186F80090FDF70B
:10F580001DBF444B002712AE4FF00A0C4FF0080E7F
:10F59000A3F13D004C4903F8407C4C4F46F8200D48
:10F5A000304603F83FCC03F83EEC09880B930AF091
:10F5B0007CF93B6830463E49DA1781FB0313C2EB06
:10F5C000A30399B20AF071F9BF6813F0CFFC0A9B4C
:10F5D000390C03F1010E3A0ACDF828E019700A9BA4
:10F5E000591C0A911A700A9B5A1C0A921F700A9B96
:10F5F0005A1C0A921870304618F0A4FDFEF71AB88B
:10F60000334F12AE9FED338AB7F9022007EE902AEE
:10F61000204AF8EEE77A02F8403C0B92A2F1400350
:10F62000082267EE887AD91C5A701E2246F8201DDF
:10F630003046FDEEE77A9A70CDED027ABDF80810FB
:10F640000AF033F9B7F90030304607EE903AF8EE99
:10F65000E77A67EE887AFDEEE77ACDED027ABDF8BB
:10F6600008100AF022F9B7F90430304607EE903A54
:10F67000F8EEE77A67EE887AFDEEE77ACDED027A6A
:10F68000BDF808100AF011F9304618F05BFDFDF7DF
:10F69000CEBF00BF44810120BB340120A4E7030892
:10F6A0009CE70308B0E7030800000000E8800120A1
:10F6B00067666666E480012038A6012044E60308F8
:10F6C000849E012060E60308F4730120608001201D
:10F6D000C480012058A08B41078101209AF8024084
:10F6E000D4B1013C00235146E4B21A4601345444DB
:10F6F00011F8013B160A53408C4283EA0313DBB234
:10F700004FEAC30246EA032682EA131386EA03029B
:10F71000EED1002A7FF4E3ACBF4A0021BF4E12882D
:10F72000BF4BF261BF4C1A68DFF830939B68F262FE
:10F73000B4F84A21F066F364D9F80000F163F26589
:10F74000F8F752FD029000287DF4A5AE0221D9F809
:10F750000000FDF777FD94F84C3104229AF803106D
:10F76000642B049186F8742040F07C8194F84D312C
:10F77000072B00F0118294F84D31AB4A06EB031AC7
:10F7800006930292DAF804100846039128F084FBED
:10F79000DAF808105FFA80FA0846059128F07CFB39
:10F7A000069BC0B2039903F00F0E024623F00F0030
:10F7B0009D4B039252449872039883F80DE002F136
:10F7C000080E00EBCA00524683F807E0987303F175
:10F7D0000F0029F06BFB954B0AF109000599039A7C
:10F7E000184429F063FB9049CB7903F1010AF3B186
:10F7F00003F1FF3CC81D0023DFF864E25FFA8CFCD4
:10F800000CF1080C8C4410F8011B594084454FEA58
:10F8100081034FEAD10283EA410302F0180283EA2E
:10F8200001034EFA02F283EA0203DBB2EBD17F4A14
:10F8300004980AF8023027F0CBFE94F84D310022EC
:10F84000013384F84C2184F84D31029B9B786BB1D5
:10F85000DDF808A01AF805100135D9F80000FDF709
:10F8600005FD9AF80230EDB2AB42F3D894F84C3172
:10F870000322013386F874203A7084F84C31FFF784
:10F880007AB902213868FDF7DDFC94F82431FDF7E0
:10F89000C2BD0123664E0293FDF721BF326882EAA2
:10F8A000E273002AA3EBE27303EB5303A1FB0331E2
:10F8B0004FEAD101B8BF41F08041FFF724BB5D4959
:10F8C000881F16F061FA84F83E01FFF7F5B90026AB
:10F8D000102004230AA98DF828008DF829308DF80E
:10F8E0002A608DF82B608DF82C608DF82D6016F055
:10F8F000BBFB84F82F61FDF7B8BD342639E44E4BCD
:10F90000DB78002B0CBF04270527FEF7B2BE0123CE
:10F9100038683370FDF7A2FC06463868FDF79EFC98
:10F92000720602D080287DF449AD8A2856D08E28F0
:10F930007DF444AD94F81831002B7DF45BAD3F4A63
:10F940002D23C4F8202184F82431FDF73EBD324B2D
:10F950001888FFF796BB4FF47A71C8E54FF0010A9B
:10F96000334EFEF787B92C489179028802EB820268
:10F9700002EB82024FEA82091FFA89F9002900F09E
:10F980001881274A126803930FFA82FA13F0EEFAED
:10F99000039B40B2FDF76EBF03262949D4E5084614
:10F9A0008A4689468E460591FEF751B8254B264A70
:10F9B0001B68264903F4800383420ABF11460326CD
:10F9C0000426B5E52426FFF7D4BB04262049BBE571
:10F9D0001026FFF7CEBB2026FFF7CBBB1D4B1B68C5
:10F9E0009B067DF5EBAC94F81831002B7DF402AD4D
:10F9F000194A2D23C4F8202184F82431FDF7E5BCF1
:10FA00004B1C0906DBB2042B84F841313FF446ACB1
:10FA100047E40826FFF7ADBBF47301201000012076
:10FA20006080012054250120CCB80120D2B80120EB
:10FA3000E88001208C2601200C9E0120C481012039
:10FA400098E70308FC7D012048E6030844E6030824
:10FA500058E60308E0800120F08101202C88012075
:10FA60000007090E96F875C01CF00F0F03D10CF1BA
:10FA7000010C5FFA8CFCBCF1070F584B059528BFB1
:10FA80004FF0010C1A46029300234FEA0C1A02F1C0
:10FA90000D0E937206EB0A035FFA8AF2197C504B43
:10FAA00003920B4493F82420039B012A0EF10105D5
:10FAB00041EA030106EB0A038EF80010DB680CD95B
:10FAC000901E2A46C0B2811C714402F8013B8A4252
:10FAD0004FEA1323F9D101300544B2440CF1010C73
:10FAE00023F0600305F1010E9AF811205FFA8CFCF7
:10FAF0001343BCF1080F2B7042D003994FEA0C1A44
:10FB0000384B103106EB0A02AEEB0303C9B2039186
:10FB1000117C334A0A4492F8242098181328C3DD34
:10FB2000059DDBB20298DFF8C8E09A1DD2B242F020
:10FB3000400102F1010AC171D2B1053302990EF1FF
:10FB400001000022DBB20833CB18039310F8011B2D
:10FB500051408A00CB0882EA410203F018034A4070
:10FB6000214941FA03F35A40039B8342D2B2EDD1BB
:10FB700004980AF80E2086F875C027F029FD64E67F
:10FB8000184B059DAEEB0303CBE7184A894664206A
:10FB9000B2F900A0FDF76EBE9DF8083084F84D3133
:10FBA000E9E508468A4689468E4605910E46FDF7E8
:10FBB0004EBF4FF0FF32E6E60846FDF748BF084665
:10FBC0008A46FDF744BF08468A468946FDF73FBF8F
:10FBD00008468A4689468E46FDF739BFCCB80120D3
:10FBE00008B80308D9B801200007090E6080012079
:10FBF000D2B80120B0F908302DE9F04FDDB293B052
:10FC00000C460B81442D00F0C982064643D9812D54
:10FC100000F0FA8100F29A80542D00F0CD8040F27D
:10FC2000E2816E2D00F08882802D40F01681B94B64
:10FC300093F8009009F1020919F0FF0900F099808A
:10FC4000B54B0A25B54F994403F10108B44EDFF8CE
:10FC50000CA317E0322D00F0D682A5F13C00C0B213
:10FC6000132840F2D88200232268C14502F1010125
:10FC700021601570226802F101012160137078D0B3
:10FC800018F8015B0A2DE5D1BAF80030FF2BA8BFA8
:10FC9000FF23DBB2E8E7052D00F06E821FD8022DAE
:10FCA00000F0828040F28B81032D00F03482042D1D
:10FCB00040F0D3802A469B49204609F0D6FD00211A
:10FCC000204609F015FE216802200123CD181A46AE
:10FCD000256008701846628113B0BDE8F08F242DAE
:10FCE00060D040F2F480282D00F0D781382D40F00C
:10FCF000B4800A68012005270A26131800258A49BE
:10FD000023600346107020681A4600EB030EC4F807
:10FD100000E007702068C718276006702068C618C2
:10FD20002660057020680D78C6182660057020686A
:10FD30004D78C6182660057020688978C51825603A
:10FD400001701846628113B0BDE8F08FA02D17D066
:10FD500040F20681B82D00F0DC81FE2D7DD1734D7F
:10FD600005F1080635F8021B204609F0C1FDB54231
:10FD7000F8D101231A461846628113B0BDE8F08F0E
:10FD80006B4B0846196809F09DFD6A4B20461968BF
:10FD900009F098FD684B1968204609F093FD01238E
:10FDA0001A46E8E7654BF6E704226549204609F064
:10FDB0005CFD01231A46C4E70B681121614A204605
:10FDC0005D1C614F256007F148061970BD1E236850
:10FDD0001278591C21601A70236897F85B20591C0F
:10FDE00021601A70236897F85A20591C21601A70F4
:10FDF000B7F8561009F07CFD0021204609F078FD87
:10FE0000B7F85810204609F073FD35F8021F204658
:10FE100009F06EFDAE42F8D122680C214B4B501C0C
:10FE20005D1820601170226813F8011F501CAB424E
:10FE300020601170F7D1236802222046591C2160EE
:10FE40001A70B7F85C1009F053FDB7F85E10204641
:10FE500009F04EFD01231A4673E721462846FBF7B9
:10FE6000CBFB002885D1742D00F0C380772D0AD1FB
:10FE7000336872689A4240F09D810146344A2046B8
:10FE800023F008FF75E7762D00F09881392D37684B
:10FE900000F0968200F21A82212D01F0B482292D01
:10FEA00040F0CE827B1C33603B780A2B01F0DF826E
:10FEB000502B41F09281274D304609F0C6FC288036
:10FEC000304609F0C2FC012368801A4639E7202D2C
:10FED000C3D10B680846204D591C6A7821601A70FE
:10FEE00023682A78591C21601A702368AA78591C43
:10FEF00021601A70298909F0FBFC216801236879C7
:10FF0000CE181A46266008702168A879CD18256099
:10FF1000087016E7D8BB01205CB803086766666600
:10FF2000484E0120BB340120B13401202C73012044
:10FF3000107AF01F147AF01F187AF01F483601204B
:10FF400018E80308D0A30120F63301203F34012034
:10FF5000612F0308304E0120CC800120704E01201B
:10FF6000822D7FF47AAF0B680846B84A5E1CB84D04
:10FF70001178B84A26601970118909F0B9FCB64B9E
:10FF8000226820461B88511CFF2B2160A8BFFF233D
:10FF90001370A96881F3100189B209F0A9FC2968DE
:10FFA000204601F30F0189B209F0A2FC2168AB4A97
:10FFB00001231078CD181A4625600870C1E6012D7E
:10FFC0007FF44BAF096800262B4624204F1C2A469D
:10FFD00027600E7021684E1C26600D7021684D1C34
:10FFE00025600870ADE6522D7FF437AF2168002000
:10FFF0006BE6336872689A4240F0D8800146984AAE
:020000040801F1
:10000000204623F047FEB4E6964B1E78033616F0E2
:10001000FF063FF4AEAE944B4FF00A08934F1E44D8
:1000200003F1010920E0B8F1500F00F0F280B8F1BF
:10003000320F00F00581A8F13C00C0B2132840F255
:100040002D8100252946236820465A1C226083F80A
:10005000008009F04DFC2946204609F049FCB145D5
:100060003FF487AE19F8018BB8F10A0FDBD1804954
:100070008B684FF6FF72096803EB830391424FEAE6
:100080004305A8BF1146954221EAE171A8BF154674
:1000900089B225EAE575ADB2D5E70B6802210125E5
:1000A0000627581C0A22DFF8F081206020461970CC
:1000B0002368704E591921601F70236859192160F7
:1000C0001A7023685A1922601D70B8F8001009F0E0
:1000D0000FFCB8F80210204609F00AFC23685021F2
:1000E000002203EB050E2046C4F800E01F702368D1
:1000F0005F19276019702368591921601A703188B7
:1001000009F0F6FB7188204609F0F2FB2B462A46DF
:1001100017E6594B3FE60968012302260020CF1855
:100120001A4627600D702168CD1825600E70216871
:10013000CD182560087004E6474B08460A681B88FE
:10014000511C434DFF2B2160A8BFFF231370A968EA
:1001500081F3100189B209F0CBFB484B2046198886
:1001600009F0C6FB2968204601F30F0189B209F0A6
:10017000BFFB01231A46E4E50B224149204609F062
:1001800074FB08223F49204609F06FFB07223E49D5
:10019000204609F06AFB01231A46D2E5002A3FF403
:1001A000E8AD3A49012311601A46CAE55A1C32608B
:1001B000197824E75A1C326019785FE633685A1CB4
:1001C00032601B78002B01F03E81102B01F04A8138
:1001D0000546014622682046561C2660137009F029
:1001E00071FB2946204609F06DFB294B2046196812
:1001F00009F068FB2046002109F07AFB0021204627
:1002000009F076FBF2E63388FF2BA8BFFF23DBB2B1
:100210002AE520492CE715F0EDFB00283FF423AD3B
:1002200003780A2B50D8B0F9023087FB0312DB1792
:10023000C3EBA2039BB2FF2BA8BFFF23DBB213E5E6
:100240007B684FF6FF72396816E700BF0A74012019
:1002500060800120CC800120F4730120099E0120E0
:10026000413B0308D8BB01206CB80308404E012075
:10027000FC4D0120304E0120C42B0120069E0120A0
:1002800020E803082CE8030838E80308EDB5000867
:1002900018280120344E01207C2E012015F0AAFBE5
:1002A00000283FF4CEAE03780A2B3FF6CAAEB0F971
:1002B0000430B0F9061003EB830321EAE17183F304
:1002C000500589B2ADB2BEE60023B7E7552D00F068
:1002D0008780572D40F0B4807B1C0DF107023360FE
:1002E00017F8375B013333609F4213F8011C02F8A3
:1002F000011FF7D1DFF840A19AF80060002EFDD170
:100300000127DFF838B1102148488AF80070FAF761
:1003100053FADBF800000DF1080808F0CCFE444B5E
:10032000314642481F70FAF70BFB31463F48FAF757
:1003300007FB09213D484646FAF702FB0DF13E094D
:1003400029463A4D3948FAF7FBFAA6EB08070A2185
:100350002846FFB2FAF7F4FA28463946FAF7F0FAD7
:1003600016F8017B0B212846FAF7EAFA39462846A7
:10037000FAF7E6FA0020FCF7C3FFB145E5D12B48B8
:1003800008210546FAF7DCFAA0212846FAF7D8FA40
:10039000A0212846FAF7D4FA00212846FAF7D0FA25
:1003A00010F02006F4D1DBF8000008F08AFE0421EA
:1003B0001E48FAF701FA01238AF800601A46C0E4E1
:1003C0007B1C33603B780A2B01F05480304609F0E7
:1003D00047FA304609F044FA304609F041FAC8E4D9
:1003E0007B1C33603D78FF2D01F0B680FE2D01F0BF
:1003F0005280304609F029FA96E80C009B1A002B2F
:1004000041F32680531C33601378002B41F0208089
:100410000B2D01F21D80074A00304FF001031544F7
:1004200018BF01201A4685F84A008AE400380040C7
:10043000463A0120F63301203D3A0120C8A30120AD
:1004400072680B3DD31BEF2D00F2748201A151F8AD
:1004500025F000BFED100108350901083509010834
:100460003509010835090108350901083509010870
:100470003509010835090108350901083509010860
:100480003509010835090108350901083509010850
:100490003509010835090108350901083509010840
:1004A0003509010835090108350901083509010830
:1004B000350901089D100108350901084511010899
:1004C000350901082311010835090108350901081A
:1004D0003509010875100108350901081B100108CC
:1004E00035090108C3130108350901089D130108E6
:1004F00035090108F513010835090108B51201088D
:1005000035090108311301083509010835090108C9
:10051000350901083509010873FD0008350901088E
:10052000151301083509010835090108831301086D
:10053000350901089111010835090108350901083B
:10054000350901083509010835090108350901088F
:100550003509010835090108391201083509010872
:10056000EB11010835090108350901087912010864
:10057000350901083509010835090108350901085F
:100580003509010835090108350901084B0F010833
:1005900035090108D70E010835090108690E01085F
:1005A00035090108A10D010835090108790D010877
:1005B000450D01083509010835090108350901080B
:1005C000350901083509010835090108350901080F
:1005D00035090108350901083509010835090108FF
:1005E00035090108350901083509010835090108EF
:1005F00035090108350901083509010835090108DF
:1006000035090108350901083509010835090108CE
:1006100035090108350901083509010835090108BE
:1006200035090108350901083509010835090108AE
:10063000350901083509010835090108350901089E
:10064000350901083509010835090108350901088E
:10065000350901083509010835090108350901087E
:10066000350901083509010835090108350901086E
:10067000350901083509010835090108350901085E
:10068000350901083509010835090108350901084E
:10069000350901083509010835090108350901083E
:1006A000350901083509010835090108350901082E
:1006B000350901083509010835090108350901081E
:1006C000350901083509010835090108350901080E
:1006D00035090108350901083509010835090108FE
:1006E00035090108350901083509010835090108EE
:1006F00035090108350901083509010835090108DE
:1007000035090108190D010835090108630D0108B3
:1007100035090108350901083509010835090108BD
:1007200035090108350901083509010835090108AD
:10073000350901083509010835090108350901089D
:100740003509010835090108BD0C01086B0C0108C9
:100750002F0C010835090108930B0108790B0108DA
:100760000D0B010835090108F30A01088D0A01087B
:10077000650A0108530A0108F90901083509010849
:10078000CB0901083509010835090108A909010843
:10079000530901083F0901088109010817090108E7
:1007A000F5080108C3080108A9080108350901086E
:1007B000350901083509010835090108350901081D
:1007C000350901083509010835090108350901080D
:1007D00035090108350901083509010835090108FD
:1007E000350901088F080108350901083509010894
:1007F0002F080108350901083509010835090108E4
:1008000035090108350901083509010835090108CC
:1008100015080108C44B1B78DB0700F18B80FBF740
:100820008BFFFCF731F801231A46FFF78ABA7B1CCD
:1008300033603B780F2B7DD8BD1CC3EBC302BB4993
:10084000F81C356007F1040E7D788B188D547D1DE2
:100850003060B81DBA78F91D5A7007F10802C6F861
:1008600000E097F803E083F802E035603D79DD7041
:100870003060787918713160B97959713260FA79DC
:100880009A711CF0A1FC01231A46FFF75ABAA84D31
:10089000304608F0DAFFE881304608F0D6FF012341
:1008A000A8811A46FFF74DBA3046A24D08F0CDFF99
:1008B000012300EB80001A4600FA03F12980FFF7BC
:1008C00040BA3A467B1C9C49FD1C3360381D12F827
:1008D00002EB012381F800E032601A4697F801E04C
:1008E00081F801E03560BD788D703060F878C870AF
:1008F000FFF727BA914D304608F0A7FF288230460F
:1009000008F0A3FF6882304608F09FFF0123A88209
:100910001A46FFF716BA791C3B46FA1C316013F8E9
:10092000020B336079783260BA7817F0D7FF00286D
:100930007FF41FAA4FF0FF331A46FFF702BA804B2D
:100940004E228049186828F0B1FA01231A46FFF7B1
:10095000F8B93A46781C7C4BF91C3060304612F8E6
:10096000025B1D7032607A785A703160BA789A7082
:1009700008F06BFF754A0123D0801A46FFF7E1B9F2
:1009800039467B1C724AF81C3360012311F8025B64
:1009900015701A46316066497D788D703060654902
:1009A000B8788870FFF7CDB9684D304608F04DFF34
:1009B0002880304608F049FF6880304608F045FF3F
:1009C0000123A8801A46FFF7BCB9DFF8A48198F884
:1009D0000030002B3FF4CDA95E4F00253046013595
:1009E00008F033FF1DF02CF998F80030A7EC010A4D
:1009F0009D42F3DBFFF7BDB90D2B9BD17B1C336010
:100A00003D78072D96D80C27DFF86881304607FB24
:100A100005F708F01AFF08EB0705A880304608F034
:100A200014FFE880304608F010FF33682881304614
:100A30001A46591C316012F8021BA97232605B78A9
:100A4000EB7208F0EBFE012348F807001A46FFF7A7
:100A500078B9304608F0F9FE3F4A012310801A4663
:100A6000FFF76FB97B1C33603878060600F1978575
:100A70002D4B1B78DD073FF57CA9032828BF0020FC
:100A8000FBF740FE01231A46FFF75BB97B1C30469B
:100A9000336097F8009008F0C1FE8046304608F0B9
:100AA000BDFE0746304608F0B9FE0546304608F060
:100AB000CCFE304608F0C9FE304608F0D1FEB9F150
:100AC000000F00F08B85B9F1100F7FF452A9234B72
:100AD000C3F800805F600DB1214B1D6021490222E7
:100AE000214B081F1A7011F049FC01231A46FFF729
:100AF00028B90D4B1B78D8073FF53BA9FCF7B8F890
:100B0000FBF7C2FE01231A46FFF71BB9064B1B7801
:100B1000DA073FF52EA91548012301781A4641F05E
:100B200004010170FFF70DB9D0890120088B012065
:100B30008C2E01209C2E01208C3E0120309401201F
:100B4000C834012020DA0308842E012004910120FA
:100B5000EC7501205C900120C49F0120082B01202E
:100B6000182801200C2B0120AE9E0120E4800120DA
:100B7000D8BB0120148A0120AD4B1B78D9073FF563
:100B8000F8A8AC4A4FF4C871012311801A46FFF748
:100B9000D8B8092B7FF7CEAE3B467A1CDFF8C4826B
:100BA000F81C391DD8F80050326013F8022B2A7057
:100BB0007A1D33607B78AB703060B81DBB78642BD6
:100BC000A8BF64236B713160F91DFB78642BA8BF4B
:100BD0006423AB71326007F108023B79EB7130603E
:100BE00030467B79642BA8BF64232B723160BB79BC
:100BF000EB703260FB792B7108F027FE7268336866
:100C00006881D11A00290CDD581CD8F80010121A7E
:100C100030601878002A487203DD9A1C32605B78D5
:100C20004B701EF0A9FB01231A46FFF78AB8824ACF
:100C3000FB1C2137106802469D1E591E0332356089
:100C400013F8035C02F8035C316013F8021C02F82D
:100C5000021C3360033313F8041C9F4202F8011C8A
:100C6000EAD11CF09BFEFFF784B87B1C734A33600B
:100C70003B78002B00F03885137843F00203B91C51
:100C800013706F4D304631607B782B7508F0C6FDD0
:100C90002860304608F0C2FD6860304608F0D5FD97
:100CA00028813046674E08F0D0FD01233178E88175
:100CB0001A4641F002013170FFF743B8C3F347050C
:100CC000122D3FF637AEB5B112AB0DF1060903EBAD
:100CD0004507C846423F304608F0B7FD28F8020FE6
:100CE0004745F8D1584B39F8022FC84523F8022F51
:100CF000F9D1112D0AD86B00544A0020023B02F1B1
:100D00002201134423F8020F9942FBD101225049DA
:100D100013460A70FFF715B8791C3B46FA1C316080
:100D200013F8025B336078783260B978002D00F0F8
:100D30006A84012D7FF41DA822F0DCF82B462A4698
:100D4000FEF7FFBF3A4B1B7813F001017FF4F2ADC1
:100D50007B1C3360387822F07FF801231A46FEF7B7
:100D6000F0BF00233B4D30462B6008F057FD0123B8
:100D700028601A46FEF7E5BF39467B1C364AF81C48
:100D80003360012311F8025BD5701A463160334994
:100D90007D784D7130603249B878C870FEF7D1BFA8
:100DA0003046254D08F051FD304608F04EFD3046E6
:100DB00008F04BFD304608F053FD33682A68304692
:100DC00019465F1C3760DF1C11F802EB82F82CE03B
:100DD0003160597882F8361037609B7882F8373066
:100DE00008F03EFD304608F03BFD304608F038FD87
:100DF0002F68304608F029FD788730462F6808F0C4
:100E000024FD96E80A0038875A1A012A0ADD4A1C8E
:100E10002B68304632600A7883F82E2008F020FDD7
:100E200096E80A005B1A032B00F36384286818E72E
:100E3000D089012016920120C8340120E4800120CD
:100E4000E8800120AC9E01204286012044860120DA
:100E500068860120C42B01208C2E01202C840120C7
:100E60009C2E0120F89101207B1CBD4DDFF81C83D6
:100E700030463360D5F800903B7888F8053008F0AC
:100E8000E4FCA9F8200030462F6808F0DEFC96E864
:100E90000A00F8835A1A072A00F30E845A1A032A02
:100EA00000F3FC835B1A002B05DD4A1C2B683260C3
:100EB0000A7883F82620FBF749FC15F017FCA94BAC
:100EC0001B68002B00F0238428681CF003FA012320
:100ED0001A46FEF736BF3B467A1CDFF8B082F91C93
:100EE00032603A1D13F8025B304688F802503360D6
:100EF0009D4D7B782B7031609C4DBB782B7132609F
:100F0000FB78092BA8BF0923AB7008F09EFC96E87C
:100F10000A0028805A1A012A05DD304608F095FC9F
:100F200096E80A00E8818B4240F04483FBF70EFC10
:100F300096E80A008B423EF41CAF4A1C0123326043
:100F40001A460978E970FEF7FCBE304608F07DFCD1
:100F5000054611F01DFBFF283EF40BAF3F2D00F2BC
:100F600087834FEAD508002312AF0DF1070008F17F
:100F700001088DF8073007F8403D394611F0E8FACE
:100F80009DF807305FFA88F805F00705434505F13D
:100F9000010503D19DF80830AB4203D029464046F5
:100FA00011F0E2FA33687268D21A012A7EF7E1AED4
:100FB000591C002212A831601D7800F8412D11F053
:100FC000BBFA9DF80730AB420AD0694B1B683BB1B6
:100FD0009A79AA4204D31B681B690BB1284698472B
:100FE000336800223846591C31601D788DF808207E
:100FF00011F096FA9DF80830AB423EF4BAAE5C4B65
:101000001B68002B3EF4B5AE1B685B69002B3EF4F9
:10101000B0AE28469847FEF7ACBE7B1C554D304617
:1010200033603B782B7208F010FCA883304608F040
:101030000CFC2883304608F008FC336868835A1C8F
:1010400032601B78EB7473689A1A032A00F3F182FA
:1010500031685A1A052A00F3DC825B1A002B7EF7EE
:1010600088AE4A1C012332601A46097885F821109F
:10107000FEF767BE7B1C4048D21A33603B78002ADB
:1010800003707EF776AEBA1C012332601A46797877
:10109000003118BF01214170FEF753BE7B1C336045
:1010A0003D78132D3FF646ACBB1C3360787822F0B8
:1010B0002BFE00283FF43EAC0078FA1C2F4B391D64
:1010C00003F8250003EB850332607A1DBD782448C0
:1010D0005D703160F9780068997032603A79DA7041
:1010E0001EF0D8F801231A46FEF72BBE102B244A17
:1010F0004FF0000128BF1023116051609160D16052
:101100001174002B3EF435AE3168013A0B440131C5
:1011100031608B4211F8010C02F8010FF7D1FEF794
:1011200028BE184D304608F090FB2860304608F085
:101130008CFB6860304608F088FB0123A8601A46E3
:10114000FEF7FFBD104D002330462B6008F066FB14
:101150002A68012310431A462860FEF7F2BD00BF3B
:10116000C8340120142F0120802E0120309401204A
:1011700078400120707F0120182F01201C2F0120B2
:10118000682E0120A06E012048360120EC75012058
:101190007A1CDFF870830021C84B326030463A7801
:1011A000C8F800101A7008F039FB3268D8F800301F
:1011B000571CC3490343C34D3046C8F8003037605D
:1011C00013780B7208F041FB2860304608F03DFBB5
:1011D0006860304608F039FBA860304608F035FBFF
:1011E000304608F032FBFEF7C4BD7B1C336097F835
:1011F0000080B8F1110F3FF69DABBB1CB24D3046DD
:10120000336019267B7805F8183005EB480508F09F
:101210001CFB40F6CA0340F2EE229842A8BF1846D3
:1012200001239042B8BF10461A46A0F2EE2191FB6E
:10123000F6F16970FEF785BD3B467A1CA34D30463A
:10124000326013F8022B2A7133607B786B7108F0DF
:10125000FCFA3368288030465A1C32601B78AB7128
:1012600008F0F3FA316801236880C8181A46306024
:101270000978E971FEF765BD954B1B78012B3EF6A9
:1012800078ADF91C781C3B46924D521A306013F829
:10129000020B012AA870336097F801E03160B8783A
:1012A00040F39181304608F0D0FA012328801A4695
:1012B000FEF747BD7B1C336039780E293FF63AAB09
:1012C000BB1C3360787803283FF634AB0623824A90
:1012D000FD1C07F1040C03FB01F307F1050ED11807
:1012E00048713560BD1DB878D054F81DC6F800C0EF
:1012F0000123FA784A701A46C6F800E097F804E02D
:1013000081F802E035607D79CD703060B879087180
:10131000FEF717BD39467A1C70480123326011F878
:10132000025B1A468570316079784170FEF709BD1D
:101330000722B3FBF2F2C2EBC2055B1B7FF4FAAAF1
:10134000D2B202F1FF395FFA89F9002A3EF411ADF9
:1013500009F101091D46DFF888B17A1C604B4FF096
:101360000008326097F9001093F9022008338A428E
:1013700000F0CA8008F10108B8F1060FF4D1FFF7B8
:10138000D9BA584B07F1080201373760974217F86E
:10139000011C03F8011FF7D1FEF7EBBC7A1C326089
:1013A0003D781F2D3FF6C6AA052B7FF4C3AA304611
:1013B00008F034FA4C4B43F8250023F061FBFEF7AC
:1013C000D8BC494D05F140073046043508F03DFAD8
:1013D0003368A5F87C00591C1A46316012F8021BCC
:1013E00085F87E1032605B7885F87F30BD42EBD1A6
:1013F000FEF7BFBC7A1C32490123326038781A46A6
:101400004875FEF79EBC3B46791C384DFA1C31608E
:10141000304613F8021B697033607B782B703260A2
:10142000BB78AB7008F011FA316801232881CF181E
:1014300008461A46376010F8027B6F7130604978B1
:10144000A971FEF77EBC2A4A92E82200FEF7C2BECE
:10145000242D3FF66FAA274A012322F815001A46C9
:10146000FEF76FBC244A92E82200FEF7B3BE234D7C
:10147000FEF722BDBB1C2249FD1C381D3360012331
:101480007A780A701A463560BD784D703060F87809
:101490008870FEF756BCBB1C33607D78022D3FF68A
:1014A00049AA304608F0D1F912494FF0FF3301EB59
:1014B00045011A46A1F85C00FEF743BC182F012035
:1014C000707F0120A06E012098890120002D01204D
:1014D0001336012016360120D02B0120A82E012022
:1014E000DCA301206F7F012034820120CC80012009
:1014F000F09E0120F6330120082B01207C2E0120D4
:10150000B1340120483601200BEBC80A30460135C2
:101510008AF8021008F099F933682BF83800A945C9
:101520001A4603F1010003F1030103F104073060DF
:1015300012F8020B8AF8030032605A788AF8042005
:1015400031609A788AF806203760DB788AF80530AF
:101550007FF403AFFEF70DBCBB1C7249FA1C724D41
:1015600033603B1D97F801E0304681F800E03260BF
:10157000BA7885F85B203360FB7885F85A3008F03C
:1015800064F9A5F85600304608F05FF9304608F0D7
:101590005CF90123A5F858001A46FEF7D2BB00F00B
:1015A0007F00032828BF002021F0C2FC01231A4637
:1015B000FEF7C7BB4B1C33600B78003318BF012309
:1015C00088F80730B2E4594A012311881A4611FB02
:1015D0000EF191FBF0F12980FEF7B3BB544B1020C4
:1015E000C3F800805F601FF05BF9524A137843F044
:1015F00001031370002D3EF4BCAB4F4A012315606C
:101600001A46FEF79EBB1CF02FF801231A46FEF780
:1016100098BB4B1C304633600B78EB7208F0FEF839
:101620003368E8605A1C32601B782B7496E80A0015
:1016300013E5304608F009F9A884304608F005F9AA
:1016400096E80A00E8845A1A032A7FF702AD0B468F
:101650004A1C3046326013F8022BAA7733604B786D
:1016600085F8203008F0F1F896E80A006884F0E484
:1016700002AF384610F048FFBDF80830AB423FF4E7
:1016800091AC2E4B1B68002B3FF48CAC1B689B6904
:10169000002B3FF487AC2846984783E4304608F097
:1016A000D4F8A8F80E00304608F0CFF896E80A0003
:1016B000A8F81000FFF7F6BB304608F0C6F8A8F807
:1016C0000A00304608F0C1F82F68A8F80C00304630
:1016D00008F0BBF878842F68304608F0B6F896E832
:1016E0000A00B884FFF7DABB137803F0FD03FFF7B5
:1016F000C6BAD5F80080304608F0A7F82F68A8F8D9
:101700003200304608F0A1F8B886FFF78FBB0C49CD
:1017100001230C4E0C4D1A460C48316029600160C3
:10172000FEF70FBBD0A30120F6330120B8A401209F
:10173000F09E0120E480012018280120784001203B
:101740000D8C0108808B0120D48B0120D48F0120C7
:101750003F4B2DE9F04F2DED0A8B1B7895B0012BF7
:10176000089001F0D1853B4C94F80021002A41F00B
:101770005380072B384D01F0C285002304936B681A
:1017800035489847002800F063810022B5F8B880FA
:1017900085F85920B8F1000F40F0EE86AB6AE96A8F
:1017A000B5F94000B5F94220C01AB5F94430521AD3
:1017B000296BDFF8B0B05B1A686395F85A102748B8
:1017C000EB63AA630DF03EFFDBF800309E0040F1B2
:1017D000E98095ED0E7AD5ED0D7AB8EEC78A95EDD4
:1017E0000F7AD4F8A831F8EEE77AF8EEC78A1C4AE7
:1017F00094ED676A0133D4ED686A94ED697A77EE07
:10180000867A126838EE268A78EE878AC4F8A8317C
:101810009342C4ED677A84ED688AC4ED698A01F069
:1018200049830B4B93F80080B8F1140F02F0E78660
:101830000023D4F8B0610593062E00F2A680DFE8FD
:1018400016F080155F16F613751613000F15691440
:10185000287301201C280120007601203476012005
:10186000802F0120FC7D0120D14B1A78D4F8B4E1FF
:10187000D04F4FEACE009FEDD07A3B1883ED007A2F
:10188000002A77D0B0EE476ACC49F0EE476A0023D1
:101890000133F1EC017A05EE903A67EEA77A9A42AD
:1018A000F8EEE55A87FE277A76EEA76AA7EEA56AD4
:1018B000EED1F5EEC06A3B1883ED007AF1EE10FA36
:1018C00058DDC6EE265ABE4ABE4BD2ED007A1A88C3
:1018D000B7EE007A75EEC75A65EEA77AFDEEE77AA5
:1018E00017EE903A812B43F380859342A8BF1346AD
:1018F00007EE903AF8EEE77A00EB0E01B24B03EBFD
:10190000810393ED007A93ED056A93ED015AA7EEFA
:10191000276AD3ED066A93ED047AE5EE276AD3EDE4
:10192000034A93ED025A27EE467ABDEEC64AE6EE2A
:10193000646AA5EE277A14EE101A8129C3ED056AB0
:1019400083ED067A43F34E858A42A8BF0A4607EE26
:10195000902AF8EEE77AFCEEE77ACDED067ABDF84C
:1019600018303A189380BEF1000F03D1B8F1130F6D
:1019700004F07D81B8F1150F42F0B2833844D4F8F9
:10198000B061924F838827F81E300136904A82FB5F
:101990000632F3173244C3EBA203C3EBC303F61AB8
:1019A000C4F8B0618B4B1B78002B01F044808A4E49
:1019B0000027DFF8749206F2DC68DFF810A2874B8C
:1019C0001B78172B01F00D8396ED007A082BD5EDCF
:1019D000097AB8EEC78A28EE278A07D1B0EE480AFE
:1019E000059327F027FC059B2AF81700DBF8002059
:1019F00090000BD5002F04F0EA85B0EE480AD5F828
:101A00007C3708F170009847B0EE408AB0EE480A83
:101A1000D5F89C36A8F170009847D5F80C374046A9
:101A200098476E4BB0EE408A1B78032B01F0D382AF
:101A30000137D6F85C06B0EE480AD5F8BC309847B6
:101A4000032F08F1240806F10406A9EC010AB6D117
:101A5000624B93F80090B9F1070F00F04B8694F8B1
:101A6000C031002B40F051865D4B5B79002B40F07C
:101A70007D850123594A84F8C0311278072A01F084
:101A8000E68700230B93574BF7EE007ADFF89C8133
:101A9000002693ED007A544B3546D4ED729AD3F874
:101AA00000A008F1680377EEE98A504F0A93504B83
:101AB00068EE878ADFF8789104934E4BD4ED71BAC3
:101AC000C8FEE78A05934C4BDFF868B107934B4B90
:101AD0009FED4B9A0993DFED4BAA4B4B9FED36BA26
:101AE0009FED4AAA06934A4B98ED008A3344D3ED02
:101AF000007AF5EE407AF1EE10FA17D0454B3344F8
:101B0000D3ED006A38EE667AB0EEC76AF4EEC67AB4
:101B1000F1EE10FA08D5B5EEC07AF1EE10FACCBFAE
:101B200037EEA68A36EEE78A83ED008A059B1A888F
:101B3000910700F08180022D7ED037489AF82E1050
:101B400030F915000A9B07EE901A07EE100A68009C
:101B50003344B8EEE76AB8EEC77AD3ED006A4B4279
:101B6000A6EE267A07EE903AF8EEE77AB4EEE77A38
:101B7000F1EE10FA05D407EE901AF8EE677AC7FE78
:101B8000C77A264BD20726490344085EB3F90C30C6
:101B9000A0EB030007EE100AB8EEC77AE7EE497A29
:101BA00040F1BB851F4B93ED008A27EE888A43E006
:101BB000862F0120A4310120000000001C280120F4
:101BC000882F0120842F0120BC3101202C7301209B
:101BD00093244992792F0120347601202873012023
:101BE000EC75012028900120C8340120B82E012076
:101BF000AC2E0120849E012088000120D089012084
:101C0000CDCCCC3DAE47813FEC7D01200000C842E9
:101C10001C900120E8290120AC2901208C2E0120F4
:101C2000C480012004900120F07D012020290120A2
:101C3000C42E01207C8B0120069B94F8D8213344CC
:101C4000D3ED01CA38EE6CCA002A3BD0D4F8DC21AF
:101C5000CF4B08991B688A1A9A4233DD9AF84830AC
:101C6000022B01F05387022D04F02884C94B1B6816
:101C70009B0740F1C786C84BC84903EB4500DFF816
:101C800090C331F915E0B0F90C009CED008AA0EB8F
:101C90000E0EC34828EE098A87ED00BA07EE90EAD7
:101CA0000068F8EEE77A904227EE888A38EE6CCA30
:101CB000C1F2B780F7EE007AF4EEE79AF1EE10FA8F
:101CC00001F18680B74B022D334493ED000A049B4B
:101CD0002BEE800A20EE0C0AA3EC010A049304F018
:101CE000AF83079ADBED006AD2ED007AAE4B66EE69
:101CF000A77A97ED006A334467EEA87A93ED007AED
:101D0000AA4B67EE877AD3ED005AB0EE467AF1EE31
:101D1000656AA7EE8C7AB4EEE67AF1EE10FA01D499
:101D2000C5FEC76AF7EE007A94ED727AB4EEE77AF0
:101D3000F1EE10FAACBF0123002343B1B0EEC66A46
:101D4000F0EEE67AF4EEC67AF1EE10FA01D5C7EDC0
:101D5000006A022D58D0964AB0EE6C0A954B52F8A4
:101D600025001B689847944A944B52F825001B683D
:101D700098479AF8373023B1059B1B88002B00F059
:101D80001D85B0EE4B8A8E4B38EE400A9BED007AF3
:101D9000334493ED008A83ED000A30EE480A9AF846
:101DA0004830C0EE077A2BB3099B1B78D90721D5A1
:101DB000B7EE007AF4EEC79AF1EE10FA04DB94F86D
:101DC000D831002B00F0EE86D4F8DC31089AD31A13
:101DD0006F4A12689A420DDD7A4BB0EECCCA93ED91
:101DE000007AB4EEC7CAF1EE10FA41F13680002352
:101DF00084F8D831744B334493ED007A2BEE877A14
:101E000067EE277AC9ED007A94F8E83133B9049B7C
:101E100087ED00BA03ED01BA89ED00BA013508F18A
:101E20000408043709F10409032D06F104067FF4C0
:101E30005AAE664B1B78072B01F08982012B01F00B
:101E4000F6854FF0000B94F8F031002B40F0A5859B
:101E50005F4A604B11681B6893F82C2011F4805383
:101E6000049300F01186099B1B78DB0703D45A4BBF
:101E70001B8BA4F8FC31594B59481B8890ED037A11
:101E800007EE903AF8EEE77AB4EEE77AF1EE10FA60
:101E900041F28A865348008807EE900AF8EEE77A06
:101EA000B4EEE77AF1EE10FAC1F2088677EE677ABF
:101EB0004D4BBCEEC77A4D48D3ED006A17EE103A91
:101EC00090ED007A0120C4ED806A37EE666AA4F8CE
:101ED000FC31474BC4ED7E6A84ED817A84ED7D6AE6
:101EE00084F8080293ED007A424BC7EE875ADFED83
:101EF000424A93ED006A414BD3ED007AB7EE005AA7
:101F00003F4B36EE276ADFED3F7A93ED004A3E4BBA
:101F100036EE046A93ED007A26EE246AF1EE476A03
:101F2000C5FEC55AC5FEA75AB4EEE66AC4ED835A8B
:101F3000F1EE10FA01F1488086FE476A2D4BD3ED91
:101F4000017A2E4B93ED015A2D4B77EE857A9FED5A
:101F50002A5AD3ED014A77EEA47A67EE857AF4EE39
:101F6000E76AF1EE10FA01DCC7FE676A214B9FEDCC
:101F7000225AD3ED027A214B93ED027A234B77EE6E
:101F8000877A93ED007A67EE857AF1EE473A41E081
:101F900030900120E08001208C2E0120C48001209F
:101FA0002C900120D88F0120E48F01204C9001203B
:101FB000848B0120808B0120D88B0120D48B0120C1
:101FC000FC2901203C900120F08F01202873012082
:101FD000FC7D0120C8340120707F01201091012078
:101FE0000C74012012910120FC9001205C2E012034
:101FF00018910120AC2E01206F12833AB82E0120D7
:10200000C42E0120000000005090012054900120B7
:1020100004900120F4EEE37AF1EE10FA01D4C7FE49
:10202000C73AE64B5B780BB9F1EE633A002A41F010
:10203000D682B7EE004AE24D2A78002A02F0508696
:10204000E04B9FEDE17A93ED025AD3ED014A26EE83
:10205000855AD3ED037AA6EE245AA3EEA75A24EEAE
:10206000055AB4EEC75AC5FE474A8DED0C5AC5FE57
:10207000077AF1EE10FA88BFF0EE474A012A02F023
:10208000508693ED067AD3ED052A26EE877A93EDF6
:10209000073AA6EE227AA3EE837A24EE077AB4EE0C
:1020A000E77A8DED0D7AC7FE277A87FE647AF1EE26
:1020B00010FA88BFB0EE647A022A00F0AD80D3ED4A
:1020C0000A4AD3ED092A66EEA44A93ED0B3AE6EEEE
:1020D000224AE3EE834A64EE244AF4EEE74ACDED69
:1020E0000E4AC4FEA77AC4FEC74AF1EE10FA98BFA2
:1020F000B0EE647A032A00F08F80D3ED0E4AD3ED60
:102100000D2A66EEA44A93ED0F3AE6EE224AE3EE7C
:10211000834A64EE244AF4EEE74ACDED0F4AC4FE4A
:10212000A77AC4FEC74AF1EE10FA98BFB0EE647AFF
:10213000042A71D0D3ED124AD3ED112A66EEA44AD7
:1021400093ED133AE6EE224AE3EE834A64EE244A24
:10215000F4EEE74ACDED104AC4FEA77AC4FEC74AA2
:10216000F1EE10FA98BFB0EE647A052A54D0D3EDA0
:10217000164AD3ED152A66EEA44A93ED173AE6EE19
:10218000224AE3EE834A64EE244AF4EEE74ACDEDB8
:10219000114AC4FEA77AC4FEC74AF1EE10FA98BFEE
:1021A000B0EE647A062A37D0D3ED1A4AD3ED192A55
:1021B00066EEA44A93ED1B3AE6EE224AE3EE834A2A
:1021C00064EE244AF4EEE74ACDED124AC4FEA77A43
:1021D000C4FEC74AF1EE10FA98BFB0EE647A072A3F
:1021E0001AD0D3ED1E4A93ED1D3A66EEA46AD3EDE4
:1021F0001F4AE6EE036AE4EEA36A66EE846AF4EE32
:10220000E76ACDED136AC6FEA77AC6FEC76AF1EE8D
:1022100010FA98BFB0EE667A77EEC77AF7EE006AEA
:10222000C4ED727AF4EEE67AF1EE10FA43F3078524
:1022300086EEA77ADDED0D7A022A27EE055A67EEC3
:10224000877A8DED0C5ACDED0D7A2DD0DDED0E7A1D
:10225000032A67EE877ACDED0E7A25D0DDED0F7A71
:10226000042A67EE877ACDED0F7A1DD0DDED107A66
:10227000052A67EE877ACDED107A15D0DDED117A5B
:10228000062A67EE877ACDED117A0DD0DDED127A50
:10229000072A67EE877ACDED127A05D0DDED137A45
:1022A00027EE877A8DED137A484B1B6813F0805820
:1022B00001F04080F6EE005AC4ED835A002A02F085
:1022C0000685D4ED817A01F01006414B01F48001BE
:1022D000FDEEE77AD4ED804ADF7894F90832099868
:1022E00006EE903A17EE903AFDEEE47A0078DFF8C9
:1022F000E8A0F8EEE66ADFF8E49000F00100DFF80D
:10230000E0C0DFF8E0E0059117EE901A9AF800A01F
:10231000D9ED007ABCF906C0BEF81AE094ED7D6AEA
:1023200094ED7E7A002F41F09181002E41F04C8097
:10233000244F9DED0C5AD7ED007A264E65EEA77A14
:10234000E6EE857AB0EE475AA6EE275AFDEEC57A3C
:1023500017EE90CA17EE90EA9C45A8BF9E466145CD
:10236000C8BF8E46012A07EE90EAF8EEE77AC6ED7E
:10237000007A00F0F480D7ED047A9DED0D5A65EEF9
:10238000A77AE6EE857AB0EE475AA6EE275AFDEE1A
:10239000C57A17EE90CA17EE90EA9C45A8BF9E46F4
:1023A0006145C8BF8E46022A07EE90EAF8EEE77A4A
:1023B000C6ED017A00F0D38016E000BF182F01208F
:1023C000D8BB01207C9001200000000038A601202D
:1023D0000C9E0120F02E01205494012058900120E1
:1023E0005C9E0120707F0120D7ED087A9DED0E5A8A
:1023F00065EEA77AE6EE857AB0EE475AA6EE275A42
:10240000FDEEC57A17EE90CA17EE90EA9C45A8BF7C
:102410009E466145C8BF8E46032A07EE90EAF8EE55
:10242000E77AC6ED027A00F09A80D7ED0C7A9DED3E
:102430000F5A65EEA77AE5EE267AB0EE475AA7EE78
:10244000865AFDEEC57A17EE90CA17EE90EA9C45C3
:10245000A8BF9E466145C8BF8E46042A07EE90EA93
:10246000F8EEE77AC6ED037A79D0D7ED107A9DEDD4
:10247000105A65EEA77AE5EE267AB0EE475AA7EE37
:10248000865AFDEEC57A17EE90CA17EE90EA9C4583
:10249000A8BF9E466145C8BF8E46052A07EE90EA52
:1024A000F8EEE77AC6ED047A59D0D7ED147A9DEDAF
:1024B000115A65EEA77AE5EE267AB0EE475AA7EEF6
:1024C000865AFDEEC57A17EE90CA17EE90EA9C4543
:1024D000A8BF9E466145C8BF8E46062A07EE90EA11
:1024E000F8EEE77AC6ED057A39D0D7ED187A9DED8A
:1024F000125A65EEA77AE5EE267AB0EE475AA7EEB5
:10250000865AFDEEC57A17EE90CA17EE90EA9C4502
:10251000A8BF9E466145C8BF8E46072A07EE90EACF
:10252000F8EEE77AC6ED067A19D0D7ED1C7A9DED64
:10253000135A65EEA75AE6EE855AA6EE257AFDEE09
:10254000C77A17EE907ABB42A8BF3B46B942C8BFD4
:102550000B4607EE903AF8EEE77AC6ED077A0028C8
:1025600040F02882002A40F0208223E29E4B1B7814
:10257000013BDBB2FFF77EBA9C4B4FF47A769C4965
:1025800006931B689B4F91F801A09B49B7F9060081
:1025900091F80090B6FBF3F3C3EB431603EB86030D
:1025A000DE00B6B2B04502F01181D5F88C10B5F955
:1025B00040E02B6F4A1C07EE90EA7344012AF8EEC4
:1025C000E77AC5F88C202B6702F00B8195ED1F5A36
:1025D00007EE102AD5ED216AB8F1010F77EEC55A42
:1025E000B8EEC76A85EE867A37EE057A77EEC77A57
:1025F00085ED207A85ED1F7AE7EEA56AF0EE667A22
:10260000C5ED226AC5ED216A02F0D284D5F8A0108A
:10261000B5F942E06B6F4A1C07EE90EA7344012A59
:10262000B8EEE77AC5F8A0206B6702F0F48095ED6C
:10263000245A07EE902AD5ED266AB8F1010F77EEFD
:10264000455AB8EEE76AC5EE867A77EE857A37EEB8
:10265000677AC5ED257AC5ED247AF0EE667AE7EE65
:10266000257AC5ED277AC5ED267A02F0D584D5F80E
:10267000B410B5F944E0AB6F4A1C07EE90EA73441E
:10268000012AB8EEE77AC5F8B420AB6702F0DD8026
:1026900095ED295A07EE902AD5ED2B6AB8F1010F76
:1026A00077EE455AB8EEE76AC5EE867A77EE857A18
:1026B00037EE677AC5ED2A7AC5ED297AF0EE667AAB
:1026C000E5EE877AC5ED2C7AC5ED2B7A02F0988479
:1026D000F880B5F8B830484A013B92F80090A5F868
:1026E000B83000230699B9F1070F4B608B60CB60BF
:1026F0007FF4B5A9FAF7F2FB049B3E4FC01A94F899
:10270000C0313880002B3FF4AFA9013B84F8C031C1
:1027100015B0BDEC0A8BBDE8F08FB1F90020B1F91E
:10272000021082EAE27394ED5E7AD4ED5F6AA3EB65
:10273000E27381EAE17286FE876AA2EBE1722F49B9
:102740009342B8BF13460A7807EE103AB8EEC77A3C
:1027500027EE097A002A00F0BA81294BD3ED005AFE
:10276000F5EEC05AF1EE10FA40F3E085254B93EDFB
:10277000005AB5EEC05AF1EE10FA40F3D78526EEB6
:102780004A6A35EE477AF7EE004AC6EE256A87EECA
:10279000056A76EEA46A86FE646A86FE0B6A66EEB9
:1027A000266AC6FEE46AC6FE8B6A174B93ED007A72
:1027B00067EE877AA7EEA68AFFF73EBA134BF7EECD
:1027C000006A134A3344D2ED007A93ED007A114B3C
:1027D00067EE277A93ED007AC7FEE67A67EE877A8E
:1027E00027EE888AFFF7CFBA802E0120EC7D0120EA
:1027F000EC7501202C73012028730120109001201A
:102800000C900120149001200890012094290120AF
:1028100000900120FC8F0120072B02F07D824FF0F9
:102820000008DFF870B3C14DDBF80030590501F145
:10283000F480DFF864A3DAF800301A0701F192801F
:10284000BB4A1278002A40F0D881DFF8289394F828
:10285000126126B1B74A1288970742F0F78194F8BF
:102860001821002A41F00D8099F81E60002E00F01A
:10287000D183022E02F04580032E01F0B682AE49CC
:10288000488899F81F100231C9B2002802F031803F
:10289000002A02F02E80A94E3668B0FBF6F006B290
:1028A000A4F84861B1B307EE906AF7EE005AA44865
:1028B0000129B8EEE76AD4ED576AD0ED007A85EECB
:1028C000867A77EEE67A67EE877AC4ED537A21D07E
:1028D000D0ED017A0229D4ED586A77EEE67A67EEF8
:1028E000877AC4ED547A15D0D0ED027A0329D4ED5D
:1028F000596A77EEE67A67EE877AC4ED557A09D0A1
:10290000D0ED037AD4ED5A6A77EEE67A67EE877AED
:10291000C4ED567A8B480078092803F03482002EE3
:1029200040F37A83002902F05A8594ED577A012901
:10293000D4ED537A824877EE877AC4ED577AC0EDAA
:10294000007A21D094ED587A0229D4ED547A77EEAA
:10295000877AC4ED587AC0ED017A15D094ED597A92
:102960000329D4ED557A77EE877AC4ED597AC0ED14
:10297000027A09D0D4ED5A7A94ED567A77EE877AB6
:10298000C4ED5A7AC0ED037A01390229B8BF022199
:10299000C9B2002A18BF022143E3099B6A4D1B7884
:1029A000DA0700F148812A7822B192006749684825
:1029B00026F07CFA674B1B68002B40F00983664BBE
:1029C0001B7893B1287868B1614F0026DFF8CC817D
:1029D000F0B2D8F80030B7EC010A013698472878F1
:1029E0008642F5DB5D4B1B689847564B1B78072BDF
:1029F00000F0A584012384F8003115B0BDEC0A8BEA
:102A0000BDE8F08F564B87ED00BA1B689342BFF6C6
:102A100051A9544A0023128884F8D831002A41F081
:102A2000AA86514A514B1178186881F0010106F0CD
:102A30004DFBFFF747B94E4FDFF8649107F24C7634
:102A400007F5F768F7EC017A304695ED090AF8EEDC
:102A5000E77AD5F87C3727EE800A9847A6F1E000A0
:102A6000D5F89C369847A6F17000D5F80C37243677
:102A70009847D7F85806D5F8BC309847B045A9EC28
:102A8000010ADFD1FEF7E4BF3A480123408B84F806
:102A9000083207EE900A2A4B3748B8EEE77AD3EDB2
:102AA000037A364BD0ED006A93ED006A77EEC77A71
:102AB000334B76EE665AC4ED806A93ED007AC4ED2E
:102AC0007E6AC4ED7D5A84ED816AFFF70DBA2D4B05
:102AD000D3ED005AF4EEEA5AF1EE10FA40F1CC864A
:102AE000B7EE005ADFED286ADFED284A36EEC77AE6
:102AF000274B35EE655AD3ED006A25EE245AE7EEF2
:102B0000055A65EEA65AF5EEC05AF1EE10FA40F2FB
:102B10000D84CAEE256AB7EE007AF0EE475AE6EE6B
:102B2000665AC5FEC76AC6FE8B6A3EE6007601207D
:102B3000DF220120849E012034860120142F0120F1
:102B40000C74012028730120D8BB01205C90012067
:102B5000F02E0120788B01205C9C012050940120F4
:102B60002C9001204C9301204E9301205093012082
:102B700034760120707F0120D4A401205C2E012036
:102B80000C9101201890012000003443610BB63BEA
:102B90000C900120FC7D0120E08001204894012060
:102BA000F07D0120B44AB0EEE77AD2ED006AB4EECF
:102BB000E67AF1EE10FA7FF707A9B04AB0EECC7AC8
:102BC000D2ED006AB4EEE67AF1EE10FA7FF7FCA8D7
:102BD00098ED007AAA4AB0EEC77AD2ED006AB4EE58
:102BE000E67AF1EE10FA7FF5EFA80122089984F851
:102BF000D821C4F8DC11FFF7EBB8A24ADFF8B09295
:102C0000B2F90610B9F81A2091423FF720AE9E4A59
:102C10001278192A02F09780012A02F09480082A7B
:102C20003FF415AE0E2A3FF412AE00229748C4F8C6
:102C30000C2182600BE62B78002B3FF4BBAED4ED69
:102C40005F3AF3EE046A94ED5E4AD4ED7E7AF4EED8
:102C5000C43A8F4A77EEA64A94ED7D7A92ED005AF7
:102C6000F1EE10FAD4ED5C5A94ED5B6A894F8A4E0E
:102C700001F10C8097ED026AB0EE674A26EE656AB4
:102C8000A6EE074AB4EEE44A34EE666AF1EE10FAB4
:102C900048BFB0EE456A012B86ED006A3FF48AAE6C
:102CA00097ED066AB0EE674A26EE656AA6EE074A19
:102CB000F4EEC44A34EE666AF1EE10FA88BFB0EE64
:102CC000456A022B86ED016A3FF474AE97ED0A6AFD
:102CD000B0EE674A26EE656AA6EE074AB4EEE44A0D
:102CE00034EE666AF1EE10FA48BFB0EE456A032B87
:102CF00086ED026A3FF45EAE97ED0E6AB0EE674A6B
:102D000026EE656AA6EE074AF4EEC44A34EE666A19
:102D1000F1EE10FAC8BFB0EE456A042B86ED036AE7
:102D20003FF448AE97ED126AB0EE674A26EE656A48
:102D3000A6EE074AF4EEC44A34EE666AF1EE10FAE3
:102D4000C8BFB0EE456A052B86ED046A3FF432AE8B
:102D500097ED166AB0EE674A26EE656AA6EE074A58
:102D6000B4EEE44A74EE666AF1EE10FAB8BFF0EE23
:102D7000456A062BC6ED056A3FF41CAED7ED1A6A0C
:102D8000B0EE674AB3EE046A66EEE56AA6EE874ADD
:102D9000F4EEC44A74EE466AF1EE10FAC8BFF0EEE3
:102DA000456A072BC6ED066A3FF404AED7ED1E6AEE
:102DB00066EEE55AE5EE877AF4EEE74A77EEC67AF4
:102DC000F1EE10FAC8BFF0EE457AC6ED077AF1E5EC
:102DD000069A324BD2ED017A93ED007AF0EEE77A63
:102DE000F4EEC77AF1EE10FA7EF56CAFD2ED027A0E
:102DF000F0EEE77AB4EEE77AF1EE10FA7EF762AF22
:102E0000D2ED037AF0EEE77AB4EEE77AF1EE10FA5B
:102E10007EF758AF224B1B6898077FF5FAAD214922
:102E2000214BB3F90C20B1F900E02048AEEB020EC3
:102E300000688EEAEE72A2EBEE728242BEF642AFFC
:102E4000B3F90E30B1F90220D21A82EAE273A3EB91
:102E5000E27398427EF736AFDBE598ED007A084BD7
:102E6000B0EEC77AD3ED006AB4EEE67AF1EE10FA6E
:102E70007EF7C0AFFEF7BBBF409001203C90012021
:102E8000449001205C9E0120182F01200C74012029
:102E9000589001207C900120F02E012038900120D4
:102EA000E0800120C48001208C2E0120349001207C
:102EB000707F012007EE103A524BF7EE006A524F36
:102EC0001B78B8EEC77AC4F8A881132BB7F90400B1
:102ED00086EE879AB4F8AC6195ED090A01F0D483C7
:102EE0004A4B4B4AD3ED006A67EE897A93ED053A77
:102EF00029EE088A93ED097A69EE288AD3ED0E3A15
:102F0000A6EEA73A93ED174AD3ED126AE7EE083A18
:102F1000D3ED064A02EB860193ED017AA6EEA84AAC
:102F200093ED0A6A8E46D3ED0F5AE7EE274AD3EDAA
:102F3000186A93ED137AE6EE085A93ED045AE7EE19
:102F4000286A93ED0D6A93ED167A25EE435A93EDB8
:102F5000032A26EE636AD3ED022A27EE447AD3EDE4
:102F60000C1AE2EE434AA2EEA75A93ED0B2AD3EDD8
:102F7000152AE1EEE35AD3ED147AA2EE086AE2EEE6
:102F8000C46A81ED003AA7EEA87A0021C3ED054A94
:102F900083ED065AC3ED0E5ACEED203A83ED0F6A4B
:102FA0008EED404AC3ED176A83ED187AC4F89C1180
:102FB000C4F8A011C4F8A411731CB88003F01F0357
:102FC000A4F8AC31FEF72DBCB0EE666AFEF7B6BFD2
:102FD00019F05CFDF3E426F02DF92AF81700FEF74E
:102FE00027BD96ED007A05EB4702D5ED097AB8EEDC
:102FF000C78AB2F840202AF8172028EE278AFEF761
:10300000F5BC00BF287301202C7301202832012059
:10301000A42F0120A4F84861002A00F05181022168
:10302000D448D54BB0EE007AD44A1B6892F800E041
:103030001A78DFEDD36A07EE902A9A78F8EEE77AED
:1030400067EEA67AF4EEC77AF1EE10FA40F3EE825C
:1030500037EEC77ADFEDCB6AB0EE676AA7EE266A75
:10306000F0EE466A9FEDC86A90ED007A27EE067A88
:10307000B0EEC76A84ED5B7A84ED5E6A9AB105EEC4
:10308000902A9FEDBF4A67EE074AB8EEE55AF7EE81
:10309000005A64EE864A25EE045A75EEC55AE4EEEF
:1030A000855A27EE257ADFEDB95A5F7966EEA56A73
:1030B00026EE877ACFB19FEDB25A06EE907ADFED19
:1030C000B45AF8EEE66A26EE056A26EE266AB4EEF3
:1030D000E56AF1EE10FA00F39C85F7EE005A35EE42
:1030E000C66AC5EE866A27EE267ABEF10C0F00F09E
:1030F0001E859FEDA88ADFEDA86A87FE488A88FEB4
:10310000268A84ED418A002900F0CC80B0EE007A56
:10311000F4EEC77AF1EE10FA05DD37EEC77ADFED8F
:10312000996AE7EE267A90ED017ADFED976A27EE4D
:10313000267AB0EEC76A84ED5C7A84ED5F6A9AB154
:1031400006EE902ADFED8E4A27EE075AF8EEE66A81
:10315000F7EE005A25EE065A66EEA46A75EEE65AB8
:10316000E5EE265A27EE257ADFED886A9A7967EE32
:10317000A67A67EE877AAAB107EE102ADFED805AA9
:10318000F8EEC76A9FED827A66EE866A66EEA56AF9
:10319000F4EEC76AF1EE10FA40F32D859FED7F7AC9
:1031A00067EE877ABEF10C0F00F0DF84DFED796AFD
:1031B00001299FED797AC7FEE67AC7FE877AC4EDCA
:1031C000427A6FDD5A78B0EE007ADFED6D6A07EE75
:1031D000902A5A7AF8EEE77A67EEA67AF4EEC77A82
:1031E000F1EE10FA05DD37EEC77ADFED666AE7EE3D
:1031F000267A90ED027ADFED646A27EE267AF0EE09
:10320000C75A84ED5D7AC4ED605A9AB106EE902AF1
:10321000DFED5B4A27EE075AB8EEE66AF7EE006A82
:1032200025EE255A26EE246A76EEC66AE6EE056A93
:1032300027EE267ADFED556ADB7967EEA67A67EE30
:10324000877A0BB307EE103A9FED4D6AF8EEC76A26
:103250009FED4F7A66EEA56A66EE866AF4EEC76A5F
:10326000F1EE10FA0CDCF5EEC06AF1EE10FA01F1A5
:103270003683B7EE006A76EE666A86EE267A01E05D
:103280009FED467A67EE877ABEF10C0F00F06584F9
:10329000DFED406A9FED407AC7FEE67AC7FE877A87
:1032A000C4ED437ABEF1090F00F0278499F821603C
:1032B000002E40F0D1830022DAF8003084F8182183
:1032C000980609D5364B1B8803F0300323B1354BE4
:1032D0001B78D90702F10E80334B1B7823B9334E8C
:1032E000B378002B41F01483244B1B78072B00F09C
:1032F00051840022072B84F800217EF43EAAF9F7BE
:10330000EDFD0490FEF73BBA294A2A4B12682A4C7D
:103310002A4FD2691B8894F800013A807B800028EC
:103320007FF47DAA0490264DFEF729BADFED256AC9
:10333000FFF73BBA4F023EF5BDAFFEF7BFBFF9F74F
:10334000CDFD1E4BA0EB0B00D880FFF753BBF9F768
:10335000C5FD0B9B194FC01A084B1B787880012BB9
:1033600000F06683072B7EF46CADF9F7B7FD83465A
:10337000FEF769BD0C740120F8910120287301202B
:103380000AD7233CD7A368416F12033B0000484390
:10339000A4707D3F00C0F94400C0F9C40000C842D9
:1033A000849E0120E48001203C3A01201636012051
:1033B00050840120FE2C01201C2801202C730120A8
:1033C0000076012000000000002841F0E384994FBE
:1033D0009DED0C5AD7ED007A974E65EEA77AE5EE93
:1033E000267AB0EE475AA7EE865AFDEEC57A17EE5A
:1033F00090EA17EE900A9E45A8BF18467145C8BFCF
:103400000846012A07EE900AF8EEE77AC6ED007A40
:103410003FF4CBAAD7ED047A9DED0D5A65EEA77A5D
:10342000E5EE267AB0EE475AA7EE865AFDEEC57A4B
:1034300017EE90EA17EE900A9E45A8BF1846714510
:10344000C8BF0846022A07EE900AF8EEE77AC6EDF2
:10345000017A3FF4AAAAD7ED087A9DED0E5A65EEDF
:10346000A77AE5EE267AB0EE475AA7EE865AFDEE29
:10347000C57A17EE90EA17EE900A9E45A8BF184647
:103480007145C8BF0846032A07EE900AF8EEE77AAE
:10349000C6ED027A3FF489AAD7ED0C7A9DED0F5A5A
:1034A00065EEA77AE5EE267AB0EE475AA7EE865A81
:1034B000FDEEC57A17EE90EA17EE900A9E45A8BF7A
:1034C00018467145C8BF0846042A07EE900AF8EE70
:1034D000E77AC6ED037A3FF468AAD7ED107A9DED3E
:1034E000105A65EEA77AE5EE267AB0EE475AA7EEB7
:1034F000865AFDEEC57A17EE90EA17EE900A9E45C1
:10350000A8BF18467145C8BF0846052A07EE900AAD
:10351000F8EEE77AC6ED047A3FF447AAD7ED147ABD
:103520009DED115A65EEA77AE5EE267AB0EE475A80
:10353000A7EE865AFDEEC57A17EE90EA17EE900ACE
:103540009E45A8BF18467145C8BF0846062A07EE23
:10355000900AF8EEE77AC6ED057A3FF426AAD7ED91
:10356000187A9DED125A65EEA77AE5EE267AB0EE4E
:10357000475AA7EE865AFDEEC57A17EE90EA17EE87
:10358000900A9E45A8BF18467145C8BF0846072A3D
:1035900007EE900AF8EEE77AC6ED067A3FF405AA40
:1035A000D7ED1C7A9DED135A65EEA75AE6EE855AC3
:1035B000A6EE257AFDEEC77A17EE900A8342A8BFE1
:1035C00003468142C8BF0B4607EE903AF8EEE77A11
:1035D000C6ED077A002A7FF4E8A9FFF7EBB9174B8D
:1035E0005A79002A3EF425AD154A1278002A3EF495
:1035F00020AD1B7807EE902AB7EE005ADFED114A96
:1036000007EE103A104BF8EEE77AB8EE477A1B88CF
:1036100067EE277A07EE103AB8EE477A87EE874AC8
:1036200084FE644A84FE054AFEF705BDF0EE676A33
:1036300018E500BF7C900120F02E0120CC800120F5
:103640000A740120713DAA3FF4730120002E00F09E
:10365000D683002842F04880B94FBAF1000F41F0FC
:10366000FB86FDEEE77A9DED0C5AB64E17EE901AEA
:10367000D7ED007A65EEA77AE5EE267AB0EE475AE6
:10368000A7EE865AFDEEC57A17EE90EA17EE900A7D
:103690009E45A8BF18467145C8BF0846012A07EED7
:1036A000900AF8EEE77AC6ED007A3FF47EA9D7EDEE
:1036B000047A9DED0D5A65EEA77AE5EE267AB0EE16
:1036C000475AA7EE865AFDEEC57A17EE90EA17EE36
:1036D000900A9E45A8BF18468E45B8BF0846022AE4
:1036E00007EE900AF8EEE77AC6ED017A3FF45DA99D
:1036F000D7ED087A9DED0E5A65EEA77AE5EE267AAB
:10370000B0EE475AA7EE865AFDEEC57A17EE90EA5C
:1037100017EE900A9E45A8BF18468E45B8BF0846CA
:10372000032A07EE900AF8EEE77AC6ED027A3FF434
:103730003CA9D7ED0C7A9DED0F5A65EEA77AE5EE20
:10374000267AB0EE475AA7EE865AFDEEC57A17EEF6
:1037500090EA17EE900A9E45A8BF18468E45B8BF5E
:103760000846042A07EE900AF8EEE77AC6ED037AD7
:103770003FF41BA9D7ED107A9DED105A65EEA77A9C
:10378000E5EE267AB0EE475AA7EE865AFDEEC57AE8
:1037900017EE90EA17EE900A9E45A8BF18468E4590
:1037A000B8BF0846052A07EE900AF8EEE77AC6ED9C
:1037B000047A3FF4FAA8D7ED147A9DED115A65EE1C
:1037C000A77AE5EE267AB0EE475AA7EE865AFDEEC6
:1037D000C57A17EE90EA17EE900A9E45A8BF1846E4
:1037E0008E45B8BF0846062A07EE900AF8EEE77A3B
:1037F000C6ED057A3FF4D9A8D7ED187A9DED125A97
:1038000065EEA77AE5EE267AB0EE475AA7EE865A1D
:10381000FDEEC57A17EE90EA17EE900A9E45A8BF16
:1038200018468E45B8BF0846072A07EE900AF8EEFC
:10383000E77AC6ED067A3FF4B8A8D7ED1C7A9DED7D
:10384000135A65EEA75AE6EE855AA6EE257AFDEEE6
:10385000C77A17EE900A8342A8BF03468142D8BFB9
:10386000194607EE901AF8EEE77AC6ED077A002AB5
:103870007FF49BA8FFF79EB8334BD3ED005AFFF7B8
:1038800042B9324944F620663148D1F8EC1000685C
:10389000B142A8BF3146B1F57A7FB8BF4FF47A7113
:1038A00010F0100FDBF8000089B2A4F81A1101F033
:1038B0007A83C00400F1B3832648D0F800E0BEF953
:1038C00032C0254F64262548A7FB0171D4F81C712E
:1038D000D0ED037A8809791CBDEEE77A04EB47073F
:1038E000C4F81C1196FBF0F014288DED047ABDF895
:1038F0001060A8BF1420A7F82061814203DB0020DC
:103900000146C4F81C0104EB4101B1F9201107EE96
:10391000101AB8EEC77A77EEC77AFDEEE77ACDEDEA
:10392000047ABDF9100080EAE071A1EBE071614515
:1039300002F376814FF07E5109480160FEF794BF93
:103940007C900120F02E01200C9001209C1D012074
:1039500038A60120C8340120D34D62100C74012018
:1039600088000120AD48B2EE0E7AD0ED027AF0EE7A
:10397000E76AF4EEC76AF1EE10FA41D5A84A128858
:1039800057073DD5A74AA849B2F90420A74E81FBA5
:103990000271D2173688C2EBA102921B92B211B209
:1039A00011F1B30F02DA02F5B47211B2B32902DDDC
:1039B000A1F5B47211B29E4F4FF6FF729D4E3F7942
:1039C0003678002F18BF012236077EF539AF9A4EA0
:1039D00011FB02F29949366892B2367E16FB02F666
:1039E00081FB0621F2173144C2EB211207EE102AA7
:1039F000B8EEC77A77EEC77AC0ED027AFEF720BF3D
:103A0000884A8949B2F90420884881FB0261D217AB
:103A1000C2EBA1020280FEF713BFAB68002B3EF49D
:103A200008AF05F1540128469847FEF702BF844FBE
:103A3000F9F754FAD4F8EC31824A8346C31AC4F831
:103A4000EC011268BB809B1AFB80FEF7FCB9F9F70A
:103A500045FA0B90FEF717B81E217B4806F087FA4F
:103A600000283FF428AC6E4B1B885F063FF523AC63
:103A700094F88431B34242F01981744BD4ED627AE8
:103A8000D3ED016A94ED435A28EE277ADFED705AA0
:103A900067EEC57A9FED6F6AA5EE267AE8EE267A84
:103AA00087FE657A87FE067A84ED437AC7FEE57A5B
:103AB000C7FE867AC4ED417AFFF7FDBBB4F8FC017E
:103AC000984240F2B085644B0120644D93ED007A3A
:103AD000D5ED007A624B77EE676AC4ED807AC4ED6B
:103AE0007E7A84ED817AC4ED7D6A84F80802DFED88
:103AF0005D7A93ED007AFEF7F7B9FDEEC87A504F84
:103B0000BE8017EE903AFB80FFF7D0BB564B1B8868
:103B1000002B40F0A785554A554B1178186805F0E1
:103B2000D5FAD4F8DC21089B9A1AFEF79CB8FDEE72
:103B3000C76A9FED478A424F87FE488A16EE90CAB1
:103B4000DFED446AA7F800C088FE268A84ED418A2A
:103B500000297FF4DBAAFFF7A9BBBDEEE77A384F57
:103B600017EE103ABB80FFF793BBBDEEE77ADFEDAF
:103B7000386A334F0129C7FEE67A17EE102A9FED07
:103B8000357A7A80C7FE877AC4ED427A3FF71AAB5E
:103B9000FFF78CBBF9F7A2F9294FA0EB0800354BD2
:103BA000B8801B78FFF7A5BB334B3448D3ED006AD0
:103BB000334B90ED006A1B78C4ED806A84ED816A16
:103BC000002B40F02C8576EEC65AF0EE466ABCEE2D
:103BD000C76AFF202B4B77EEC77AC4ED7D5A16EEED
:103BE000105AC4ED7E6A84F80802A4F8FC5193EDE3
:103BF000007AFEF779B9F5EEC06AF1EE10FA00F13D
:103C00006A86B7EE006A76EE666A86EE267AFFF777
:103C1000C7BADFED1D6AFFF766BA00BF0C7401205A
:103C2000849E0120C480012067666666C49F0120CF
:103C3000842E0120E4800120C834012089888888EE
:103C40002C730120142F012038A6012088000120A8
:103C500000C0F94400C0F9C45C2E0120FC90012092
:103C600018910120000000004C9301204E93012088
:103C70005093012028730120D4A401200091012039
:103C800054940120149101200000C842D7ED015A3C
:103C9000B0EE674A65EEC65AA5EE874AF4EEC44A0E
:103CA00074EE665AF1EE10FAC8BFF0EE455A012BD9
:103CB000C6ED005A3EF47EAED7ED055AB0EE674A27
:103CC00065EEC65AA5EE874AF4EEC44A74EE665A0B
:103CD000F1EE10FAC8BFF0EE455A022BC6ED015ABC
:103CE0003EF468AED7ED095AB0EE674A65EEC65AA3
:103CF000A5EE874AF4EEC44A74EE665AF1EE10FA65
:103D0000C8BFF0EE455A032BC6ED025A3EF452AE40
:103D1000D7ED0D5AB0EE674A65EEC65AA5EE874A52
:103D2000F4EEC44A74EE665AF1EE10FAC8BFF0EE33
:103D3000455A042BC6ED035A3EF43CAED7ED115A5A
:103D4000B0EE674A65EEC65AA5EE874AF4EEC44A5D
:103D500074EE665AF1EE10FAC8BFF0EE455A052B24
:103D6000C6ED045A3EF426AED7ED155AB0EE674ABA
:103D700065EEC65AA5EE874AF4EEC44A74EE666A4A
:103D8000F1EE10FAC8BFF0EE456A062BC6ED056AE3
:103D90003EF410AED7ED196AB0EE674AF3EE045A5E
:103DA00066EEC66AA6EE874AF4EEC44A74EE656A09
:103DB000F1EE10FAC8BFF0EE456A072BC6ED066AB1
:103DC0003EF4F8ADD7ED1D6A26EEC66AE6EE077A38
:103DD000F4EEE47A77EEE57AF1EE10FAB8BFF0EEA1
:103DE000457AC6ED077AFEF7E5BD99F82010C1EBDC
:103DF000411001EB8000C00080B2FEF742BDBF4F12
:103E0000BAF1000F41F03681FDEEE77A9DED0C5AD4
:103E1000BB4E17EE901AD7ED007A65EEA77AE5EE65
:103E2000267AB0EE475AA7EE865AFDEEC57A17EE0F
:103E300090CA17EE90EA9C45A8BF9E466145C8BF50
:103E40008E46012A07EE90EAF8EEE77AC6ED007A90
:103E50003EF485ABD7ED047A9DED0D5A65EEA77A59
:103E6000E5EE267AB0EE475AA7EE865AFDEEC57A01
:103E700017EE90CA17EE90EA9C45A8BF9E468C4567
:103E8000B8BF8E46022A07EE90EAF8EEE77AC6ED52
:103E9000017A3EF464ABD7ED087A9DED0E5A65EEDB
:103EA000A77AE5EE267AB0EE475AA7EE865AFDEEDF
:103EB000C57A17EE90CA17EE90EA9C45A8BF9E46B9
:103EC0008C45B8BF8E46032A07EE90EAF8EEE77AF3
:103ED000C6ED027A3EF443ABD7ED0C7A9DED0F5A56
:103EE00065EEA77AE5EE267AB0EE475AA7EE865A37
:103EF000FDEEC57A17EE90CA17EE90EA9C45A8BF72
:103F00009E468C45B8BF8E46042A07EE90EAF8EE2E
:103F1000E77AC6ED037A3EF422ABD7ED107A9DED39
:103F2000105A65EEA77AE5EE267AB0EE475AA7EE6C
:103F3000865AFDEEC57A17EE90CA17EE90EA9C45B8
:103F4000A8BF9E468C45B8BF8E46052A07EE90EA6C
:103F5000F8EEE77AC6ED047A3EF401ABD7ED147AB9
:103F60009DED115A65EEA77AE5EE267AB0EE475A36
:103F7000A7EE865AFDEEC57A17EE90CA17EE90EAC4
:103F80009C45A8BF9E468C45B8BF8E46062A07EEC4
:103F900090EAF8EEE77AC6ED057A3EF4E0AAD7EDAE
:103FA000187A9DED125A65EEA77AE5EE267AB0EE04
:103FB000475AA7EE865AFDEEC57A17EE90CA17EE5D
:103FC00090EA9C45A8BF9E468C45B8BF8E46072AFE
:103FD00007EE90EAF8EEE77AC6ED067A3EF4BFAA5D
:103FE000D7ED1C7A9DED135A65EEA75AE6EE855A79
:103FF000A6EE257AFDEEC77A17EE907ABB42A8BFEF
:104000003B46B942D8BF194607EE901AF8EEE77A58
:10401000C6ED077A00287EF4CDACFEF7A3BA394886
:10402000D0F800E0BEF832C04FEA5C0C49E4DFF89B
:10403000E090D4ED017AB0EE006AD4ED005AF6EECD
:10404000006A77EEA77AB9F80000D9F81420013891
:10405000B0EE664AB0EE677A1032D5EE867A04EB9F
:10406000C003A5EE867A083B67EEA67A27EE267A8D
:10407000C4ED217A84ED207A234C274604F1800197
:1040800093ED036A0138D7ED036AA3F1080393EDBA
:10409000047A07F1080776EEC65AD7ED007A12EDDA
:1040A000015A76EE266A77EE674A12ED026A77EEDB
:1040B000277A02F10802B0EE657A01F10801E6EE16
:1040C000247AA5EE247AE5EE267AA6EE667A67EEE5
:1040D000847A27EE047AC1ED007A81ED017ACFD19E
:1040E000B8F1140F7DF451ACF8F7F8FE059B074FBB
:1040F000C01AD4F8B0617880FDF747BC7C900120ED
:10410000F02E0120C83401201C2801202C7301202E
:104110008C2F0120D4F8B4E1B4F8ACA1EC4BCAF177
:1041200020090AEB4E175FFA89F903EB87075FEA6C
:10413000990001F05286013007F11003E5490001B2
:10414000E54A07EB000C13ED025A103311ED027A29
:10415000103253ED075A103151ED077A25EE075A08
:1041600013ED056A13ED087A65EEA75A51ED056A5D
:104170009C4551ED087A66EE266A02ED065A67EE16
:10418000277A42ED075A42ED056A42ED087ADAD104
:104190001038D249074401EB000C221819F0030330
:1041A00009D0B7EC017A013BFCEC017A67EE277A83
:1041B000E2EC017AF5D1BAF1000F91D04FEA89070C
:1041C000C34B5FEA9A0001EB070C03EBCE1E2744BA
:1041D00002F0C88001300EF110030CF1100107F15C
:1041E00010024FEA00190EEB090013ED025A1033CA
:1041F00011ED027A103253ED075A103151ED077A62
:1042000025EE075A13ED056A13ED087A65EEA75AF5
:1042100051ED056A984251ED087A66EE266A02ED84
:10422000065A67EE277A42ED075A42ED056A42EDDB
:10423000087ADAD1A9F1100086440CEB000107449A
:104240001AF0030A3FF44CAFBEEC017ABAF1010A4E
:10425000F1EC017A67EE277AE7EC017AF4D13FE7D7
:10426000D4F8B4919E4B4FEAC9029E499FED9E7AC5
:104270001344D1ED008A4A449C4F9B88F8EE688A2B
:1042800007EB820708EE103A643B68EE878AC82B7A
:10429000F8EE487AB8EEC89AA8BFC82368EEA78A95
:1042A000782BB8BF7823B0EE680A07EE903AB8EEE4
:1042B000E78A25F00BF8F0EE409AB0EE680A24F099
:1042C00067FF78EE097A79EE486AB8F1140F28EEA4
:1042D000098AB7EE006A66EEA76AF8EE007A88EE01
:1042E000267A60EE277A77EE076A89EEA67A77EE6D
:1042F000065A36EE477AC6EE256A67EEA67AC7ED0D
:10430000006A27EE267AC7ED026AC7ED017A87EDCB
:10431000047AC7ED037A01F0028709F10109744BB1
:104320000136744A83FB093E92F80080AEEBE97EC9
:10433000C4F8B0610EEB4E0EA9EB0E0EC4F8B4E15A
:10434000EAE6DFF8B891B9F80010D9F804C04FEAEE
:10435000510804EB81064FEA8802C90804EB020702
:1043600000F0A0800131103207F110035A4807EB2A
:10437000011E32440CF1100706F1100151ED047AD0
:10438000103310ED047A103713ED085A103052ED47
:10439000041A37EE271A12ED032A77EE670A51ED59
:1043A000034A75EE218A51ED023A71EEC51A12EDFB
:1043B000026A103112ED017A103251ED055A53EDB7
:1043C000072A53ED066A53ED057A32EE828A10ED24
:1043D000074A36EE860A10ED063A72EE622A10EDB2
:1043E000055A34EE249A00ED081A74EE644A33EE4E
:1043F000231A37EE874A00ED079A35EE252A00ED9D
:10440000061A77EE677A33EE631A00ED052A76EE28
:10441000666A03ED054A75EE655A43ED088A03EDB9
:10442000078A03ED060A9E4517ED077A17ED086A1D
:1044300064EE873A27EE603A26EE624A21EE865A0B
:10444000A4EE863AF0EE634AA2EE875AE0EE864A80
:10445000B0EE446A01ED073AA1EE876A41ED084AE1
:1044600002ED075A02ED086A17ED057A17ED066AA4
:1044700065EE873A27EE414A66EE674A26EE865A8F
:10448000A5EE864AE1EE063AE6EE874AA7EE875A9F
:1044900041ED063A01ED054A42ED064A02ED055AA4
:1044A0007FF46CAF1FFA88F862461348414621F04A
:1044B000CBFC4146D9F80420304621F0C5FC0D4B19
:1044C0001B78142B3FF410AED4F8B061FDF75DBA41
:1044D000A42F0120343101202C2801202431012077
:1044E000A4310120EC7D012027D4D236807D01202B
:1044F00056555555287301201C2801208C2F01206A
:10450000DFF8B492A148D9F80820B9F80C1023F0CC
:1045100063FC9F4B93F80080B8F1140F01F0E58520
:10452000D4F8B0610136C4F8B06182E5DFF88C924E
:1045300099F80020970801F0488607F1010C95488A
:104540004FEA4C1C00F12003A0F1700100EB0C0EAF
:1045500053ED077A203353ED0D6A103113ED0B7ACA
:1045600027EEA76A53ED097A66EEA66A53ED105A54
:1045700027EE077A67EEA77A53ED0E4A13ED0C5A31
:10458000A5EEA56A53ED0A5AE4EEA46AA5EE057AF3
:104590009E45E5EEA57AF1EEC65AB1EEE66AF1EE79
:1045A000C76AB1EEE77A41ED085A01ED076A41EDBD
:1045B000066A01ED057ACBD1ACF1200C04EB0717AC
:1045C000844412F0030111D00CF1080353ED017A79
:1045D000013913ED027A03F1080367EEA77AE7EEDB
:1045E000077AB1EEE77AA7EC017AEFD1B8F1140FB0
:1045F00001F086850136C4F8B061FDF737B9F8F7E8
:104600006DFC634B059093F80080D4F8B061B8F16D
:10461000140F7DF411A9604F3E80FDF70DB976EEC1
:10462000665AFFF7D4BA5D4B5D48D3ED007A5D4B17
:1046300090ED007A1B78C4ED807A84ED817A002BAE
:1046400001F0E88277EE676AFF20574BC4ED7E7A6F
:10465000C4ED7D6A84F80802DFED5B7A93ED007AA1
:10466000FDF742BC51494B69002B3DF4FCAA504870
:104670004FF0010E4F4B008893FBF0F00B68186071
:1046800081F811E0FDF7EFBADFF8348167EE897A3F
:10469000DFF8309129EE088AD8ED006A69EE288AA1
:1046A00098ED057A09EB8603D8ED015AA6EEA77AB4
:1046B00098ED066AD8ED046AA5EEA76A98ED035A4C
:1046C000D8ED025A66EEC76A83ED007A20EE070A3B
:1046D000A5EE476AE5EEA76A88ED056AC8ED066AA9
:1046E00024F0A8FD98ED097A98ED0E5A09EB8602A0
:1046F000D8ED127A00B2D8ED175AA7EE085AD8EDC5
:104700000A6A1346E8EEA75A98ED0F6AD8ED137AB5
:1047100098ED187AA6EE886AD8ED0D6AA8EEA77A09
:10472000D8ED167A66EEC56A98ED0C3A67EEE57A32
:10473000D8ED0B3A98ED154AD8ED144AA3EE456A28
:10474000E3EE886A82ED205AA5EEC47A0022E8EEF4
:10475000A47AC3ED405AC4F89C21C4F8A02188ED86
:104760000E6AC8ED0F6A88ED177AC8ED187AC4F89A
:10477000A421FEF721BC0D494A69002A3DF4A2AAF2
:104780000A6813604B74FDF79DBA00BF1C28012016
:10479000287301209C2801202C730120D4A401201F
:1047A0000091012054940120149101205493012080
:1047B0006C93012020A107008C2F0120862F01205F
:1047C00028320120A42F012000000000B5F940107C
:1047D0000123AA6207EE901A2967C5F88C30F8EE1B
:1047E000E77A0023B8F1010FC5ED207AC5ED1F7AF5
:1047F000C5F8843001F03782B0457DF407AFB5F9D4
:1048000042100022012307EE901AEA626967B8EEAF
:10481000E77AC5F8A0300023B8F1010F85ED257ABD
:1048200085ED247AC5F8983001F01982B0457DF401
:104830001EAFB5F94430002207EE903AAB67012372
:104840002A63B8EEE77AC5F8B4300023B8F1010F57
:1048500085ED2A7A85ED297AC5F8AC307DF438AF3C
:104860001FED278AB9F1030F3DD0BAF1000F09D02F
:1048700007EE90AAF8EEE77AF4EEC87AF1EE10FAB5
:1048800001F1A884AB6F0022B34903EB5603F88013
:1048900093FBF6F60B6894F8B8112E639A621A63CC
:1048A000DA6231B1AD4B1B8823F40063002B7DF439
:1048B00010AFAB4B1B6813F4003341F0C8811946AD
:1048C000A848C25C0C33012A00F0938501311529F8
:1048D000F7D1FDF7FEBEB7EE007AFEF761BCB7EE8A
:1048E000007AFEF7CFBCB0EE480A24F0A3FC00B279
:1048F000BBE7B4F84861013E36B2A4F84861FEF760
:104900000EB8B4F81A0100F57A7080B2FDF7B9BF9D
:10491000954F3A78013A0A2A1CD8DFE812F0630171
:104920008C01CD00AC0093007700620051003F0184
:1049300007010B008D4A8E4952680968C8328A42C5
:1049400003D321F01FFF28B1B378032B01F0DF85DB
:1049500001233B70F378002B3EF4C6AC854B1B78EB
:10496000DB0740F14881DFF80892D4F89821D9F8A4
:1049700000309A4200F24B813B78012B3EF4B4ACFC
:1049800094F89421002A3EF4AFAC0B2B0DD80122F1
:1049900040F603019A4012EA01060CD112F4C06FEE
:1049A00003D0093B012B41F2F785D9F800200B21F8
:1049B0006E4B39705A60002384F89431FEF794BC32
:1049C00021F0C0FE09F0E2FA0028C3D021F0DAFE9F
:1049D0000028BFD0684A0A21684B126839701A60F3
:1049E000B8E721F0AFFE00220520654B0292114688
:1049F0000192A3F108020090532009F07DFF0028E6
:104A0000A8D15A4A082310603B70A3E721F09AFE10
:104A10005C4A4FF007090021A2F10C000292A2F1BA
:104A20000803CDF800900190143A472009F064FF84
:104A300000288FD14D4B4FF0FF3287F8009083E86C
:104A4000050087E721F07EFE002202204E4B0292F5
:104A500011460192A3F108020090482009F04CFF92
:104A600000287FF477AF414B4FF0FF31062283E8F7
:104A700003003A706EE721F065FE444A2823502176
:104A8000A2F10C0002920093A2F10A030190163ADF
:104A9000492009F031FF00287FF45CAFDBF80030DB
:104AA00013F0800301F0C084304B4FF0FF3105223A
:104AB00083E803003A704DE7DFF8B09021F042FE42
:104AC0002B4AD9F80430126864339342BFF442AFE2
:104AD000402021F01DFE00287FF43CAFD9F80030C3
:104AE0004FF0400A2A49DFF8B0B013E0049121F0FA
:104AF0006BFEDBF80020BAF1010AD9F8003002F1B0
:104B0000FF32049903F10103CBF80020C9F800300B
:104B100001F0F784CB5C1846002BE7D100214FF061
:104B2000FF32042389E806003B7013E7194B1B781A
:104B3000002B01F045831A201AF0A6FB002841F053
:104B40003F8394F89431002B41F03A8309233B7062
:104B500022F0D2FAFEE600BF50840120309E0120F0
:104B6000C42B012000C0030813360120602E012051
:104B7000A4A20120D0890120BCA40120B4A401205A
:104B800018BB0308D0BA0308B4BA0308E2B8030894
:104B90007CB803086C2F01209CA401201A201AF075
:104BA00073FB0028D4D06B4B1B88002BD0D16A4BF1
:104BB0004520D3F8009021F007FE0E2021F004FEDE
:104BC000484621F0A4FEDDF82090484621F09FFEE3
:104BD000624A634B0A211268484639701A6021F014
:104BE00057FFB5E75F4B1B78DA0701F1CE83F37807
:104BF000002B3EF479AB19F0C1FC00283FF4B3AEB2
:104C0000594A41F2883312681344C4F898313B780A
:104C1000012B7EF469AB94F89431002B7EF464ABE5
:104C2000B378032B01F0B08409F0F4FF012384F87A
:104C30009431FEF759BB4C4800234C4A03210068CD
:104C4000136050604A4A3970136083E6494ADFEDC9
:104C50004A7A92ED080AB4EEE70AF1EE10FA40F251
:104C60003B85049324F07CFBD4ED457A20EE270AA3
:104C700024F0E0FAB0F5617F049B00F36A8607EE4A
:104C8000900A07EE106AF8EEE76ADFED3C7AB8EEBC
:104C9000C77A66EEA76AFDEEE67A17EE902A203212
:104CA000402A41F248829FED360A049324F0C2FA6A
:104CB00000B2049B07EE900AB8EEE77A3148D0EDD7
:104CC000037A77EE877AC0ED037AFDF7C8BD099BBA
:104CD000187800F0010000287DF46CAEFDF742BCAE
:104CE000294BDFED2A7A1B68C4ED727A13F08058E5
:104CF00040F097834E0200F14686B6EE007AF4EE5D
:104D0000C75AF1EE10FACCBF01230023002B40F06C
:104D10003A869846FDF7D2BAF8F7E0F88046FDF7F4
:104D200080BD77EEE47AB7EE007AC4ED727AF4EEE5
:104D3000C77AF1EE10FA40F3828785EE277A8DED7F
:104D40000C7AFDF7B1BA1249897B00297DF47FAD59
:104D5000FDF765BFACA40120A8A40120BCA40120DC
:104D6000B4A40120D0890120A4A20120602E01203A
:104D70009CA40120502B01208FC2753CD06D393A84
:104D8000000000000C74012038A601200000008003
:104D90006C9201200498B54F002800F02586D7EDCD
:104DA000007A9DED0C5A65EEA77AB14EE5EE267AB3
:104DB000B0EE475AA7EE865AFDEEC57A17EE90EA96
:104DC00017EE900A9E45A8BF18467145C8BF084611
:104DD000012A07EE900AF8EEE77AC6ED007A3DF474
:104DE000E9ADD7ED047A9DED0D5A65EEA77AE5EEB3
:104DF000267AB0EE475AA7EE865AFDEEC57A17EE30
:104E000090EA17EE900A9E45A8BF18467145C8BFA4
:104E10000846022A07EE900AF8EEE77AC6ED017A14
:104E20003DF4C8ADD7ED087A9DED0E5A65EEA77A30
:104E3000E5EE267AB0EE475AA7EE865AFDEEC57A21
:104E400017EE90EA17EE900A9E45A8BF18467145E6
:104E5000C8BF0846032A07EE900AF8EEE77AC6EDC7
:104E6000027A3DF4A7ADD7ED0C7A9DED0F5A65EEB1
:104E7000A77AE5EE267AB0EE475AA7EE865AFDEEFF
:104E8000C57A17EE90EA17EE900A9E45A8BF18461D
:104E90007145C8BF0846042A07EE900AF8EEE77A83
:104EA000C6ED037A3DF486ADD7ED107A9DED105A2C
:104EB00065EEA77AE5EE267AB0EE475AA7EE865A57
:104EC000FDEEC57A17EE90EA17EE900A9E45A8BF50
:104ED00018467145C8BF0846052A07EE900AF8EE45
:104EE000E77AC6ED047A3DF465ADD7ED147A9DED11
:104EF000115A65EEA77AE5EE267AB0EE475AA7EE8C
:104F0000865AFDEEC57A17EE90EA17EE900A9E4596
:104F1000A8BF18467145C8BF0846062A07EE900A82
:104F2000F8EEE77AC6ED057A3DF444ADD7ED187A90
:104F30009DED125A65EEA77AE5EE267AB0EE475A55
:104F4000A7EE865AFDEEC57A17EE90EA17EE900AA4
:104F50009E45A8BF18467145C8BF0846072A07EEF8
:104F6000900AF8EEE77AC6ED067A3DF423ADD7ED68
:104F70001C7A9DED135A65EEA75AE6EE855AA6EE09
:104F8000257AFDEEC77A17EE902A9342A8BF134602
:104F90008A42A8BF194607EE901AF8EEE77AC6EDE6
:104FA000077AFDF707BDC6003EF583ACFDF75CBC94
:104FB000012A40F3588607EE101AB8EEC77AC7EEFA
:104FC000876AB1EEE68AB9F1030F13D0BAF1000F88
:104FD00009D007EE90AAF8EEE77AF4EEC87AF1EE7F
:104FE00010FA01F1F7802B6F03EB560393FBF6F3F6
:104FF000AB6201E4B0EE480A24F01CF900B2E5E728
:10500000012A7FF72DAC07EE101AB8EEC77AC7EE6B
:10501000876AB1EEE68A25E4012A40F3208607EE8E
:10502000101AB8EEC77AC7EE876AB1EEE68AB9F110
:10503000030F14D0BAF1000F09D007EE90AAF8EED2
:10504000E77AF4EEC87AF1EE10FA01F1C3806B6FE3
:1050500003EB560393FBF6F3EB62FFF7E7BBB0EE0F
:10506000480A24F0E7F800B2E4E700BF7C90012092
:10507000F02E0120BDEEE75A9DED0C4AED4E15EEE7
:10508000101A97ED005A25EE855AA4EE265AB0EE76
:10509000474AA5EE064AF4EEC44AB0EE445AF1EE91
:1050A00010FA88BFB0EE675ABDEEC55A15EE10EA89
:1050B00015EE10CA9E45A8BF9C467145C8BF8C46D8
:1050C000012A05EE10CAB8EEC55A86ED005A3DF425
:1050D00046AA97ED045A9DED0D4A25EE855AA4EE99
:1050E000265AB0EE474AA5EE064AF4EEC44AB0EEA0
:1050F000445AF1EE10FA88BFB0EE675ABDEEC55AB9
:1051000015EE10EA15EE10CA9E45A8BF9C468E45C6
:10511000B8BF8C46022A05EE10CAB8EEC55A86ED15
:10512000015A3DF41CAA97ED085A9DED0E4A25EE52
:10513000855AA4EE265AB0EE474AA5EE064AF4EE8A
:10514000C44AB0EE445AF1EE10FA88BFB0EE675A86
:10515000BDEEC55A15EE10EA15EE10CA9E45A8BF61
:105160009C468E45B8BF8C46032A05EE10CAB8EEA1
:10517000C55A86ED025A3DF4F2A997ED0C5A9DED01
:105180000F4A25EE855AA4EE265AB0EE474AA5EE00
:10519000064AF4EEC44AB0EE445AF1EE10FA88BF63
:1051A000B0EE675ABDEEC55A15EE10EA15EE10CAFC
:1051B0009E45A8BF9C468E45B8BF8C46042A05EE86
:1051C00010CAB8EEC55A86ED035A3DF4C8A997ED4A
:1051D000105A9DED104A25EE855AA4EE265AB0EEDF
:1051E000474AA5EE064AF4EEC44AB0EE445AF1EE40
:1051F00010FA88BFB0EE675ABDEEC55A15EE10EA38
:1052000015EE10CA9E45A8BF9C468E45B8BF8C4679
:10521000052A05EE10CAB8EEC55A86ED045A3DF4CB
:105220009EA997ED145A9DED114A25EE855AA4EEDC
:10523000265AB0EE474AA5EE064AF4EEC44AB0EE4E
:10524000445AF1EE10FA88BFB0EE675ABDEEC55A67
:1052500015EE10EA15EE10CA9E45A8BF9C468E4575
:10526000B8BF8C46062A05EE10CAB8EEC55A86EDC0
:10527000055A3DF474A997ED185A9DED124A25EE92
:10528000855AA4EE265AB0EE474AA5EE064AF4EE39
:10529000C44AB0EE445AF1EE10FA88BFB0EE675A35
:1052A000BDEEC55A15EE10EA15EE10CA9E45A8BF10
:1052B0009C468E45B8BF8C46072A05EE10CAB8EE4C
:1052C000C55A86ED065A3DF44AA997ED1C5A9DED44
:1052D000134A65EE855AE6EE845AA6EE257AF4EE78
:1052E000C74AF1EE10FAD8BFF0EE477AFDEEE77A42
:1052F000FEF782BE504A5149B2F90430DFED507AD0
:1053000081FB0312DB17C3EBA2031BB208EE103ABA
:10531000B8EEC88A28EE278AB0EE480A04F054FD99
:10532000F0EE408AB0EE480A04F0D6FC454BD9783E
:10533000002900F03883444E44F25060B4F98E21C5
:10534000B6F902309B1A834240F3A784A3F50C43BD
:10535000A03B4842984200F394848B42A8BF0B467E
:105360001344B6F90020B4F98C6144F250671BB2C3
:10537000921BA4F88E31BA4240F38684A2F50C4207
:10538000A03A904203DC9142A8BF11460846321869
:1053900007EE903A9FED2D6A13B2F8EEE76A07EE3A
:1053A000903AA4F88C31F8EEE77A27EEE87A60EECE
:1053B000277AA0EE267AE8EEA67A27EE067A67EE3E
:1053C000867ABDEEC77AFDEEE77A17EE102A17EE61
:1053D000903AA4F89021A4F89231FDF77DBF1C48C3
:1053E000FDF7D7BA8223FCF7BCBADFED1A7AFCF7D7
:1053F00083BAD4F8BC214B003AB156785A1800EB66
:1054000082025278B242BDF464A90B44002200EB40
:105410008300A4F81022C4F81422C4F8BC01FDF7DC
:1054200058B9B7EE007A77EE677AC5FEE75AFCF70F
:1054300043BF00BFF02E0120C4800120676666666E
:1054400035FA8E3C489F0120A49F0120CDCCCC3D55
:105450000C74012000000243BDEEE75A9DED0C4A9A
:105460009F4E15EE101A97ED005A25EE855AA4EEC0
:10547000265AB0EE474AA5EE064AF4EEC44AB0EE0C
:10548000445AF1EE10FA88BFB0EE675ABDEEC55A25
:1054900015EE100A15EE10EA9842A8BF9E4681420A
:1054A000C8BF8E46012A05EE10EAB8EEC55A86ED51
:1054B000005A3DF47AAA97ED045A9DED0D4A25EE67
:1054C000855AA4EE265AB0EE474AA5EE064AF4EEF7
:1054D000C44AB0EE445AF1EE10FA88BFB0EE675AF3
:1054E000BDEEC55A15EE100A15EE10EA9842A8BF97
:1054F0009E468842B8BF8E46022A05EE10EAB8EEF4
:10550000C55A86ED015A3DF450AA97ED085A9DED13
:105510000E4A25EE855AA4EE265AB0EE474AA5EE6D
:10552000064AF4EEC44AB0EE445AF1EE10FA88BFCF
:10553000B0EE675ABDEEC55A15EE100A15EE10EA28
:105540009842A8BF9E468842B8BF8E46032A05EE01
:1055500010EAB8EEC55A86ED025A3DF426AA97ED38
:105560000C5A9DED0F4A25EE855AA4EE265AB0EE50
:10557000474AA5EE064AF4EEC44AB0EE445AF1EEAC
:1055800010FA88BFB0EE675ABDEEC55A15EE100A84
:1055900015EE10EA9842A8BF9E468842B8BF8E46D4
:1055A000042A05EE10EAB8EEC55A86ED035A3DF41A
:1055B000FCA997ED105A9DED104A25EE855AA4EEF0
:1055C000265AB0EE474AA5EE064AF4EEC44AB0EEBB
:1055D000445AF1EE10FA88BFB0EE675ABDEEC55AD4
:1055E00015EE100A15EE10EA9842A8BF9E468842B2
:1055F000B8BF8E46052A05EE10EAB8EEC55A86ED0C
:10560000045A3DF4D2A997ED145A9DED114A25EEA6
:10561000855AA4EE265AB0EE474AA5EE064AF4EEA5
:10562000C44AB0EE445AF1EE10FA88BFB0EE675AA1
:10563000BDEEC55A15EE100A15EE10EA9842A8BF45
:105640009E468842B8BF8E46062A05EE10EAB8EE9E
:10565000C55A86ED055A3DF4A8A997ED185A9DED57
:10566000124A25EE855AA4EE265AB0EE474AA5EE18
:10567000064AF4EEC44AB0EE445AF1EE10FA88BF7E
:10568000B0EE675ABDEEC55A15EE100A15EE10EAD7
:105690009842A8BF9E468842B8BF8E46072A05EEAC
:1056A00010EAB8EEC55A86ED065A3DF47EA997ED8C
:1056B0001C5A9DED134A65EE855AE6EE845AA6EE15
:1056C000257AF4EEC74AF1EE10FAD8BFF0EE477A29
:1056D000FDEEE77AFEF7BDB89FED027AFFF7EEBA6E
:1056E000F02E012000000000B74F9DED0C4A97ED11
:1056F000005A049925EE855AA4EE265AB0EE474A80
:10570000A5EE064AB0EE445A002900F0AA83BAF189
:10571000000F06D0F4EE444AF1EE10FAC8BFB0EE26
:10572000675AFDEEE77A17EE900AFDEEC57A05EEB0
:10573000100A17EE901A884200F303869942A8BF18
:10574000194607EE901AF8EEE77AA04E012AC6ED48
:10575000007A3DF42FA9D7ED047A9DED0D4A65EE50
:10576000A77AE4EE267AB0EE474AA7EE864AF0EE34
:10577000447ABAF1000F00F07285F4EEC44AF1EEFB
:1057800010FA40F36C8501469942A8BF194607EE0E
:10579000901AF8EEE77A022AC6ED017A3DF40AA9DA
:1057A000D7ED087A9DED0E4A65EEA77AE4EE267AEB
:1057B000B0EE474AA7EE864AF0EE447ABAF1000FFF
:1057C00000F04285F4EEC44AF1EE10FA40F33C8555
:1057D00001469942A8BF194607EE901AF8EEE77AFB
:1057E000032AC6ED027A3DF4E5A8D7ED0C7A9DEDCB
:1057F0000F4A65EEA77AE4EE267AB0EE474AA7EEA6
:10580000864AF0EE447ABAF1000F00F01285F4EE09
:10581000C44AF1EE10FA40F30C8501469942A8BF44
:10582000194607EE901AF8EEE77A042AC6ED037AD5
:105830003DF4C0A8D7ED107A9DED104A65EEA77A29
:10584000E4EE267AB0EE474AA7EE864AF0EE447AB6
:10585000BAF1000F00F0E284F4EEC44AF1EE10FA5F
:1058600040F3DC8401469942A8BF194607EE901A1E
:10587000F8EEE77A052AC6ED047A3DF49BA8D7ED49
:10588000147A9DED114A65EEA77AE4EE267AB0EE21
:10589000474AA7EE864AF0EE447ABAF1000F00F0CC
:1058A000B284F4EEC44AF1EE10FA40F3AC8401463F
:1058B0009942A8BF194607EE901AF8EEE77A062A31
:1058C000C6ED057A3DF476A8D7ED187A9DED124A1B
:1058D00065EEA77AE4EE267AB0EE474AA7EE864A4E
:1058E000F0EE447ABAF1000F00F08284F4EEC44A7C
:1058F000F1EE10FA40F37C8401469942A8BF1946A4
:1059000007EE901AF8EEE77A072AC6ED067A3DF41C
:1059100051A8D7ED1C7A9DED134A65EEA75AE4EE27
:10592000265AA5EE867ABAF1000F00F05884B4EE3C
:10593000E47AF1EE10FA40F1528402469A42A8BF8E
:105940001A4605EE102AB8EEC55A86ED075AFDF73D
:1059500031B807EE906ADFED1E6AB8EEE77A66EEC0
:10596000A65A9FED1C5A9FED1C6ADFED1C7AA5EE2E
:10597000856A26EEA55AE5EE867AE5EE276A26EEDA
:10598000870AFFF792B94FF00008B6EE007A67EE8B
:10599000877AF4EEE75AF1EE10FA7FF542ADF0EEB9
:1059A000675AFCF789BC0E4B9FED0E6AB3F90020D5
:1059B000B3F9023007EE902A06EE903AF8EEE77A55
:1059C000F8EEE66AF1E400BF7C900120F02E0120A1
:1059D00084F9223F92E741B99730083C15A82ABEC6
:1059E000A49F0120CDCCCC3D97ED005ADDED0C4AB3
:1059F00025EE855AA4EEA65AF0EE474AE5EE064A91
:105A0000BDEEE45A15EE100A814200F32782984257
:105A1000A8BF184605EE100AB8EEC55AB8F1000F37
:105A200000F0F085EF4E012A86ED005A3CF4C2AF3B
:105A300097ED045ADDED0D4A25EE855AA4EEA65ADF
:105A4000F0EE474AE5EE064ABDEEE45A15EE100ABE
:105A5000814200F300829842A8BF184605EE100A62
:105A6000B8EEC55AB8F1000F00F02286022A86ED82
:105A7000015A3CF49FAF97ED085ADDED0E4A25EE32
:105A8000855AA4EEA65AF0EE474AE5EE064ABDEE68
:105A9000E45A15EE100A814200F3DA819842A8BF59
:105AA000184605EE100AB8EEC55AB8F1000F00F01E
:105AB000F585032A86ED025A3CF47CAF97ED0C5A2B
:105AC000DDED0F4A25EE855AA4EEA65AF0EE474AC0
:105AD000E5EE064ABDEEE45A15EE100A814200F3E7
:105AE000B4819842A8BF184605EE100AB8EEC55A10
:105AF000B8F1000F00F0C885042A86ED035A3CF483
:105B000059AF97ED105ADDED104A25EE855AA4EEF7
:105B1000A65AF0EE474AE5EE064ABDEEE45A15EE07
:105B2000100A814200F38E819842A8BF184605EE04
:105B3000100AB8EEC55AB8F1000F00F09285052A98
:105B400086ED045A3CF436AF97ED145ADDED114A58
:105B500025EE855AA4EEA65AF0EE474AE5EE064A2F
:105B6000BDEEE45A15EE100A814200F333819842EB
:105B7000A8BF184605EE100AB8EEC55AB8F1000FD6
:105B800000F06585062A86ED055A3CF413AF97EDC3
:105B9000185ADDED124A25EE855AA4EEA65AF0EE0B
:105BA000474AE5EE064ABDEEE45A15EE100A814278
:105BB00000F30D819842A8BF184605EE100AB8EE12
:105BC000C55AB8F1000F00F0F584072A86ED065A91
:105BD0003CF4F0AE97ED1C5ADDED134A65EE855AA4
:105BE000E6EEA45AA5EE867ABDEEC77A17EE102A25
:105BF000914203DC9A42A8BF1A46114607EE101ADA
:105C0000B8EEC77AB8F1000F00F0668286ED077A29
:105C1000FCF7D0BE77EEC76AF0EE477AFEF714BD08
:105C2000BEF834109FED707A07EE901A6F49F8EEC7
:105C3000E77A67EE877AC1ED007AFCF715BE6C4B08
:105C40001B6813F080587FF4A0AEFFF753B8694B80
:105C50001B78032B00F089830023FEF730BE9FEDF5
:105C6000668AFFF7E4B99FED648AFFF7ACB99FED50
:105C7000630A634F25EE800A23F0DCFAF880FEF712
:105C800023BC0346FFF76CBB5E4FBA42BFF679AB4D
:105C900002F50C42A032FFF774BB5A488342BFF6AC
:105CA00058AB03F50C43A033FFF753BB07EE906AE4
:105CB0009FED557ADFED556AF8EEE77A84F8846156
:105CC00067EE877A37EEA67ABDEEC76A16EE103A0F
:105CD0002033402B40F2EF82DFED476ABDEEE77ADA
:105CE000424BC3ED016A17EE103A2033402B00F20D
:105CF000DF829FED477AF4EEC77AF1EE10FA40F3B7
:105D00001B84DFED445A9FED446AF4EEC67A37EE09
:105D1000E57AF1EE10FAF0EE477AF6DCDFED3F7A45
:105D2000B4EEE77AF1EE10FA40F10384DFED395A70
:105D30009FED3B6AB4EEC67A77EE257AF1EE10FA63
:105D4000B0EE677AF6D49FED317AF4EEC77AF1EED1
:105D500010FA40F3FA829FED2E7A77EE677A67EEBB
:105D6000A75A9FED305A9FED306A9FED307AA5EE2D
:105D7000856A27EEA55AA5EE867AE5EE077AC4ED88
:105D8000627AFDF77FBE2A48069390ED000A0591DE
:105D9000049223F04FFADFF8A4E0DFF8A4C0DEF8A5
:105DA000ECE0174F8CFB0E3C4FEAEE7E3880CEEBDA
:105DB000AC1E049A059907EE90EA069BF8EEE77A86
:105DC000FDEEE77A17EE900A7880FCF7A8BD05EEA5
:105DD000101AF4E605EE101ACEE61649164A8C465D
:105DE000FEF7DCB9F02E01206F12833A8800012003
:105DF00038A60120099E0120000000000000C842D2
:105E00002C730120B0B9FFFF35FA8E3CDB0FC93F80
:105E1000DB0F4940DB0FC940E4CB1641DB0F49C023
:105E2000E4CB16C192E741B99730083C15A82ABEC9
:105E30000C740120243101201C2801209C1D01200C
:105E4000D34D621005EE101A73E605EE101A4DE6FA
:105E500005EE101A27E605EE101A01E605EE101AF7
:105E6000DAE5BAF1000F06D0F4EE444AF1EE10FA8A
:105E7000C8BFB0EE675ABDEEE74ABDEEC55A14EE94
:105E8000100A14EE109A15EE101A884200F3C98217
:105E90009942A8BF194605EE101AB8EEC55AB8F1D6
:105EA000000F00F0E883F34E012A86ED005A3CF41F
:105EB00081AD97ED045A9DED0D4A25EE855AA4EE6D
:105EC000265AB0EE474AA5EE064AB0EE445ABAF159
:105ED000000F00F09182F4EEC44AF1EE10FA40F3A4
:105EE0008B8201469942A8BF194605EE101AB8EEFA
:105EF000C55AB8F1000F00F0A183022A86ED015ABD
:105F00003CF458AD97ED085A9DED0E4A25EE855AA2
:105F1000A4EE265AB0EE474AA5EE064AB0EE445A21
:105F2000BAF1000F00F05F82F4EEC44AF1EE10FA0D
:105F300040F3598201469942A8BF194605EE101A4E
:105F4000B8EEC55AB8F1000F00F06F83032A86ED52
:105F5000025A3CF42FAD97ED0C5A9DED0F4A25EEF9
:105F6000855AA4EE265AB0EE474AA5EE064AB0EE90
:105F7000445ABAF1000F00F02D82F4EEC44AF1EE5B
:105F800010FA40F3278201469942A8BF194605EE50
:105F9000101AB8EEC55AB8F1000F00F0E982042AD1
:105FA00086ED035A3CF406AD97ED105A9DED104A6C
:105FB00025EE855AA4EE265AB0EE474AA5EE064ACB
:105FC000B0EE445ABAF1000F00F0FB81F4EEC44A7F
:105FD000F1EE10FA40F3F58101469942A8BF194647
:105FE00005EE101AB8EEC55AB8F1000F00F0B782EE
:105FF000052A86ED045A3CF4DDAC97ED145A9DED6C
:10600000114A25EE855AA4EE265AB0EE474AA5EE6F
:10601000064AB0EE445ABAF1000F00F0C981F4EE1E
:10602000C44AF1EE10FA40F3C38101469942A8BF79
:10603000194605EE101AB8EEC55AB8F1000F00F077
:10604000EB82062A86ED055A3CF4B4AC97ED185A5B
:106050009DED124A25EE855AA4EE265AB0EE474A27
:10606000A5EE064AB0EE445ABAF1000F00F097814F
:10607000F4EEC44AF1EE10FA40F3918101469942E0
:10608000A8BF194605EE101AB8EEC55AB8F1000FB0
:1060900000F05982072A86ED065A3CF48BAC97ED46
:1060A0001C5A9DED134A65EE855AE6EE845AA6EE1B
:1060B000257ABAF1000F40F0A881BDEEC77A17EE3D
:1060C000102A904240F3A88107EE109AB8EEC77AE2
:1060D000B8F1000F7FF49AAD059B002B7FF496ADCD
:1060E000F445B8BFB0EE677A90E5F6F7F7FE059B8A
:1060F000614FC01A614B788093F80080FEF710BAA8
:10610000F6F7ECFE059B5C4FC01A5C4B99F800203B
:10611000D4F8B061B88093F80080FEF76BBAF6F758
:10612000DDFE059B544FC01AD4F8B491D4F8B06189
:106130007880FEF7F2B8DFED587AF4EEE76AF1EE18
:1061400010FA40F34182DFED515A9FED4F6AF4EEB1
:10615000C66A76EEE57AF1EE10FAF0EE676AF6DCE2
:10616000DFED526AF4EEE67AF1EE10FA40F10982C0
:10617000DFED465A9FED466AF4EEC67A77EEA56AE1
:10618000F1EE10FAF0EE667AF6D4DFED427AF4EE34
:10619000E76AF1EE10FA05DDDFED3F7A77EEE66AA9
:1061A000FFF7DDBBDFED407AF4EEE76AF1EE10FABF
:1061B0007FF5D5ABDFED3D7A77EEE66AFFF7CFBB33
:1061C000089820F065FCFEF7C3BC2D4F07F1800C4A
:1061D000FEF7F7B9F880A5F8B860FCF782BAFDEED3
:1061E000C77A17EE902A8242FFF6ADABFFF7A6BB47
:1061F000FDEEE77A17EE901A8142BFF67EAB07EE0E
:10620000900AFFF77FBBFDEEE77A17EE901A814206
:10621000BFF64EAB07EE900AFFF74FBBFDEEE77AF5
:1062200017EE901A8142BFF61EAB07EE900AFFF7F9
:106230001FBBFDEEE77A17EE901A8142BFF6EEAA79
:1062400007EE900AFFF7EFBAFDEEE77A17EE901A25
:106250008142BFF6BEAA07EE900AFFF7BFBAFDEE75
:10626000E77A17EE901A8142BFF68EAA07EE900ADF
:10627000FFF78FBAF02E01202C7301202873012024
:106280001C28012000000000E4CB1641DB0FC940B0
:10629000E4CB16C1DB0FC93FDB0F494092E741B9A0
:1062A0009730083C15A82ABEDB0FC9BFDB0F49C0D9
:1062B0005FED0C7A63E5F4EEE67AF1EE10FA40F366
:1062C000FA805FED0E5A1FED106AB4EEC67A77EED3
:1062D000656AF1EE10FAB0EE667AF6DC1FED0D7A23
:1062E000F4EEC76AF1EE10FA40F1A7805FED195A9B
:1062F0001FED196AF4EEC66A36EEA57AF1EE10FAD1
:10630000F0EE476AF6D45FED1D6AB4EEE67AF1EE80
:1063100010FA2EDD5FED206A36EEC77A67EE075A77
:106320001FED225A1FED226A5FED226AA5EE856AF3
:1063300027EE255AE5EE866AA5EE267AF0EE476A44
:10634000CCE407EE900AFFF7FEB91FED297AF4EED0
:10635000C77AF1EE10FA7FF502AD1FED2C7A77EED9
:10636000677AFCE46146FDF76BBF1AF041F9FCF770
:10637000B0B95FED336AB4EEE67AF1EE10FACDD53E
:106380005FED366A36EEC77AC8E7802021F0C4F8A0
:1063900008B10DF0B5FD08F03DFCFEF7DBBABDEE2F
:1063A000C55A15EE101A8142BFF669AE014669E67C
:1063B000BDEEC55A15EE101A8142BFF637AE014642
:1063C00037E6BDEEC55A15EE101A8142BFF605AE8E
:1063D000014605E6BDEEC55A15EE101A8142BFF61C
:1063E000D3AD0146D3E5BDEEC55A15EE101A814274
:1063F000BFF6A1AD0146A1E5BDEEC55A15EE101AD6
:106400008142BFF66FAD01466FE5F4EEC74AF1EE8B
:1064100010FA7FF752AE02469342A8BF1346994640
:1064200052E614EE101A36E5A64A4FF0FF30072167
:10643000136050603970FEF78DBAB0EE667A62E78D
:10644000A14AA24B10681B689847079BDBED007AB6
:1064500093ED007A9E4B27EE277A97ED006A33443E
:1064600027EE287AD3ED007A9A4B67EE277AD3EDA0
:10647000005AB0EE467A984BF1EE656A83ED020A57
:10648000ACEE277AF4EEC76AF1EE10FA01DCC5FE35
:10649000C76A924B1B78012B02D0192B7BF442ACBC
:1064A000DFED8F7AB4EEE7CAF1EE10FACCBF01232C
:1064B0000023FBF742BCF0EE476A0FE7DFED897A75
:1064C000F4EEE7CAF1EE10FA3ADCDFED877AF4EE8B
:1064D000E7CAF1EE10FA33D4844B93ED007AF1EE73
:1064E000477AB4EEE7CAF1EE10FA35D48CFE47CA0B
:1064F0007F4B87ED00BA1B689342BBF6DBABFCF722
:1065000089BCCB5C002B7EF425AAFEF707BBDFF825
:10651000F891D9F800000DF0C7FC764B00221B78EB
:10652000C9F80020022B7EF413AA0CF0BAFFFEF784
:106530000FBAF0EE477A06E4B0EE677AFFF7EEBBEB
:106540009FED6DCAD4E7059900297FF4A3ADF4450A
:10655000B8BFB0EE675A9DE5B0EE67CAC8E70599C7
:1065600000297FF445ADF445B8BFB0EE675A3FE56A
:10657000059900297FF413ADF445B8BFB0EE675A12
:106580000DE5F0EE676A00E6802020F0C5FF0028E8
:106590007CF4AAAEFEF748BB452020F015F9FF2099
:1065A00020F012F9554820F0FBF8304620F00CF9A5
:1065B000FEF7FBB9059800287FF407ABF445B8BF98
:1065C000B0EE675AFFF701BBF0EE667AC8E5132B11
:1065D00005D1B0EE480A22F02DFEAAF80000B0EE78
:1065E000480AD5F87C3746489847464BB0EE408A73
:1065F0001B78132B7BF40AAA22F01CFEAAF80200D7
:10660000FBF704BA059800287FF40CAAF445B8BF3C
:10661000B0EE675AFFF706BA059900297FF411AD6D
:10662000F445B8BFB0EE675A0BE5059900297FF431
:106630008DACF445B8BFB0EE675A87E405990029E0
:106640007FF45BACF445B8BFB0EE675A55E40598EB
:1066500000287FF497AAF445B8BFB0EE675AFFF759
:1066600091BA059800287FF46AAAF445B8BFB0EE45
:10667000675AFFF764BA059900297FF414ACF44512
:10668000B8BFB0EE675A0EE4059800287FF434AA2C
:10669000F445B8BFB0EE675AFFF72EBA0598002848
:1066A0007FF407AAF445B8BFB0EE675AFFF701BA06
:1066B000059800287FF4DAA9F445B8BFB0EE675A10
:1066C000FFF7D4B9602E0120C08F0120D48F0120A4
:1066D000E48F01204C900120AC2E0120108A012073
:1066E0000000964200C0F84400C0F8C44890012061
:1066F0002C900120102F01200000000044E8030826
:10670000807D012028730120A0A4012044F620638D
:10671000974A984903442DE9F04F2DED028B91B033
:1067200014780B600590002C00F0CD86924B0599F3
:106730001B689942914B049340F28480013C1F688E
:106740008F49147007F480578E4CDFF878B20291AD
:10675000002F40F08280029B5B7D002B40F0398649
:10676000894B059A9A429BF8023000F21185002B62
:1067700040F01285854B0593049B1F6817F48059E0
:1067800040F0CB85029BB4F906605B8B9E42B4BFA0
:10679000002601267E4B1B6813F0805367D0059AB4
:1067A000127812F0010268D00299498C07EE901A13
:1067B0007849F8EEE77A91ED037A0391B4EEE77A3F
:1067C000F1EE10FA81F26D81002E5ED1724D95F8D6
:1067D0008810002959D171480025714900680D6061
:1067E00090F82D004D608D606E4900284ED10870E4
:1067F000002A4FD0F9064DD56B4A1278D20649D4FB
:10680000B9F1000F46D1002B44D17B0242D4674B33
:106810001B78002B01F0F087654B9B78002E42F02F
:1068200056803BB1634A644B12681B689B1A002B6D
:10683000C2F25E801020584D19F0F6FE012385F853
:10684000893027E01F684E4A07F480574D4C02926A
:10685000DFF870B1002F3FF47EAF00214C4803F009
:1068600086FB00287FF477AF1BF05EFD73E77802AC
:1068700095D4059A127802F001020021464D85F860
:10688000881044490391002EA5D046490120087084
:10689000002AAFD1494B1978002952D1029AB4F994
:1068A00000E0578B908B7745B4BF80220022B4F96B
:1068B0000250B4F904C042F040037045D8BF1346FB
:1068C000B4F906E09B0843F08002AF42B8BF13461C
:1068D00043F04002A842D8BF1A462F4D920895F8BF
:1068E0008A9042F080036745B8BF1A4642F04003E1
:1068F0006045D8BF13469B0843F08002BE45C8BF21
:10690000134643F040028645ACBF18461046814509
:1069100001F0B6820B46A5F88C1085F88E10234A3C
:1069200085F88A001778002F01F050825F2801F067
:1069300080826F2801F01181059B1B78D90741F1F6
:10694000D480049B1B6803F00403002B40F0D28723
:1069500000221B4D0DF1380840F6330AC8F8042018
:1069600005F15009192740F283360E922FE000BF3F
:10697000DC87012040860120D8870120FC7D012092
:10698000707F01205C9E0120404B4C00D08901208B
:1069900038A601200C740120382A0120C8340120B7
:1069A000B82E0120042A0120E4800120DF220120EA
:1069B000A82E0120A4A20120309D012054360120E0
:1069C0001C2F01200C9E012004354D4520D0AA78B3
:1069D000EB7817FB02619A42F6D26A7817FB0363E1
:1069E000043234F912205245A8BF5246B2F5617FF5
:1069F000B8BF4FF461728A42E6DD9A42E4DC29783E
:106A00002429E1D80435404603F0A2FA4D45DED1F1
:106A1000644A654B177898E8030083E80300002F69
:106A200000F09686614B079301215F4803F09FFABF
:106A3000002840F0AD829BF80330002B40F0A88284
:106A40005B4B06935B4E33881DB225F00105AFB258
:106A5000BB42378000F0D587574D4FF002084FF00A
:106A600014094FF0FF0A0E2085F8008085F8019088
:106A700085F802A019F0D8FD41464B48378803F04D
:106A800076FA002800F09E8227F0010292B2BA4204
:106A9000328009D00E2085F8008085F8019085F8B5
:106AA00002A019F0C1FD3788BB0741F16F80434B4D
:106AB000BD07434A1978506808BF81F00201089366
:106AC0000992C1F3400102F001FB2421364803F092
:106AD0004EFA30B9059A1378590702D523F004030A
:106AE0001370069B196811F00A0F1DD005212E485E
:106AF00003F03DFA002800F0A48735886B0741F1C8
:106B0000D6800621284803F032FA002800F0868754
:106B10006F0641F1E9800721234803F028FA002895
:106B200040F07A84069B1968880600F185843788CE
:106B30000C211D4803F01BFA002800F0568247F490
:106B40008073BB42338009D01B4B02201421FF22EB
:106B500018700E2059709A7019F066FD194B1B7849
:106B60000E2B00F04E82082B00F04B82049B1B681A
:106B7000580560D5144B1B79002B00F02681142199
:106B8000094803F0F4F9002840F0248111F050FB8B
:106B9000012019F08BFC0025DFF830A04FF0CC0964
:106BA00017E000BF3C3A012038A60120F8910120EF
:106BB000E0800120849E0120082D01203C930120CB
:106BC00040930120182F0120FC730120F4B801200C
:106BD000DDB209FB05F86B1C68B3022D2BD85AF8FF
:106BE0000870002FF4D1C3784FF0030ED1493A4614
:106BF00090F9020051F8233001210197CDF800E00F
:106C000018F044FF0346CC2205EB450039460693B5
:106C100053B100EB001001350AEB800024F025FC95
:106C2000069BEDB24AF808301FF062FC09FB05F83C
:106C30006B1C0028D1D1059B1D7815F0010500F0D3
:106C40001082BD4B01221A70079B4FF0010EB4F960
:106C500006101868B94F428987F800E0914280F227
:106C6000E6814FF07E52B64B1A60B64A029BB4F9E9
:106C700000E01F8B92F904301078002BAEEB070375
:106C800092F801C014BF01224FF0FF32002BB8BFB1
:106C90005B42B3F5FA7FA8BF4FF4FA73984280F2D3
:106CA000C3811B1A07EE903AF8EEE77A039BBE45C4
:106CB000C3ED007A03DAF1EE677AC3ED007AB4F936
:106CC00002E0AEEB0703002BB8BF5B42B3F5FA7FDF
:106CD000A8BF4FF4FA73984280F257821B1A07EE4E
:106CE000903AF8EEE77A039B7745C3ED017A03DD2E
:106CF000F1EE677AC3ED017AB4F90400C31B002BEF
:106D0000B8BF5B42B3F5FA7FA8BF4FF4FA7363458F
:106D1000CCBFA3EB0C030023B84202FB03F3039A9E
:106D200007EE903AF8EEE77AC2ED027A03DAF1EE76
:106D3000677AC2ED027A049B1A6812F4805200F05E
:106D40000182B1F5FA6F804BA8BF4FF4FA61187851
:106D5000B1F57A7FB8BF4FF47A71A1F57A71002846
:106D600040F0098279484FEAE17C794C6FF0630387
:106D700080FB018ECCEB6E1C0CF1010E03FB0C139F
:106D800034F91C1034F91E40641A03FB04F380FB31
:106D90000340DB17C3EB60130B441BB207EE903AC2
:106DA000039BB8EEE78A83ED038A002A40F046850C
:106DB00033885A0624D4002D40F0AE8018F0BFFC72
:106DC00011B0BDEC028BBDE8F08F059B1B78D90795
:106DD0007FF5DCAE3C2020F09FFB00283FF42BAF7A
:106DE0000DF08EF83C2020F039FB00283FF423AF53
:106DF0000DF086F83C2020F031FB0028F0D11AE796
:106E0000544B554AB3F90430544982FB0302DB1753
:106E10000988C3EBA203DFED526A9FED527A5B1A39
:106E20001BB207EE903AF8EEE77A67EEA67A77EEB5
:106E3000876ABDEEE66A16EE103A2033402B40F228
:106E40005F87DFED496ABDEEE77A17EE103A20332F
:106E5000402B00F251879FED457AF4EEC77AF1EEB0
:106E600010FA41F3E282DFED425A9FED426AF4EEFE
:106E7000C67A37EEE57AF1EE10FAF0EE477AF6DCF4
:106E8000DFED3D7AB4EEE77AF1EE10FA41F1E982F6
:106E9000DFED375A9FED396AB4EEC67A77EE257A80
:106EA000F1EE10FAB0EE677AF6D49FED2E7AF4EE9A
:106EB000C77AF1EE10FA00F30B869FED317AF4EE0B
:106EC000C77AF1EE10FA03D59FED2B7A77EE677A49
:106ED00067EEA75A9FED2B5A9FED2B6A9FED2B7AF9
:106EE000A5EE856A27EEA55AA5EE867AE5EE077A25
:106EF000039A92ED016AD2ED005A27EEC67A65EE4A
:106F0000A77AA5EEA67AE6EE267A82ED007AC2EDA1
:106F1000017A002D3FF452AF089B1978099B01F0CC
:106F20000101186802F0D2F811B0BDEC028BBDE887
:106F3000F08F00BF2CD90308D1890120342901200A
:106F4000E0290120842E0120A04E01201F85EB5155
:106F5000FC910120C4800120676666662C9D01209B
:106F600035FA8E3CDB0FC93F00000000DB0F4940C3
:106F7000DB0FC940E4CB1641DB0F49C0E4CB16C19F
:106F8000DB0FC9BF92E741B99730083C15A82ABE6C
:106F9000BC4B06931B6899077FF554ADBA4E3788F2
